:020000040000FA
:1000000092EF01F01200FFFF10EF04F01200FFFF6B
:1000100000000901C80E926F66806650010B06E071
:100020000901925103E009019207F7D7120000007D
:100030000901C80E926F66846650040B06E0090140
:10004000925103E009019207F7D71200D9CFE6FFDA
:10005000E1CFD9FF3F0E6816676A666AFE0EDB5075
:100060006712FD0EDB506812678AE552E7CFD9FFB1
:100070001200D9CFE6FFE1CFD9FFFE0EDB506A6E4A
:1000800067AE02D0FF0E30D00F0E671408080CE0E8
:100090000F0E67140B0808E06850040B03E168506A
:1000A000010B1FE0000E20D00F0E6714080804E0BB
:1000B0000F0E67140B0818E10901C80E926F685003
:1000C000010B04E0925102E09207F9D76850040B4B
:1000D00001E0010E496E1F0E66144910F7E166AC8F
:1000E00002D0FE0E01D0000EE552E7CFD9FF12007C
:1000F000D9CFE6FFE1CFD9FF0000FE0EDBCFE6FF50
:10010000B8DFE552006E005003E091DF005000D0F0
:10011000E552E7CFD9FF120000007ADF700EE66EDD
:10012000E7DFE552000901E028D0800EE66EE0DF4F
:10013000E552000901E021D0E66ADADFE552000964
:1001400001E01BD0400EE66ED3DFE552000901E06E
:1001500014D0016A1E0E015C0FE20150EA6A000F22
:10016000E96E060EEA22EF50E66EC2DFE5520009A4
:1001700001E003D0012AEED75ADF12000000016A25
:100180001E0E015C09E20150EA6A000FE96E060EDC
:10019000EA22EF68012AF4D712000000016A1E0E5D
:1001A000015C09E20150EA6A000FE96E060EEA22DC
:1001B000EF6A012AF4D712000000EFDFE66A080EAA
:1001C000E66E44DFE552E552090E696E21DF700EDE
:1001D000E66E8EDFE552000901E01CD0800EE66E6F
:1001E00087DFE552000901E015D0C80EE66E80DF1A
:1001F000E552000901E00ED0E66A7ADFE552000917
:1002000001E008D0E00EE66E73DFE552000901E080
:1002100001D00DDF12000000CFDF0601050E026FD6
:100220000601340E036F0601460E146F0601050E1B
:10023000176F0601040E186F0601640E196F060190
:10024000010E1A6F0601670E1B6F0601020E1C6F6E
:100250000601600E1D6F60DF1200000037D836D82F
:100260008D8A8D8C84848C80120009018E6B09012B
:100270008A07000E8B5B09018D5109018C5D04E03A
:1002800084948C908D9A8D9C8E2FFED709018D5170
:1002900009018C5D06E009018CB18C8009018CB3E9
:1002A00084848E2FFED78CC98DF9120000000900BE
:1002B000F5CF89F90900F5CF88F9090188510901BD
:1002C00086270901895109018723120000000901CD
:1002D000886B896B0901540E885D3D0E895905E2D2
:1002E0000901882B000E8923F5D7120000000901AF
:1002F000886B896B0901220E885D060E895905E21B
:100300000901882B000E8923F5D7120000008250C6
:10031000010B03E08250020B02E1010E02D0000E3D
:1003200000D01200C16A0F01DF0E256F0F01F70E1A
:10033000246F0F01E00E236F3A0EC06EEF0E896E30
:100340008A6A8B6A9E0E8C6E900E8D6E8E6A8F6A94
:10035000010E906E916AEF0E926E070E936E930EE1
:10036000946E600E956E030E966E7F0E976E060E5F
:10037000986EFE0E996E9A688A8AC79EC698C78C38
:10038000F00EC616C680C68A240EAC6E190EAF6E6D
:10039000900EAB6EF29EA698636AFE0E626E010E20
:1003A000616E7F9E7F9C7F84550E7E6EAA0E7E6E50
:1003B0007F82F28E01DFB0DE50DF0901916BA6DF94
:1003C000000904E10A0E0901915D09E2640E0901C8
:1003D000915D05E27BDF7ADF0901912BF0D77F94F5
:1003E00009019151630802E216EF02F00901866BE0
:1003F000876BF66A080EF76EF86A58DF000009018D
:100400008851891102E102EF04F050DF800EF618E6
:1004100005E1FD0EF71802E1010EF81801E0F5D72D
:1004200009018651871102E102EF04F001D81200A0
:10043000F2DE09018C6B09018BA703D00901010EC3
:100440008C6F13DF9EAA17D0AECF8FF9490E09012A
:100450008F5D0AE14B0EAD6E49DF580EAD6E46DF83
:10046000330EAD6E43DF02D08FC9ADFF440E0901DC
:100470008F5D01E101D0DDD709018A6B8B6B09012A
:10048000020E8C6F09018AA902D009018C6BEDDE86
:100490002FD8020EF85C05E1420EAD6EF86A0ED858
:1004A000FF000CD8410EAD6EEAD712000000550EC9
:1004B0007E6EAA0E7E6E7F8200001200940E7F6E0A
:1004C000F5DF000EE96E090EEA6E0A000901100E52
:1004D000846F0901080E856FEE50F56E0F00852FB1
:1004E000FBD7840E7F6EE2DF842FF3D77F94120058
:1004F00000000901906B0901846B09018451496E68
:100500004A6AD8904A5004E6840E495C000E4A5864
:1005100014E29EAAFED7AECF8FF909018451EA6A90
:10052000000FE96E090EEA228FC9EFFF09018F5112
:10053000090190270901842BE0D7090190510BE1B3
:10054000030E0901825D07E280C9F6FF81C9F7FF4A
:1005500082C9F8FF03D04E0EAD6ECBD71200FFFF5D
:10056000FFFFFFFFFFFFFFFFFFFFFFFFFFFFFFFF9B
:10057000FFFFFFFFFFFFFFFFFFFFFFFFFFFFFFFF8B
:10058000FFFFFFFFFFFFFFFFFFFFFFFFFFFFFFFF7B
:10059000FFFFFFFFFFFFFFFFFFFFFFFFFFFFFFFF6B
:1008000000001200280EE66E2EECFEF0E552CCEF52
:10081000FDF01200FFFFFFFFFFFFFFFFFFFFFFFFE5
:100820001EEF24F01200FFFFFFFFFFFFFFFFFFFF9F
:100830000000C6ECC9F09E0E496EDB0E4A6E010E3A
:1008400075EFD5F0C6ECC9F0050E496EDC0E4A6EA8
:10085000010E75EFD5F0C6ECC9F0EA0E4B6EDC0E5A
:100860004C6E010E4D6EFE0EDBCF4EF0CEECCBF09B
:100870008EECD9F0C2EFC9F0C6ECC9F0730E496E28
:10088000DA0E4A6E010E75EFD5F0C6ECC9F05E0EB9
:10089000496EDA0E4A6E010E75EFD5F0C6ECC9F05E
:1008A000D30E496ECD0E4A6E010E75EFD5F069EC90
:1008B000D5F0050D07ECD6F00A0E49260A0E4A229D
:1008C000FD0EDB504924E96E000E4A20EA6EEF501F
:1008D000C2EFC9F02EC1E6FFBEDFE5521200350EB1
:1008E0000124F0EFD3F0C6ECC9F0FC0E496ECE0E39
:1008F0004A6E010E75EFD5F07CEFCFF024ECD2F00C
:1009000024EFDBF0E4ECD4F024EFDBF0E80E496EEA
:10091000030E4A6E24EFDBF001015551050DF3CFB4
:1009200016F2F4CF17F202013C0E1703F3CF17F2C1
:100930001603F3CF16F2F45017271200E4ECD4F0AC
:1009400037C23DF038C23EF08EEFDAF0E66AD5EC01
:1009500026F0E5521200010E7EEFCAF0020E7EEF85
:10096000CAF087C2E6FFD3EFD8F0E66AD3EFD8F03B
:1009700001018AB73B0C300CD6ECD1F019E3E2EC64
:10098000D6F002E6F5ECD3F013E2D6ECD1F010E3AA
:10099000E2ECD6F002E6F5ECD3F00AE2D6ECD1F0C8
:1009A00007E3E2ECD6F002E6F5ECD3F001E2010C4D
:1009B000000C020E0101805D0BE2805102E0010E8D
:1009C00001D0000EE8B08A88E8B003D08A9801D040
:1009D0008A98070E936EF18E8051010803E2F19E12
:1009E000170E936E12002150100B08E0640E0201E6
:1009F0000B5D04E380ECCBF001E021981200E8EC01
:100A0000D4F00101AC6BB59F1200020E0101805DB4
:100A100003E18150100B06E0030E805D04E181507C
:100A2000100B01E0000C010CF0DF000901E1000CEB
:100A3000010156A1010CD70EF5ECD9F01E0803E216
:100A4000F00E005C01E3000C010C3C0EE66EE40EBF
:100A5000E66E010EF6ECC9F0BBECD2F006E19CECC0
:100A6000D0F003E001011E0EAC6F66C100F03DEC5A
:100A7000CFF00A0E665D02E2200E1A6F1200350EEC
:100A8000E66EE40EE66E010EF6ECC9F0BBECD2F0B9
:100A900006E19CECD0F003E001011E0EAC6F67C1D3
:100AA00000F000500FE00101030E016F7EECE1F059
:100AB00001012D0E196F0A0E675D04E2200E196FF9
:100AC0002D0E1A6F12002E0EE66EE40EE66E010E6B
:100AD000F6ECC9F068C100F000500AE00101030E15
:100AE000016F3DECCFF00A0E685D02E2200E1A6F36
:100AF0001200010148511200800E071403E020503B
:100B0000010B01E0000C010C800E071406E02050E0
:100B1000010B03E10201215101E0000C010C020173
:100B2000010E3A6F7E0EDFECCAF001011E0EAC6FB3
:100B3000120012EFD3F069ECD5F004080FE0E9ECF5
:100B4000CAF00EE0FE0EDB500A0808E0FE0EDB5095
:100B50000D0804E0FE0EDB50090802E1010E01D091
:100B6000000EC2EFC9F007019551D880945502E2FA
:100B700094C795F794079251922BEA6A000FE96E99
:100B80000C0EEA22EF5012000101E651100B03E0B7
:100B90000401FA510AE1420EE66E460EE66E4DEC95
:100BA000A1F0E552E5520101E6891200D9CFE6FF36
:100BB000E1CFD9FFFE0EDB50D80805E1300EF36E11
:100BC000FE0EF3CFDBFF060EAB1406E0AB98000081
:100BD00000000000AB8840D1FE0EDB50100805E09D
:100BE000FE0EDB50110801E037D10201050E146F33
:100BF000FE0EDB50110837E1020124510DE12050B7
:100C0000800B0AE1050105014751010B0AE10501CD
:100C100005014751400B05E1100EE66E8FD9E552F4
:100C200022D0050105014751400B02E00F0E01D013
:100C3000060EE66E83D9E552C4C1E6FF7FD9E552C0
:100C4000C5C1E6FF7BD9E552C6C1E6FF77D9E552BB
:100C50000A0E0101C703F3500101C825E66E6ED9E3
:100C6000E552050147910401F051496E4A6A4A3440
:100C700004E24950D208000E4A5405E20701042B51
:100C800007010407E9D00501475104E10501485176
:100C900001E1E2D00201245101E0DED02050800BBE
:100CA00001E0DAD00490050148A10BD04E0EE66EAB
:100CB000420EE66E4DECA1F0E552E5520501486B9F
:100CC000CBD0050147A11AD001010101E651080B63
:100CD00003E00401FA510DE1410EE66E460EE66EA8
:100CE0004DECA1F0E552E5520101E687050147B35D
:100CF0004BDF0501479305014791AED0050147A39E
:100D000004D042DF05014793A7D0050147A726D0AD
:100D1000440EE66E4D0EE66E4DECA1F0E552E55246
:100D20000480440EE66E4D0EE66E4DECA1F0E552E9
:100D3000E552030E0101D45D04E0030E0101D55D0F
:100D400008E1540EE66E440EE66E4DECA1F0E5525D
:100D5000E55205014797050147857ED0050147A566
:100D600024D0570EE66E420EE66E4DECA1F0E55231
:100D7000E5520480570EE66E420EE66E4DECA1F091
:100D8000E552E552530EE66E490EE66E4DECA1F0CB
:100D9000E552E5524A0EE66E460EE66E4DECA1F0C7
:100DA000E552E5520501479557D0050147A90BD0FB
:100DB000410EE66E500EE66E4DECA1F0E552E552A6
:100DC0000501479949D0050147AB0BD0410EE66EAE
:100DD000520EE66E4DECA1F0E552E5520501479B3F
:100DE0003BD0050147AD13D04F0EE66E520EE66EB6
:100DF0004DECA1F0E552E552540EE66E520EE66E51
:100E00004DECA1F0E552E5520501479D25D00501C5
:100E100047AF22D04E0EE66E4C0EE66E4DECA1F0C2
:100E2000E552E552560EE66E440EE66E4DECA1F02C
:100E3000E552E552420EE66E530EE66E4DECA1F021
:100E4000E552E552570EE66E430EE66E4DECA1F00C
:100E5000E552E5520501479F200EF36EFE0EDBCFF3
:100E6000F4FFF350F45C04E3FE0EDB507E0807E26F
:100E7000FE0EDBCFE6FF5FDEE552000944E0040131
:100E8000F051496E4A6AD8904A5004E6FF0E495C18
:100E9000000E4A5838E2FE0EDB503B0804E0FE0E1E
:100EA000DB507C0802E10401F92BFE0EDB50210827
:100EB00004E0FE0EDB5040080AE13B0E0401FE5D3B
:100EC00004E07C0E0401FE5D02E10401F92BFE0E3C
:100ED000DBCFFEF40401F151EA6A000FE96E0B0E5C
:100EE000EA22FE0EDBCFEFFF0401F12B0401F02B11
:100EF0000401F05108E10401FE6BFEC4F9F4FEC4E4
:100F0000F1F4FEC4F2F4E552E7CFD9FF1200ACA22F
:100F100012000401F85143ECD6F0006E0050E66E6A
:100F200019ECCFF000C0EFFF3B0E005C03E07C0E3D
:100F3000005C01E129900401F82B1200C6ECC9F015
:100F4000ACA2FED779ECD5F019ECCFF0FE0EDBCFDA
:100F5000EFFFC2EFC9F08BEC10F0010EE66EA0ECD3
:100F600010F0E55284948C908D9A8D9CF29E000036
:100F7000F66A080EF76EF86A940E7F6E550E7E6E56
:100F8000AA0E7E6E7F82000000EC00F012000401C9
:100F9000F007F251EA6A000FE96E0B0EEA22EF50F9
:100FA000006EF22B12009CECCAF00AE11F50020BFB
:100FB00007E102018951020B04E18951010B01E1B2
:100FC000000C010CD9CFE6FFE1CFD9FFE65220504B
:100FD000200B01E176D08250010B03E18250020B1D
:100FE00003E02F50400B6DE00101E7890601880EF8
:100FF000FD6F130EFE6F33AC45D08BEC10F0060185
:10100000880EFD6F130EFE6F010EE66EA0EC10F061
:10101000E55285EC96F033AC2DD00601880EFD6FBD
:10102000130EFE6F0101016B260EE66EE40EE66EF6
:10103000010EE66E25ECE2F0E552E552E5526EEC6B
:10104000DFF0010EE66EB3ECE4F0E552000901E0DA
:10105000FF00500EE66E87ECFDF0E5528250010B6A
:1010600008E18250020B05E10101E79985EC96F059
:10107000FF00D1D70601880EFD6F130EFE6FD1EC75
:1010800010F01FD02F9C8BEC10F0010EE66EA0EC40
:1010900010F0E5526CECDBF07CECDBF01E0EE66E43
:1010A000E40EE66E010EE66E25ECE2F0E552E55246
:1010B000E5526EECDFF00101E79985EC96F0D1EC9A
:1010C00010F0E552E552E7CFD9FF120043ECD5F01E
:1010D000DF6A880E4C6ED00E4D6E010E4E6EFD0E08
:1010E000DBCF4FF0506A516A090E416E426A436A83
:1010F0004FC03CF050C03DF051C03EF0B6ECF9F0AE
:1011000039C04FF03AC050F03BC051F0B3ECD0F0D2
:10111000DFCF52F0536A546A59ECCEF00800F5CF95
:1011200000F0F5500DE0090EDF5C0AE2FE0EDB5028
:1011300003E1ECECE1F002D00FECE2F0DF2AC9D7DA
:10114000E552C2EFC9F02750200B06E0050110510F
:10115000020119112D1101E1000C010C0101E651F0
:10116000400B0CE00201685109E1080E155C07E034
:10117000290E155C04E00A0E155C01E0000C010C60
:10118000C7EC21F0FAECD3F02D6B3751381102E0A7
:1011900020944DDA4DEF65F00701BE51010B07E0D9
:1011A00019ECCCF004E0050ED45D01E0000C010C5C
:1011B0000101269D010E0D6E26BF0D681200030E63
:1011C0007EECCAF0258E12006A0E2CEFCAF06B0E70
:1011D0002CEFCAF001018E51010B08E032EC0FF048
:1011E000000904E001013B51800B01E0000C010CFF
:1011F000040E7EECCAF001013C0EAC6F120001013E
:10120000AC510DE12DAC08D00F0EE66ED40EE66E9B
:10121000010ED1ECCDF001D0EBDF258E2D8C12002C
:10122000258E050E7EEFCAF07AECCCF000010E6E32
:10123000E66AE5ECD6F00F6E120087C1E6FFA80E55
:101240000AECCAF093C100F0EBECD4F007E10A0E0F
:1012500001019503F350FE0BE842006E0050E66E6C
:10126000A90E0AEFCAF0C6ECC9F0FE0EDB50E3ECA3
:10127000CAF0EF500BE1FE0E43ECCBF007E35DEC60
:10128000D1F0E3ECCAF0100EEF6EEFD7C2EFC9F069
:10129000C6ECC9F0FE0EDB5068ECCBF0EF50300826
:1012A0000BE1FE0E43ECCBF007E35DECD1F068EC14
:1012B000CBF0200EEF6EEED7C2EFC9F0830E096EB1
:1012C000FA0ECBECCBF000500E6E0EC00FF00E6A93
:1012D000FB0E4DECDBF000503EEFCCF03AC18BF250
:1012E000120001013A51130804E2010E3A6F2BA6D5
:1012F0003A6B39EFBCF069ECD5F0020802E1BAC7ED
:10130000B9F7FE0EDB0402E1B9C7BAF7C2EFC9F0C4
:10131000F9ECD7F04BEFD2F042C1ABF242C1AAF2E6
:10132000F9ECD7F0EF50400B03E00201020EAA6F78
:101330000101D5512CECCBF0EF50400B03E0020142
:10134000020EAB6F120043ECD5F02850010B17E1F1
:1013500063ECD1F016E14A5014E11750010B03E0A1
:101360001C0E155C0CE01750100B03E0150E155CFD
:1013700006E01F50100B05E00C0E155C02E1000E9C
:1013800001D0010EDF6E2C50800B03E12C50400B7E
:1013900002E0010EDF6E2890DF50E552C2EFC9F087
:1013A0001A9C238A12000101E38B11C512F5050175
:1013B000106B279A1200EAECD0F01EE00901E6510A
:1013C0001BE034ECD7F0E6C9E6FF75EC10F0E5520F
:1013D0000901E75105E0E7C9E6FF75EC10F0E552B9
:1013E0000901E76BE7C9E6F9010136990450010BE1
:1013F00001E03689E4EF08F0010136AF05D004A022
:1014000002D01A8812001A8A1200C6ECC9F0EAEC5F
:10141000D0F00CE0FE0EDB5009E0C5DFBAECD7F0EF
:101420000901E6AF02D001013689CEDEC2EFC9F074
:10143000C6ECC9F0EAECD0F011E0FE0EDB500EE095
:10144000FD0EDB500BE0AFDFBAECD7F018ECD3F0B9
:10145000FE0EDBAE02D001013689B6DEC2EFC9F066
:10146000C6ECC9F0010136AD12D034ECD7F0BAECBD
:10147000D7F0FD0EDB5002E018ECD3F001013699F5
:10148000FE0EDBBE3689DB5008E09EDE06D0FE0E87
:10149000DBAE02D01A8801D01A8AC2EFC9F05CEC28
:1014A000DAF0DBCFFBF60201D25101E105D80201EF
:1014B000190ED26FC2EFC9F047ECD5F0010EFBC692
:1014C000DBFFEAECD0F062E02050200B5FE0060189
:1014D000FB51FC5D5BE067DF77DE01013689890E39
:1014E000C9ECCAF00101E3A50BD0530EC9ECCAF058
:1014F000570EC9ECCAF0520EC9ECCAF00101E395CF
:10150000640E11ECD6F0D8ECD8F0DF50300805E2CC
:10151000DFCFE6FF75EC10F0E552640EBDECD0F0C5
:101520003AC0DBFF6BECCAF0D8ECD8F00101E7A5BC
:1015300003D0520EC9ECCAF0DF50300808E30601B0
:10154000FB51630804E30101E751040B08E0300E8E
:10155000DF5C02E1540E01D0DF50C9ECCAF001019A
:10156000E7A303D0520EC9ECCAF06BECCAF0010E2F
:10157000DBCF3EF0EFECD4F0300FDF6E300EDF5CEF
:1015800002E1540E01D0DF50C9ECCAF0FBC6FCF6F4
:10159000020EE15C02E2E16AE552E16EC2EFC9F0DF
:1015A000690E2CEFCAF0060EA4ECD6F0280EF1EC72
:1015B000C9F0D0EF0AF0010136BFF5DF12000601D5
:1015C000980ED880B0553A0EB15509E20E50B05D74
:1015D0000101D86F0F500601B159010108D0B05177
:1015E0000E240101D86F0601B1510F200101D96FFE
:1015F0001200190E3D6E3E6A0EC042F00FC043F05D
:1016000098ECF9F03BC037F23CC038F2180E426E4D
:10161000436A37C23DF038C23EF0E2ECFDF03DC017
:1016200037F23EC038F21200EB0E2CEFCAF0010187
:10163000E693199A139209EC19F0F6DF0201376B61
:10164000386B1994CEEF0CF0E0ECA7F00A0EF1EC39
:10165000C9F0E30E76ECCBF0006E0050F5E112001D
:10166000C6ECC9F0F1DFEC0EFDECD7F007EC74F03E
:1016700000C709F0FC0E016E0FC000F0F9EC3AF063
:10168000012A0EC000F0F9EC3AF0096AC2EFC9F085
:10169000660E2CECCAF019801200670E2CECCAF012
:1016A0001990120043ECD5F044EC20F0DF6EBFEC53
:1016B000D2F007E019A00ED0F0DFDF500BE1006A96
:1016C00007D019B007D0E4DFDF5004E1010E006E4F
:1016D0003DEC75F0E552C2EFC9F083ECCAF003E0CF
:1016E0003450400B04E001015751040B01E1000CA0
:1016F000010C43ECD5F001018AA10AD044EC20F0A2
:10170000DF6EDF0403E0020EDF5C02E1010E01D0B8
:10171000000EE552C2EFC9F0ECDF000905E144EC30
:1017200020F0040801E0000C010CF6DF000904E1E0
:10173000C3ECD2F001E0000C010C43ECD5F01E50DC
:10174000010B0EE01EECCDF00BE083ECCAF003E0E1
:10175000EEECD0F005E11950020B02E1000E01D0D1
:10176000010EDF6EDF5002E08CEC04F0DF50E5523A
:10177000C2EFC9F043ECD5F01D50040B1AE01D5028
:10178000080B17E01E50010B14E01EECCDF011E029
:10179000050110510EE12050040B0BE12050010B0C
:1017A00008E183ECCAF003E0EEECD0F002E1000EB9
:1017B00001D0010EDF6EDF5002E08CEC04F0DF5050
:1017C000E552C2EFC9F08A0E98ECCEF0010136ADB9
:1017D00005D0410EE66E4E0E57EFCAF036BF258E8D
:1017E000120047ECD5F0C20EDE6E010EDD6E44EC49
:1017F00020F0010804E044EC20F002080BE1F40EB4
:10180000DE6E010EDD6E0101345104E0260EDE6E47
:10181000020EDD6EE4ECD5F00CE001ECD8F0020134
:101820000051495C01514A5804E2DECF00F2DDCF9D
:1018300001F201C2E6FF00C2E6FF740EECECC9F053
:10184000020EE15C02E2E16AE552E16EC2EFC9F02C
:101850001D9CDBECD1F0BBDCE50E98ECCEF0258EC8
:10186000120069ECD5F00A0DF3CF5AF3F4CF5BF315
:10187000000E03015A27030E5B23C2EFC9F06B0E63
:10188000005C05E20201AA510101245F1200E2ECB2
:10189000D6F004E6990E495C000E4A5804E20201B3
:1018A000AA510101242712001200280E0101D8803C
:1018B0006855040DF328016E0150E66EAA0E0AEF7A
:1018C000CAF0C6ECC9F02AA40AD0EEECCBF0CBECFF
:1018D00026F03DECDAF00101500EAC6F2A94C2EF15
:1018E000C9F0149E0A01DA51800B03E19CECCAF0A6
:1018F00001E1148E12000201996999C28BF799C215
:101900008AF799C289F799C288F799C287F70701C0
:10191000906991698E698F698EC78CF78FC78DF733
:101920001200040E0101805D03E18150100B07E0FD
:10193000050E805D03E18150100B01E1000C010CEC
:10194000120043ECD5F00101A85103E19E5120089B
:1019500021E2DF6A090EDF5C10E2DF50F8ECCBF029
:10196000EF50040B08E0100EDF24E66E0BEC2DF0B8
:10197000E552000902E1DF2AEDD7090EDF5C0AE239
:10198000100EDF262986DFCFE6FFC9EC2CF0E552EA
:10199000DF5001D0000EE552C2EFC9F01F86DBEC2C
:1019A000D1F0B599B59B2582238A1200D9CFE6FFE5
:1019B000E1CFD9FFE6528C9600000000FE0EDBCF8F
:1019C000E6FF8DEC5CF0E5520000C950DF6E0000D0
:1019D0008C86030EE66E57ECFEF0E552DF5000D029
:1019E000E552E552E7CFD9FF12009AEC5CF0F00E19
:1019F000C616C680C68A1200800EE66EC7ECD2F00C
:101A0000EBECFCF03DECDAF0F5EF0CF0128212801A
:101A10000601019102011E0E306F120012901FA2EA
:101A2000128012921FB21282120088ECD6F02CECB7
:101A3000CBF0EF50E840E8403F0BDF6E000EDF9444
:101A4000DF96DF98DF9ADF9CDF9E0A0E006EFE0EA7
:101A5000DB500DE1DF5002E1010E006EDF0402E118
:101A6000020E006E020EDF5C44E1050E41D0FE0E58
:101A7000DB50030804E1DF5002E1010E006EFE0EB0
:101A8000DB5004080EE1DF0402E1320E006E020EAC
:101A9000DF5C02E15A0E006E030EDF5C02E1640EB1
:101AA000006EFE0EDB50050810E1320E006EDF0402
:101AB00002E1640E006E020EDF5C02E17D0E006E3C
:101AC000030EDF5C02E1FA0E006EFE0EDB0404E0A2
:101AD000FE0EDB5002080DE1DF5002E1010E006E48
:101AE000DF0402E1050E006E030EDF5C02E1190E59
:101AF000006EE552C2EFC9F0C9ECD8F0C4C100F0E5
:101B0000000406E10101C551460802E2020E006E22
:101B1000030E005C06E10101C551280802E2040E33
:101B2000006ED5CA03F028ECD2F005E03751080B5F
:101B300002E0040E036E980E4A6ECC0E4B6E010E40
:101B40004C6E0050CEECCAF0035043ECCFF0EF5097
:101B50004924016ECF0E4A6ECC0E4B6E010E4C6EB8
:101B60000050CEECCAF0035049ECCFF0EF504924BE
:101B7000026EF9ECD9F0E66A7D0E28ECCCF0C9ECE7
:101B8000D8F0280E026E016E28ECD2F00EE037512C
:101B9000080B0BE01CCA01F021CA02F0015002E060
:101BA000025003E1280E026E016EF9ECD9F07C0EB2
:101BB000ECECC9F0C9EFD8F0129A1FB2128A2EDFEE
:101BC000FFECD3F0DDEC69F01F50020B06E00101E1
:101BD000D551D45D02E01A8C12001AAC02D0D0ECC0
:101BE00009F01200080E0B5C04E3E4ECD5F001E10F
:101BF000000C010C095004E00701010E02ECD7F0C3
:101C0000096ABCEC04F0000907E0750EE66E280EC8
:101C1000E66E010E93ECD9F01200BCEC04F0000962
:101C200009E07E0E096E080EE66EB60EE66E020E36
:101C300093ECD9F0096A12005CECDAF0DBCF48F1E2
:101C400097ECD9F0E0ECD1F0FAECD3F01398C2EFB6
:101C5000C9F00101485112E0060E11ECD6F048C15E
:101C60003EF04BECD8F0006E005001E1002A00502D
:101C70000101485F48C15BF24DEFCCF0209430EF9A
:101C8000CEF007015A5106E1080E76ECCBF00501C3
:101C9000261501E1000C010C2C9E2C9C81EC2EF0F1
:101CA000D9EF96F0C6ECC9F003ECD4F007E12B5065
:101CB000010B04E101018A51200B09E140C243F20A
:101CC0003FC242F23EC241F21FECD3F009D0FE0EF9
:101CD000DB5006E043C240F242C23FF241C23EF254
:101CE00004802BA002D004902B90DCEC40F001018A
:101CF000320EAC6FC2EFC9F025B41200189A17B8B3
:101D0000188A12000301916B926B936B946B91C3D1
:101D10008DF392C38EF393C38FF394C390F3030EAA
:101D2000016EFF0E015C32E0056A030E026EFF0ECB
:101D3000025C22E00250EA6A890FE96E030EEA2291
:101D4000EF504B6E4C6A0150EA6A850FE96E030E44
:101D5000EA22EF5057ECCDF0FEECD0F0EF503EEC25
:101D6000CCF005503EECCCF0FEECD0F00EC0EFFF16
:101D70000FC005F00206DBD70150EA6A8D0FE96E4D
:101D8000030EEA2205C0EFFF0106CBD7120069EC73
:101D9000D5F0006E00AE04D0006C01010E0E116F84
:101DA0000101040E08ECD4F012510AE111C112F144
:101DB000100E116F135104E112C113F1100E126FC6
:101DC000130E156FC2EFC9F019ECCCF003E1030E4E
:101DD0000A5C01E0000C010C19ECCCF005E1020EEC
:101DE0000A5C03E00A0401E0000C010C19ECCCF0E1
:101DF00003E1020E0A5C01E0000C010C19ECCCF0CE
:101E000007E10A5005E1CF51040B01E0020C010C7F
:101E1000000C19ECCCF005E1020E0A5C03E00A04A8
:101E200001E0000C010C0601EC5106E019ECCCF0CD
:101E300003E10A50000801E3000C010C19ECCCF09E
:101E400004E10A0403E00A5001E0000C010C19EC63
:101E5000CCF006E1020E0A5C04E0030E0A5C01E02D
:101E6000000C010C83ECCAF003E0CFECD2F001E1EE
:101E7000000C010C0101D45104E10A01DA51040BF8
:101E800001E1000C010C0101D45104E10A01DA5115
:101E9000080B01E1000C010C2CECD2F009E003016D
:101EA000B85151ECDBF0E5ECCBF0210EECECC9F0D5
:101EB00012002CECD2F002E04CEF0FF0E66AE66A7A
:101EC000210EECEFC9F019ECCCF010E1D051040B6D
:101ED00005E00A040CE0020E0A5C09E0CF51040B95
:101EE00005E00A5004E0030E0A5C01E0000C010C5E
:101EF0000101D45103E1D051400B04E1E4DF0009BA
:101F000001E1000C010CF2ECD0F001E0030CF3EC69
:101F1000D4F001E0080C30ECD2F001E11B0CD451FC
:101F200009E0030ED45D05E10A5004E0030E0A5CEB
:101F300001E0030C010CF2ECD0F001E00A0CF3EC30
:101F4000D4F001E0380C30ECD2F001E1640CD45153
:101F500001E0500C380CEFDFE66ED5DFE66ED60EF2
:101F6000E66E0A0E04EFCAF06FEC41F0190E012480
:101F70000A01D880D75503E2190E0124D76FD3EC9C
:101F8000D2F0D75D03E2D3ECD2F0D76FD46B3388B5
:101F90004FEFCFF0F2ECD0F004E1F3ECD4F001E13C
:101FA000000C010CEF0E896E8A6A8B6A9E0E8C6E95
:101FB000900E8D6E8E6A8F6A010E906E916AEF0E92
:101FC000926E070E936E930E946E600E956E030ED6
:101FD000966E7F0E976E060E986EFE0E996E9A683C
:101FE00012001F98258A0101B59B02011A511FE0BA
:101FF000020E685D03E1D7ECD2F019E00701BE9B49
:10200000BE9B32BCBE8B88EC09F00601EA05EB6F83
:10201000020EEA5D01E2EB6BEBC600F00101D45168
:1020200002E0EDC600F00050E66E79ECD6F0020159
:102030001A6B25821200C08EA70E1BECCDF00DECA2
:10204000D4F0A70E1BECCDF0C3500E26C4500F22C7
:102050000EC04DF00FC04EF0D8904E324D320EC033
:102060004FF00FC050F0D89050324F32D8905032CD
:102070004F324D504F244B6E4E5050204C6E0EC080
:1020800051F00FC052F0040ED89052325132E80491
:10209000FBE151504B5C496E52504C584A6E0EC099
:1020A00053F00FC054F0060ED89054325332E80467
:1020B000FBE1495053240E6E4A5054200F6E0EC05F
:1020C000CDF20FC0CEF2C09E1200CDC20EF0CEC235
:1020D0000FF0E66A88EC26F0E5520101200E166F3B
:1020E0001C6F188F410E1B6F1200C6ECC9F0050162
:1020F0001151EA6A000FE96E080E06ECD8F0112BB8
:10210000115161ECCAF002E612ECD4F001E3116B5C
:10211000102BC2EFC9F0BCEC04F0000910E007EC92
:10212000CDF0020E0101395D02E1010E396F62DD71
:1021300074EC48F072DD7FEC48F021EC79F012008D
:10214000C6ECC9F00101E7890601880EFD6F130E88
:10215000FE6F71EC16F08A988A8639EC25F0010141
:10216000766B140EE66EF7ECC2F0E552FE0EDB5015
:102170000CE04DEC0BF0D0EC0AF036ECC4F0D5ECF2
:10218000C4F086ECE2F0D0ECE0F00601506B78ECA5
:102190003DF00601516B0101B96BEF0E926EC2EF7B
:1021A000C9F0F29E62ECFEF0F26AF06AB96A9D6ACA
:1021B000000EA66EA16E9E6E8D8C8D8A8C9084848E
:1021C000070E936E0000000000008A9A00000000D5
:1021D00000000000270E936E4E0E996E0000000066
:1021E000000003000000000000000000FF001200DB
:1021F00043ECD5F020AA3BD017ECD4F006E3CCECAE
:10220000D8F035E2E5ECD1F032E21B50080B2FE1BB
:1022100017ECD4F006E3CCECD8F029E2E5ECD1F0F1
:1022200026E217ECD4F006E3CCECD8F020E2E5ECA3
:10223000D1F01DE20050DF6EDF5037ECCBF013E23F
:10224000E5ECD1F010E2DF501CECD4F004E6B40E63
:102250004B5C000E4C5807E2160EE66EE40EE66E7E
:10226000010E26ECD3F0E66A6BDFE5529ADFE55209
:10227000C2EFC9F0C6ECC9F07CECDBF0EEECCBF0C1
:102280005DECCAF06EECDFF06EECCDF06EECCDF0F4
:102290006EECCDF0FA0E06ECD7F0FA0E06ECD7F0A5
:1022A000C2EFC9F00DECD4F034ECD2F034ECD2F043
:1022B000460E07ECD1F00F50496E4A6A9F0EBFECF4
:1022C000D7F0006E0050800801E2006A0201FC0EA7
:1022D000D880CD55080ECE5502E2040E0FD0080E60
:1022E000D880CD55070ECE5502E2030E07D0140E4E
:1022F000D880CD55050ECE5503E2020E002607D03C
:10230000200ED880CD55030ECE5501E2002A005094
:10231000800801E2006A080ED880CD55070ECE5520
:1023200002E2030E07D0140ED880CD55050ECE550F
:1023300003E2020E00261200200ED880CD55030EB7
:10234000CE5501E2002A120047ECD5F0C08EAF0E48
:102350001BECCDF0010157A9C5D0500ED880C35455
:10236000050EC45401E3BAD0D00EC35C0A0EC458A3
:1023700001E3B4D03C0E496E4A6ACDC23DF0CEC2F4
:102380003EF08EECDAF000503C0802E23C0E006EAB
:102390004FECDAF007014950C35CD06F4A50C45883
:1023A000D16F140ED05F050ED15B010157AB9AD0EF
:1023B000D0C7D8F1D1C7D9F121ECD4F0070E5BEC2E
:1023C000D0F0FDE16A0E4924096E21ECD4F05DECF9
:1023D000D8F0ABECCDF00101E7AF10D0E79FC80E0D
:1023E000A0ECD0F004E3840E5FECD0F002E2070131
:1023F00019D00EC0D2F70FC0D3F76DD0C80EA0EC25
:10240000D0F004E3840E5FECD0F011E20701C80EB7
:10241000D25D000ED35906E3840ED880D255030E48
:10242000D35560E2260ED26F020ED36F54D0010E48
:1024300007014A6AD225496ED3514A220BECD7F0E4
:102440000CE3D2C74BF0D3C74CF04B06000E4C5AEE
:102450004B500E5C4C500F5845E20101D4510CE139
:1024600007010E50D25D0F50D35903E2D22B000E5C
:102470001CD0D207000E2ED007010E50D25D0F5097
:10248000D35915E2D2510E5C0101D86F0701D35127
:102490000F5853ECD2F003E2050ED86FD96BD85128
:1024A0000701D2270101D9510701D32314D00E50BF
:1024B000D25D0101D86F0F500701D35953ECD2F010
:1024C00003E2050ED86FD96BD8510701D25F010125
:1024D000D9510701D35B20EC32F004D00701060E7E
:1024E00002ECD7F0A0ECCAF00701A7274A50A823B6
:1024F000A7C749F0A8C74AF010ECD7F00701A75FBB
:102500004A50A85B080ED880C354090EC45462E335
:102510000DECD4F00B0E07ECD1F0040E34ECD2F03D
:10252000E804FCE1360ED8800E56060E0F56CDC2DA
:1025300049F0CEC24AF05BECD0F0FDE149500E26E6
:102540004A500F2220BA0ED0B2C249F0B3C24AF0AC
:1025500010ECD7F00201B25F4A50B35B0E50B227C5
:102560000F5013D0B2C249F0B3C24AF0640EE0EC8F
:10257000C9F049500201B25F4A50B35B0CECD6F08F
:1025800010ECD7F00201B2274A50B323020E4A6A78
:10259000B425496EB5514A22B251495CB3514A58EB
:1025A00013E3020ED880B455000EB55513E2B4C241
:1025B0004BF0B5C24CF0020E4B5E000E4C5A4B5025
:1025C000B25D4C50B35906E220EC32F0B2C2B4F224
:1025D000B3C2B5F2C09EEDECCAF002E2E16AE55288
:1025E000E16EC2EFC9F047ECD5F0C08EAB0E1BEC2C
:1025F000CDF0A0ECCAF00701A9274A50AA23A9C729
:1026000049F0AAC74AF010ECD7F00701A95F4A5079
:10261000AA5BC09EEDECCAF002E2E16AE552E16E0F
:10262000C2EFC9F047ECD5F0070114A108D014910E
:102630005BECD5F07D0E976E060E64ECD8F0C08E84
:102640009B0E1BECCDF0A0ECCAF00701AB274A5063
:10265000AC23ABC749F0ACC74AF010ECD7F0070188
:10266000AB5F4A50AC5BC09EEDECCAF002E2E16A9F
:10267000E552E16EC2EFC9F069ECD5F007E1C00E9A
:10268000016E01015FA304D0E00E01D0B00E016E17
:1026900001010D51012637EC3BF0FE0EDB5013E03B
:1026A0000F0E005C03E3005030080DE2230E006EB5
:1026B0000901EB5108E0020E0101395D04E0090156
:1026C000EB51B4ECD5F00050C2EFC9F043ECD5F0BB
:1026D0007BEC0CF09CECCAF008E10701B16B0A013D
:1026E000D56BDA930BEC75F012D0D6ECCDF0EFCFC2
:1026F000B1F7D4C1DFFFD5CA00F0080EE66EE66A76
:10270000DF5067ECD6F026ECD4F0E3ECCCF0149C70
:102710000101D45103E0030ED45D06E1030E0A016A
:10272000D45D07E1148C05D0020E0A01D45D01E1ED
:10273000148CDAA304D0D8CAB6F7D9CAB7F71CEC00
:1027400019F0F9ECD7F0EFCFBEF70701BE9F0101FA
:10275000D45103E0030ED45D02E10701BE8F1AECF1
:102760001FF052ECCCF083ECDFF044EC25F08CEC65
:1027700009F0E552C2EFC9F0ABECDAF067ECD6F045
:10278000E3EFCCF0F9ECD7F04BECD2F09CECCAF0D4
:102790000FE00A01DAA306D0B6C7D8FAB7C7D9FA4C
:1027A0001CEC19F0E9DF0101D6ECCDF0B1C7EFFF69
:1027B000120043ECD5F0DF6A080EDF5C04E2DFECC8
:1027C000D8F0DF2AF9D7E552C2EFC9F043ECD5F0D3
:1027D000DF6A080EDF5C0CE251ECCBF0EFCF49F082
:1027E000FE0EDB50495C02E1010E03D0DF2AF1D777
:1027F000000EE552C2EFC9F0C6ECC9F018BE08D011
:1028000079ECD5F073EC04F0E5527F0B72ECCAF072
:10281000C2EFC9F0C6ECC9F018BE15D029A003D08C
:1028200087EC07F0FBD725ECCFF00DE025ECCFF0DF
:1028300072ECCAF0D950FC0F0BECD8F0EE2A000E67
:10284000EE22EE22F0D7C2EFC9F0C6ECC9F018BEF6
:1028500025D029A003D087EC07F0FBD7B6ECCBF04E
:10286000E80E426E030E1DECCCF0492472ECCAF067
:10287000BDECCBF0ECECD8F0B6ECCBF0640E78EC21
:10288000D7F0640EE6ECD8F00A0E78ECD7F00A0E1A
:10289000E6ECD8F0300E492472ECCAF0C2EFC9F071
:1028A000C6ECC9F018BE0FD01EAE0DD0110EE66EEC
:1028B000E40EE66E010E27ECCAF0EEECCBF0AADFD8
:1028C000E552E552E552C2EFC9F043ECD5F0020102
:1028D000CF2B1EAE19D0290EE66EF20EE66E010E5B
:1028E000C4ECCAF079ECD5F087DFE552FE0EDB28A8
:1028F000E66E82DFE552FE0EDB50020FE66E7CDFF5
:10290000E5523B0E72ECCAF079ECD5F05FDFE55290
:10291000000915E1DF6A080EDF5C11E251ECCBF033
:10292000EF50FF080AE151ECCBF0FE0EDBCFEFFFDA
:10293000DDECCDF026C7EFFF02D0DF2AECD7070190
:102940002669E552C2EFC9F043ECD5F0DF6A080E04
:10295000DF5C0FE251ECCBF0EF50FF0808E0DDEC5C
:10296000CDF0EF50016E51ECCBF0EF5005D0DF2AE7
:10297000EED70201CF6BFF0EE552C2EFC9F047EC74
:10298000D5F0DF6A080EDF5C0FE251ECCBF0010EF0
:10299000EFCFDBFFDB50FF0805E0DFECD8F0010EE6
:1029A000DB5005D0DF2AEED70201CF6B000EDBEC47
:1029B000D2F002E2E16AE552E16E4950C2EFC9F09D
:1029C00043ECD5F03250100B04E1020E07015A5DC2
:1029D00002E1DF6A03D06BECD8F0309ADF50E552A9
:1029E000C2EFC9F047ECD5F03250100B04E1020EF3
:1029F00007015A5D03E1DE6ADD6A08D06BECD8F0AE
:102A0000E66AE5ECD6F064ECD0F0309AEDECCAF072
:102A100002E2E16AE552E16EC2EFC9F043ECD5F0A3
:102A200007015E6B5F6B2DA802D0010E2ED0080E41
:102A300076ECCBF0DF6E07015E2B000E5F23C9EC56
:102A4000D8F0200EDF1406E00701580E5E5D020E7E
:102A50005F59EDE307015E51605D5F51615904E22A
:102A60005EC760F75FC761F7580E5E5D020E5F5983
:102A70000BE301018B5105E15CC726F7360EFFEC35
:102A8000CAF02D88000E01D0010EE552C2EFC9F048
:102A9000C6ECC9F02AECD3F0C2EFC9F0C4ECD6F012
:102AA00003E2DFECD2F004D0FE0EDB50F60F410F54
:102AB000C2EFC9F0020E006E020178B9008E35C176
:102AC00001F00150280802E2280E016E0050E66E67
:102AD000060E0102F350E66E780EECECC9F04CECF9
:102AE00020F0016A01013551280807E27C0E30EC24
:102AF000D4F003E2280E355D016E0150E66E3A0E09
:102B00000AEFCAF043ECD5F044EC20F0DF6E0F0E74
:102B1000E66EDF5007E0030EDF5C04E001018A513E
:102B2000020B02E1000E01D0010E000905E00A0EC1
:102B300001017A03F35001D0000EE66E7E0EECEC3C
:102B4000C9F0E552C2EFC9F064C178F2CFECD2F01F
:102B500002E165C178F21200CFECD2F003E178C255
:102B600065F102D078C264F1EFDF5AEF15F08DC243
:102B70000EF08EC20FF035ECD4F0E5ECCBF05E0E2B
:102B8000ECECC9F08FC20EF090C20FF035ECD4F02F
:102B9000E5ECCBF05F0EECECC9F092C2E6FF91C21F
:102BA000E6FFE66A7B0E28EFCCF00601B46BB56B4E
:102BB000020E88ECCDF00601B42B000EB523B45103
:102BC000B65DB551B75904E2B4C6B6F6B5C6B7F6A8
:102BD000E80ED880B455030EB5550BE201018B51B8
:102BE00005E15CC726F7390EFFECCAF02D88318667
:102BF000010C84B0DDD7000C43ECD5F0FE0EDBCF2A
:102C00005CF72D50100B03E13150100B02E1000E68
:102C100020D031A604D00A0E88ECCDF001D0C5DF5B
:102C200079ECD5F0D6EC0CF0E552DF6EE66AD6EC26
:102C30000CF0E55201013851100B0AE03050200B26
:102C400007E1E7A102D02E0E01D0210EE8ECD5F06D
:102C5000DF50E552C2EFC9F08AECD5F00101E791EF
:102C6000C2EFC9F08AECD5F0FC0E6EECCAF001019F
:102C7000E791C2EFC9F08AECD5F0F2ECD8F001018F
:102C8000E791C2EFC9F08AECD5F0F2ECD8F0FA0E79
:102C90006EECCAF0F90E6EECCAF00101E791C2EFDA
:102CA000C9F0B3ECDAF0D8C1E6FFE5ECD6F0D9C153
:102CB000E6FFE5ECD6F00EC0E6FFE5ECD6F00FC07F
:102CC000E6FFE5ECD6F00101E791C2EFC9F01D0E79
:102CD000FDEFD7F01E0EFDEFD7F0D9CFE6FFC2EF24
:102CE000C9F02AB203D0600E2CECCAF02A8212007E
:102CF0002AA203D0610E2CECCAF02A9212002AB24A
:102D000003D0600E2CECCAF02A8212002AA203D053
:102D1000610E2CECCAF02A921200C6ECC9F031B256
:102D200006D0620E2CECCAF0FE0EDBCF1BF2C2EF17
:102D3000C9F0C6ECC9F0B00E2CECCAF0FE0EDBCF29
:102D40001CF2C2EFC9F0C6ECC9F007018651320D82
:102D50003AECD4F0F7ECD4F012E1FE0EDB500FE1C8
:102D60000101D45104E129510A0D3AECD4F0A4EC4C
:102D7000D0F005E00101E80ED86F030ED96FC2EF65
:102D8000C9F043ECD5F0D6CA85F7070185A1858146
:102D90001E0E866F0101D45105E1B3ECCDF03EC0AB
:102DA00086F710D0030ED45D0DE1030E0A5C03E13B
:102DB0000701140E06D08DECCDF004E0C5ECD7F081
:102DC0000701866FD7CA00F00701BEAF10D0190EF9
:102DD000006E0A01D75D06E2E3ECD2F010ECD8F009
:102DE000005E05D0190ED75D10ECD8F00026190E44
:102DF000005C05E3190E005C0701862705D0190E5B
:102E0000D88000540701865F080E006E21A20FD003
:102E10000101D45102E1020E18D0D40506E0020EE1
:102E2000D45D03E0040ED45D11E1010E0ED001016A
:102E3000D45102E1080E09D0D40506E0020ED45D9B
:102E400003E0040ED45D02E1070E006E0701855118
:102E5000FE0BE8420024056EDF6A0550865D13E232
:102E6000DF2A8551FE0BE8428625016E01500024C1
:102E7000FE0BE842866F0050015C02E20050016EDA
:102E80000050015C856F9CECCAF005E10701320E31
:102E9000856F1F0E866F30ECD2F004E2DFCFE6FFC5
:102EA00052DFE552FBECD4F05EE00701BE51800B2F
:102EB00027E0DF5025E15FDBF2ECCEF00A01D751CD
:102EC000190808E2190ED75DE9ECD6F00101D82700
:102ED0004A50D923F7ECD4F008E2E3ECD2F0E9EC65
:102EE000D6F00101D85F4A50D95B01010A0ED9031F
:102EF000F3CFD9F1D803F3CFD8F1F450D92704D0C8
:102F0000DFCFE6FF20DFE55207018551320D97EC58
:102F1000CAF019ECCCF001E1D98F200E006E070148
:102F20008851005C10E18C510101D8190CE10701B6
:102F30008D510101D91907E107018E510E1802E1E7
:102F40008F510F180DE000C088F7D8C18CF7D9C198
:102F50008DF70EC08EF70FC08FF7005073ECD8F0CE
:102F60005DDD4CEC0FF07CEC0DF03CEC4EF0E552EE
:102F7000C2EFC9F091ECCDF0005001E11200FBEC82
:102F8000D4F070E00101DC0ED86F050ED96FF00EA1
:102F90000E6E0A0E0F6E030E005C01E1D98F000465
:102FA00003E0020E005C45E179EC0BF0000915E04E
:102FB00001018951640D97ECCAF0F2ECCEF0010EDC
:102FC0000F0B05E0D890D933D833E806FBE1640E47
:102FD0000101D827000ED9232CD00101345129E05A
:102FE0003451080DF3CFD6F1F4CFD7F15C0ED627CC
:102FF000000ED723D6C149F0D7C14AF0F00ED880D1
:1030000049560A0E4A56010E0F0B03E073ECD0F03E
:10301000FDE149500101D625D86F4A50D721D96F1B
:10302000D6C10EF0D7C10FF0F00ED8800E560A0EA2
:103030000F56040ED45D08E1340ED86F080ED96F18
:10304000A00E0E6E0F0E0F6E050ED45D08E10E0E73
:10305000D86F060ED96FC40E0E6E090E0F6E300EAD
:1030600073ECD8F00EEF15F0320EE66E730E0AEF29
:10307000CAF0640E2CEFCAF047ECD5F083ECCAF02E
:1030800001E192D0E9ECCAF001E08ED007015A517B
:1030900001E08AD038ECD2F001E086D0195101E08D
:1030A00083D001013B51800B04E1050ED45D01E0AA
:1030B0007BD0080E76ECCBF0DF6E9CECCAF06EE1B4
:1030C000E49FDFB8E48FE651040B68E094510108F7
:1030D00065E20201D95162E1D85160E10101E65196
:1030E000010B5CE1E451800B54E080ECCBF051E04B
:1030F0001D50400B4EE1020168514BE12050200B66
:1031000048E0195146E1245144E12C50800B41E143
:103110002C50400B3EE12F50200B3BE12350800B05
:1031200038E13050400B35E12450010B32E1E4EC42
:1031300008F0D7DD0101030E9E6F280E9F6F440E2D
:10314000A06FA26BA2C1A1F1D3ECC5F00701148F4F
:1031500014935BECD5F00701159162ECD5F00701F3
:103160000B899BECC4F0E00E07010A150609E66E18
:10317000120E28ECDBF00701099F7F0E09114EECBF
:10318000D5F0820E2CECCAF001019405190DF3CF95
:10319000D8F20101E4BF02D0E7EC08F001013BAF37
:1031A00003D0010EDF1401D0000EDBECD2F002E2FE
:1031B000E16AE552E16E4950C2EFC9F001013B51AD
:1031C000800B06E083ECCAF003E0E9ECCAF001E012
:1031D000000C010C53C1E6FFF1DF000903E001011F
:1031E0006E5101D0000EE66E340EECECC9F06FC1EA
:1031F000E6FF350E0AEFCAF0650E2CEFCAF020503C
:10320000400B06E00101E551040B02E1E58501D820
:10321000120043ECD5F054C1DFFFCFECD2F002E155
:1032200058C1DFFF080EDF02F350E66E750E0AECA0
:10323000CAF0E552C2EFC9F00701B6510C0803E32A
:10324000B7510C0805E2B66B0C0EB76F0A01DA93A2
:103250001200016A0D0E015C07E031ECCFF002E0D4
:1032600001501200012AF6D7000C0C0E016E01501D
:1032700007E031ECCFF002E0015012000106F7D771
:10328000000C0701B46BB56BD7DFB6C701F00701BF
:10329000B751D880015409E36FEC04F0F3500701F3
:1032A000B413F450B513012AF2D71200016AF2ECFC
:1032B000D0F00BE040ECD6F006E249500508000ED5
:1032C0004A5401E2012A420E0DD0F3ECD4F012E090
:1032D00040ECD6F006E249501408000E4A5401E2D0
:1032E000012A440E0124F0ECD3F0F3CFB4F7F4CF6D
:1032F000B5F7120040ECD6F014E249504608000E33
:103300004A540FE20701F40EB46FB5699CECCAF0A1
:1033100001E1AFD00701B66B0C0EB76F0A01DA837B
:10332000A8D0006AD75137ECCBF006E249500D081F
:10333000000E4A5401E2002AD75137ECCBF006E2E6
:1033400049501308000E4A5401E2002AD7511808C8
:1033500001E2002AD751190801E2002AD75137ECBF
:10336000CBF006E249501F08000E4A5401E2002A41
:10337000D75137ECCBF006E249502508000E4A54ED
:1033800001E2002A0101D45103E0030ED45D1CE1E7
:1033900040ECD6F006E249500508000E4A5401E21E
:1033A000012A54ECDBF006E249500A08000E4A54A8
:1033B00001E2012A54ECDBF022E249501308000E2E
:1033C0004A541DE2012A1BD040ECD6F006E24950D7
:1033D0001E08000E4A5401E2012A54ECDBF006E21A
:1033E00049502808000E4A5401E2012A54ECDBF04F
:1033F00006E249503208000E4A5401E2012A2B0E1F
:103400004C6EDB0E4D6E010E4E6E00504F6E506ACC
:10341000516A030ED8904F3650365136E806FAE11D
:10342000B3ECD0F00150526E536A546AD8905236C1
:103430005336543659ECCEF00900F5CFB4F70A00F4
:10344000F5CFB5F72CECD2F005E00701B485B589CE
:10345000B49DB59B030E0A01D45D02E0D45109E18D
:10346000F8DE0701B66F01DF0701B76F0A01DA83E3
:10347000E3DE0A01D40514E10701B705056E0A0E63
:10348000B75D01E20506E5DE0701B66F0550D8809D
:10349000B65502E205C0B6F7F4DE0A01DA8312007F
:1034A000020ED45D12E10701B629056EB65102087D
:1034B00001E2052ADADE0701B76F0550B75D02E2C7
:1034C00005C0B7F7DEDE0A01DA8312001E0E006EB9
:1034D0000101D45104E1B3ECCDF03E500AD0A4EC8C
:1034E000D0F002E0140E05D08DECCDF003E0C5EC79
:1034F000D7F0006E0A01D651FE0BE842056E1200AD
:10350000050EDFECCAF0050E0A01D803F350006E79
:103510000101012B3DECCFF01B8F1200080EDFECF8
:10352000CAF00A01D951050D14ECD8F00101200EA2
:10353000196F19C118F11B8F120016ECCFF0A8EC0F
:10354000D0F03B51200B06E19CECD0F003E00101F0
:103550001E0EAC6FF9EC63F080ECCCF0300E010184
:10356000195D02E1200E196F1B8F016B2A0E006E90
:103570002388FBEF25F00101D45102E129510BD042
:10358000030ED45D11E1030E0A5C02E1640E03D068
:103590000A5004E1960E0E6E0F6A1200240E2E25BC
:1035A0007BECCBF00E6E0F6A120090DF0701BEAF0E
:1035B00011D0F8ECD8F00A01D751190804E2190E1D
:1035C000D75D3EECCCF0190ED75D18E2E3ECD2F0FB
:1035D0002FEFD3F00A01D751190803E2190ED75D76
:1035E0000026190ED75D03E2E3ECD2F0005E005036
:1035F00051ECDBF0190ED75D01E1BDDF1200570E73
:10360000DFECCAF0BBECD2F006E19CECD0F003E0BA
:1036100001011E0EAC6FC9DF2CECD2F00BE00101F2
:10362000410E166F500E176F0301B8510F6AE83044
:103630007F0B0E6E80ECCCF00101200E196F19C1CA
:1036400018F12CECD2F009E00101460E186F295157
:10365000E8240301B85D07E103D0F7ECD4F003E1FF
:1036600001012A0E196F01011B8F12000A01D451AA
:1036700002E163DF0AD0D40502E142DF06D0020E88
:10368000D45D02E14BDF01D0BADFA8ECD0F03B51B2
:10369000200B06E19CECD0F003E001011E0EAC6FA4
:1036A0001200C6ECC9F0070EE12683EC0FF00A0108
:1036B000D65D04E283EC0FF00A01D66F9BEC0FF0AD
:1036C0000A01D880D65504E29BEC0FF00A01D66FB0
:1036D000CAEC0FF0000903E00A01190ED76FF6DEFD
:1036E000F7ECD4F004E3190ED75D002603D0E3EC29
:1036F000D2F005260550005C03E30550005E0AD0B9
:10370000006AD40507E1DC51D75D04E2DCCAD7FAD0
:10371000DDCAD6FA00C0D8FAD9DE05500026F7EC8B
:10372000D4F004E3190ED75D002609D0E3ECD2F003
:10373000056E0550D880005402E20550005ECCECC6
:10374000D8F00BE249505408000E4A5406E2540ED9
:10375000006EDCCAD7FADDCAD6FA00C0D9FA00C0BA
:10376000C5F7190ED75D03E3190ED75D03D0190E07
:10377000D880D7550701B26FB36BBEAF02D00A0E27
:1037800001D0320EB303F3CFB3F7B203F3CFB2F7E6
:10379000F450B327FE0EDB5004E02050800B01E113
:1037A00065DF3450040B0DE10A01DA51020B09E028
:1037B000F2ECD0F006E1F3ECD4F003E12CECD2F023
:1037C00003E074DD349401D05CDD0701010EB06FBD
:1037D00001012AA303D00701070EB06FD5CADFFF8E
:1037E0000A01D56B0701B051010853E2E7ECD2F0B2
:1037F00050E1D251010B4DE1050ED45D4AE0040EBB
:10380000D45D47E0D40503E0020ED45D0FE1B8ECCF
:1038100004F00A01D95D0AE2D52BFCECD9F004E6EC
:103820001E0E495C000E4A5834E21ED00101D451EC
:103830001DE10A01FCECD9F004E61F0E495C000E04
:103840004A5801E2D52BFCECD9F004E60F0E495C96
:10385000000E4A5809E3D6511CECD4F004E60B0ED6
:103860004B5C000E4C5815E2D52B13D00A01FCEC32
:10387000D9F004E62D0E495C000E4A5801E2D52B22
:10388000FCECD9F004E60F0E495C000E4A5801E248
:10389000D52BDF500A01D55D0AE0D5CADFFF83ECE6
:1038A000DFF0D5CAE6FFAB0E0AECCAF0248A1EACE4
:1038B00003D00201098902D00201068B0501478568
:1038C000D6EC39F0070EE15C02E2E16AE552E16E06
:1038D000C2EFC9F0006A800E066E056E0550050243
:1038E000F350015CF4500258D8B008D000C005F085
:1038F00006420650051206BE09D0F0D705C000F0FA
:1039000006420650051206BE01D0E8D700D01200CC
:10391000C6ECC9F02A8448C102F064ECCBF03FE069
:103920005A0E025E010EE66E3CEC13F0E552016E9B
:1039300002504B0817E24B0E025C036E060E4A6EF5
:103940004AC043F001C03EF03CECFEF03EC049F0FE
:1039500049C043F003C03EF03CECFEF03EC003F033
:103960000350015E0F0E015C02E20F0E016E01506A
:10397000300802E2300E016E01C0C1F702500A0D9C
:1039800097ECCAF00150496E4A6A3CECD6F03D50C3
:10399000026E23B604D00250E8240201D56F3FEC3A
:1039A000D4F00701C06FFE0EDB50020801E187D0A2
:1039B000C0C701F00101E6A502D0040E016E01505E
:1039C0004B6E4C6A025057ECCDF0030ED8900E3679
:1039D0000F36E806FBE134ECD3F00A0E4F6E4FC011
:1039E00043F00BC23EF04BECD8F04D6E4E6A0050E7
:1039F0004B6E4C6A800E3D6E3E6A93ECDAF087ECBB
:103A0000CFF02CECDBF0EAECCCF0036A3DDB016E8E
:103A10001C50040B2FE0010403E0020E015C2AE1BC
:103A20003450400B27E1FE0EDB5024E001C202F0CF
:103A3000025020E0025061ECCAF002E644ECD4F0FF
:103A400019E20250FE0BE842D880005413E2025003
:103A5000E824005C0FE2FE0EDB0406E10C0E02011E
:103A60000027000E012305D00C0E0201005F000E9E
:103A7000015B032A03500EE1880ED8800E54130E0A
:103A80000F5404E2880E0E6E130E0F6E0EC000F27D
:103A90000FC001F22450020B06E12250400B03E05C
:103AA0003150800B0AE0036A006A31AE06D0000E86
:103AB0000201026F036B006F016BF1EC0BF0C2EFC0
:103AC000C9F0C6ECC9F0E5ECCBF079ECD5F032ECFE
:103AD00016F03DECDAF0C2EFC9F0C6ECC9F0CAEC62
:103AE000D7F0770EEAECD1F0FE0EDB5003E0100EBB
:103AF000EAECD1F0C2EFC9F091ECCDF0050E005C1C
:103B000009E0FFECD4F006E179EC0BF0000902E1EA
:103B1000000E01D0010E000902E0000E03D00101E9
:103B20003451E824E66E3C0E0AEFCAF0A7EC3FF0F1
:103B3000E3DF0201A85103E00101345106E0020174
:103B4000A85105E10101345102E0BAEC17F02A84D2
:103B5000120088ECD6F003E00101285101D0000EDC
:103B6000DF6E21B204D0040EDF02F3CFDFFF080EB8
:103B7000DF5C08E2010EE66E940E0AECCAF0DFCFBD
:103B8000E6FF07D0E66A940E0AECCAF0060EDF5C88
:103B9000E66E760E0AECCAF0DF90DF42080EDF5CBC
:103BA00005E2FE0EDB5002E0040EDF6EDFCFE6FF23
:103BB000790E0AECCAF0E552C2EFC9F0C6ECC9F0C2
:103BC000016A080E015C16E2FE0EDB50012449EC8E
:103BD000D4F0026E100E025C040DF350006E19EC6E
:103BE000CCF001E1006AA5ECDAF000502CECCAF050
:103BF000012AE7D7140EF1ECC9F0C2EFC9F0FBECD3
:103C0000D4F00CE0220E2CECCAF00101D45102E1F8
:103C1000180E01D0080EE66ED1DFE5520EEF15F05A
:103C2000FBECD4F00DE0310E2CECCAF095EC0BF06F
:103C3000000902E0100E01D0000EE66EBFDFE55273
:103C40000EEF15F0270E0101B95D02E1FFEF1DF047
:103C500010EF1EF0020199510101625D18E062C18E
:103C600099F26251020B05E1D051200B02E1000EE6
:103C700001D0010E000902E0000E01D0380EE66E00
:103C80000F0EE66EC80EE66EA10E28ECCCF0120008
:103C900086ECCCF0840E2CECCAF02A9271EC16F073
:103CA000E66A720E0AECCAF03C0EE66E710E0AEC81
:103CB000CAF0C1EC16F0FCEC18F055EC0CF01DEC61
:103CC00009F0B8D8C9ECD6F0E66A130E0AECCAF0CF
:103CD000010162855C95BEDF81EC4EF0E668B30EB3
:103CE0000AECCAF03DD83CEC4EF0C4EC4FF0E7ECE7
:103CF00008F0B7EC15F0A4EC15F05AEC15F009EC4F
:103D000019F08EDF4DECCCF0F7DE82EC15F0EAEC2A
:103D100018F0010EE66EE1DEE55286ECCCF006010D
:103D2000B26B090EB36F6BDF01015F51200B02E034
:103D3000640E01D0320EE66E1F0E0AECCAF0010EC0
:103D4000E66E0F0E0AEFCAF01200046A01015FAFBF
:103D500004D011BC048011BE04823CB9048412005A
:103D6000010112983B51100B01E012883B51100BDE
:103D70000FE02150020B0CE01E50200B09E0050E55
:103D8000D45D06E0040ED45D03E0030E006E06D0A1
:103D900031C100F0FFECD4F001E0006A0050E66EA3
:103DA000A60E0AEFCAF0016A0701BEB302D04BC1EA
:103DB00001F04CC102F0BE51020B09E00101D451E7
:103DC00004E10601EA51010802E34DC102F00F0EC1
:103DD0000101D8804155E66EF9ECD9F07DC1E6FFCE
:103DE00047C1E6FFA00EE66E43EC16F0496E060EE4
:103DF000E15E495070C1E6FF6E0E0AECCAF00701A1
:103E0000BEB10FD00101D2AD03D0D29D3CEC4EF03B
:103E10001450100B06E01450200B03E11498C4EC6E
:103E20004FF00701BE51010B02E0AE0E01D0AD0E06
:103E30002CEFCAF0D3EF1EF043ECD5F091ECCDF0AF
:103E4000000403E0020E005C08E1E66A3350040B54
:103E500002E0030E36D0000E34D0005005E1010E12
:103E6000E66E3BDEE55253D0050E005C2CE10E6A97
:103E70000F6A01015751080B0BE1E651040B08E0F2
:103E800002018951040B04E0D00E0E6E070E0F6E76
:103E9000E5ECCBF08D0EECECC9F002018951040B7E
:103EA00008E12050400B03E0330E875D02E0000E76
:103EB00001D0010E000902E0875101D0000EE66E2C
:103EC000040EE66E26D0030E005C21E1E9ECCAF098
:103ED0001EE0020E0A5C03E168ECD1F011D0E80E9E
:103EE0000E6E030E0F6EE5ECCBF03E0EECECC9F05F
:103EF000DF6A010196ABDF2ADFCFE6FF020EE66E36
:103F0000140EECECC9F00501040E266F05D0E66A2C
:103F1000E66A140EECECC9F0E552C2EFC9F043ECCE
:103F2000D5F002012F6B0601BF6BBFC6BEF6329EF5
:103F30000101D45124E10601EA51010803E31350C1
:103F4000010B17E0016AEA05EB6F020EEA5D03E37D
:103F500002011A5102E00601EB6BEBC6E6FF79ECB9
:103F6000D6F0E66A030EE66E120EECECC9F0328E65
:103F700004D0C9ECD6F00601EB6B5CDF5BD0030E1E
:103F8000D45D56E162991350010B06E1F2ECD0F0DA
:103F900003E103ECD5F048E08DECCDF00AE02D0E06
:103FA000DF6E010E016E026A13A015D002012F6FA1
:103FB00012D0A4ECD0F00DE0020E016E026A1F0ECA
:103FC000DF6E010196BB07D0010E026E3F0EDF6E61
:103FD00002D0016A026AF9ECD9F0120EECECC9F0D9
:103FE000EDC6E6FF79ECD6F0328EF2ECD0F002E0CE
:103FF000010162890701200E516F3F0EDF5C02E173
:10400000100E516F640EDF5C02E10A0E516F4B0E11
:10401000DF5C02E10D0E516F2D0EDF5C02E1160E2A
:10402000516F4E6B526B02D0C9ECD6F013DE02D04A
:10403000C9ECD6F055EC39F0E552C2EFC9F0BF0E2D
:10404000F5ECD9F0E840E8403F0B005C02010B6F53
:10405000060E00C0E7FF070B04E0E742E79EE80614
:10406000FCE1E75002010B5F0B07640E0B5D09E2F8
:104070002150100B06E10101395103E1218897EC31
:10408000D9F00BC200F012001FB203D00101D451CD
:1040900012000101D55112000C0E2CECCAF07AEC82
:1040A000CCF00E6E0F6AFF0E0E1804E10F5002E105
:1040B0000E680F681200416B426B436B446B400EFD
:1040C000456FD8903C373B373A3739373837373731
:1040D0003637353744374337423741374051445DEF
:1040E0003F5143593E5142593D51415909E34051D5
:1040F000445F3F51435B3E51425B3D51415B3C2B32
:10410000452FE0D712000101D09711BED087D19979
:1041100011BCD18912006EECD1F001010490D05194
:10412000080B01E004800492D151100B01E00482DD
:10413000119E04B0118E119C04B2118C07010A97D4
:104140000A990A8504A00ED00101D05107010A99ED
:10415000010B01E00A890101D05107010A97020B06
:1041600001E00A870A51100B06E10101775103E1D2
:104170000450020B02E007010A9507010A9104B2FC
:104180000A819DECC4F0A5EF1EF043ECD5F0FCECE9
:10419000D8F0200E4FECD8F00050026E0F0E4FEC0E
:1041A000D8F001012B51005C29E1250E025C26E1CB
:1041B000050E80ECD7F019ECCCF013E2010EE66EA0
:1041C0000A0EDF24C9ECD5F034ECCAF00F0E010161
:1041D0000617D451065D05E0288206C1D4F19BEC98
:1041E000CCF09CECCAF007E1030EE66E100EDF2463
:1041F000E66E7AECD8F0096A010E02D0096A000E68
:10420000E552C2EFC9F0C6ECC9F01EAC03D0020102
:10421000098102D0020106830501478147872B8C63
:104220002C8ABDECCBF0EE50ED1013E00101442BD5
:10423000640E445D03E2A9DF00091DE101014407AA
:10424000FF0E445D03E0A1DF0009F8E10101442B0A
:1042500012D001014407FF0E445D03E096DF000920
:104260000AE10101442B640E445D03E28EDF000984
:10427000F8E101014407C2EFC9F0C6ECC9F0EB0E4A
:10428000496ED50E4A6E010EDFECDAF07F0B006E40
:10429000FE0EDB50040806E1FD0EDB50310802E2A1
:1042A000020E006E07ECD5F006E1FD0EDB50310882
:1042B00002E2040E006EC2EFC9F0040E0101435D7C
:1042C00001E3436B395102E0190E04D0160E432569
:1042D0007BECCBF0006E0050E66EE66A3C0EE66EBC
:1042E000C2ECFBF04CEFD5F021900201320E246FAE
:1042F000295102E0140E246FC80E366F1DAC2998A8
:10430000D95102E0E7EC08F01D50400B03E02A50C1
:10431000800B02E171EC16F002010987098509831F
:1043200009817A6B0901EB6B1200C6ECC9F0FE0E35
:10433000DB500EE029A006D0FE0EDB50030B02E19D
:1043400087EC07F0280E88ECCDF0FE0EDB06EFD7E9
:10435000C2EFC9F011C512F50501106B279C0101D0
:10436000E491120027BA09D013C549F114C529F107
:10437000249223BC2482F0EC64F0278A0101369950
:10438000E7EC08F00201216B239A2592120030EC31
:10439000CEF0E0DF2750200B05E0E9ECCAF002E0A8
:1043A000080E076EDFDF2F98120027AA02D0010146
:1043B000E88B0750220A01E19ED1030A01E17FD177
:1043C000010A01E1EFD03F0A39E0010A01E0ADD175
:1043D000278C49C113F529C114F5239C24B2238CE1
:1043E00027BA15D0010136AD11D0E7B706D0365146
:1043F000070B050DF3500A0F496F640E296F36B98C
:1044000002D0430E296FDAEC64F001D0C0DF03EC78
:10441000D5F007E0200E06014A5D03E0200E11EC06
:10442000CDF01D901F0E076E02012D5101E17ED1CE
:104430002750200B01E17AD1076A23D105011051E1
:1044400001E188D0E9ECCAF016E02750200B13E018
:104450000501235107E1020E265D0DE141EC0EF04E
:10446000000909E102012D5101E12D2B080E076E13
:104470001F0E086E1200050110071251EA6A000FA4
:10448000E96E080EEA22EFCF02F7122B125161EC0F
:10449000CAF002E612ECD4F001E3126BE9ECCAF0C8
:1044A0000BE02750200B08E002C7E6FF4EEC3CF083
:1044B000E552200E076E12003C0E0701025D04E17A
:1044C0002482238C229C32D13E0E025D06E124928E
:1044D000239C1EBC2BD1228C29D1740E025D01E1DC
:1044E00025D10601EA510AE02750200B07E0298A6E
:1044F00002C7E6FFC3EC6FF0E552299A800E070170
:10450000025D0FE21D0E496EDA0E4A6E010E4B6E11
:10451000200E025D50ECCDF0CBECC9F00800F5CFD9
:1045200002F7800E025D03E10201040E526F0701E3
:104530000251800805E2800E025DFD0F0201526FFC
:10454000800E0701025D01E3B4D0025101E1EED01B
:10455000200ECFD027AAE9D0EFECD1F007E0070179
:104560000251800803E3200E11ECCDF010DFE9ECDE
:10457000CAF005E0279C080E076E100E086E275043
:10458000200B01E1D3D00201555101E1CFD0189A9F
:1045900055BF188A196B010EE66E7F0E55155BEC40
:1045A000D2F0C4D01750800B06E02750200B09E151
:1045B0000B0E155C06E01D50040B03E01D50080BAC
:1045C00058E12750200B09E01750800B06E03CEC27
:1045D000D2F003E00B0E155C1CE14DEC65F0D7DE6C
:1045E000209427AAA3D0E9ECCAF003E00201010E4F
:1045F0002D6FFAECD3F00601EA5101E197D00701E3
:104600000251800801E292D02F88200E11ECCDF0EB
:104610008DD0230E155C10E1010EE66E52EC0EF00B
:10462000E5521EAC03D00201098702D002010681C7
:104630000501478D179E7AD08EEC96F0000914E0A4
:104640002750200B11E00C50006E020E77ECD0F0DA
:104650000C50026E00500C6E0250E66E67EC74F067
:10466000E5520201196B62D027AA60D0FBEC98F0EA
:104670005DD0E9ECCAF008E02750200B05E0080EF9
:10468000076E1F0E086E52D0FE0E070102150EE0D7
:10469000228E010E016F02A102D0030E016F029162
:1046A0000243210E076E0501200E07D00201020E03
:1046B000526F220E076E05011F0E156F37D00701CE
:1046C000015112E00107238006EC65F0076A1DA086
:1046D00006D0020E076E27BA02D0F7ECCEF0210EFC
:1046E000086E1D80229E22D00201010E526F228E82
:1046F000220E076E1BD00201525114E02390520784
:1047000006EC65F0030E076E1DB007D0070E076EAE
:1047100027BA03D0006A3DEC75F0220E086E229E87
:104720001D9004D015C507F001D031DE0101E89BD2
:104730001200020171510101D880485502E271C294
:1047400048F12B510A0825E2100E2B5DF8ECCBF056
:10475000060ECDECDAF0016EE651040B13E01B50AF
:10476000080B10E101501E0802E21E0E016E6E0ED3
:1047700002010B5D02E2140E016E5A0E0B5D02E2A5
:104780000F0E016E01500101D880485502E201C0B0
:1047900048F139512CE10A0E2B5D05E148516408BE
:1047A00002E2640E486F02010B5161ECCAF002E6AE
:1047B00044ECD4F006E201014851640802E2640EC0
:1047C000486F640E02010B5D06E201014851320898
:1047D00002E2320E486F01014851780808E2010EEA
:1047E0002B5D03E32B51050802E2780E486F215040
:1047F000100B05E04851320802E2320E486F64ECBB
:10480000CBF015E1010148511E080BE2640E0201D4
:104810000B5D0DE301014851320809E3EBECD2F0E6
:1048200006E001015FB309D05F83D5EFC4F0010159
:104830005FA303D05F93D5ECC4F01200DACFE4FF9E
:10484000E2CFDAFFE9CFE4FFEACFE4FFE652FC0E65
:10485000B36EF30EB26E020111070201115105E1B0
:104860000201320E116F010121810101E7A92CD053
:104870000601FD07000EFE5B0601FD51FE1124E15D
:10488000F29EF26AF06AB96A9D6A000EA66EA16E87
:104890009E6E8D8C8D8A8C908494070E936E000092
:1048A000000000008A9A0000000000000000270EAF
:1048B000936E4E0E996E0000000000000300000091
:1048C000000000000000FF001E801D861D8481B2D4
:1048D0000BD001014FA302D01E9006D001014FA1C1
:1048E00002D01D9601D01D9481B40BD001014FA3BD
:1048F00002D01E9006D001014FA102D01D9401D01C
:104900001D9687B60BD001014FAB02D01E9006D08A
:1049100001014FA902D01D9601D01D9481B00BD08A
:1049200001014FAB02D01E9006D001014FA902D069
:104930001D9401D01D96020112070201125137E1A8
:104940000201050E126F0101B05116E00101B0071E
:10495000020102015151020B05E01D50040B02E15E
:1049600002015181020102015151080B05E01D5065
:10497000080B02E1020151850101B15106E0FF0E71
:104980000101B15D02E00101B12B1FAE04D00601AF
:10499000DE2B000EDF230701505109E0070150070D
:1049A0000701505104E151C750F701012183010172
:1049B000AF5102E00101AF070101269701012695E1
:1049C000010126A102D001012685010126A302D002
:1049D00001012687010126930101269188A202D0B8
:1049E0000101268188A002D0010126830F0E01015A
:1049F00026150101236F01012351EA6AC50FE96EF3
:104A0000060EEA22EFCF22F1010E0101221513E07A
:104A10001F50080B05E0010101013B51010B0BE1A7
:104A20002050200B08E0010122AF03D00101240730
:104A300002D00101242B9EAA11D00701942B07015B
:104A40009351932BEA6A000FE96E0C0EEA22AECF67
:104A5000EFFF0701945102E192C793F7A19207017A
:104A60004607E552E5CFEAFFE5CFE9FFE5CFDAFFFC
:104A7000110001013BAB07D03B9B238A0601425149
:104A800002E0426B436B12000701BEB103D0119AE2
:104A9000119812001198BEA31188119ABEB3118A01
:104AA00012000B0EDFECCAF0258E120083ECCAF068
:104AB00003E0E9ECCAF006E01394010156A30ED01E
:104AC00013840CD0139402013D5107E10101E6511A
:104AD000800B03E13B51040B01E01384139613A4F4
:104AE000138613981350040B04E164ECCBF001E03F
:104AF00013881200ECC1E9FFEDC1EAFFEECF49F0E7
:104B0000EECF4AF0EECF4BF0EECF4CF0EFCF4DF0C2
:104B1000EAC1E9FFEBC1EAFF49C0EEFF4AC0EEFF80
:104B20004BC0EEFF4CC0EEFF4DC0EEFF1200C6ECD6
:104B3000C9F063ECCEF0FB0EDBCFECF1FC0EDBCF6B
:104B4000EDF10101A30EEA6F010EEB6FD3DFC2ECB2
:104B500031F0D850010B06E0FF0E01019E5D02E02E
:104B6000010E01D0000EC2EFC9F047ECD5F00050A5
:104B7000E66EF8ECFDF0E552140EE66E57ECFEF032
:104B8000E5526CECFEF067ECFEF00009FCE1C4506D
:104B9000006E0050F80812E2C20410E0050EC25C7C
:104BA0000DE0090EC25C0AE00D0EC25C07E0110EBA
:104BB000C25C04E0390EC25C01E00006020EE15C5A
:104BC00002E2E16AE552E16EC2EFC9F043ECD5F0D2
:104BD0000050DF6EFE0E496ECD0E4A6E010EE6EC01
:104BE000DAF00150006E009EECECE1F001AEF2D77D
:104BF000E552C2EFC9F043ECD5F00050DF6E235010
:104C0000100B1DE10050E66E73EC04F0E552800BD2
:104C100016E01B0EDF5C08E10101200E166F500E3E
:104C2000176F410E186F07D00101450E166F520E17
:104C3000186F18C117F1200E196F040E016F2A8822
:104C400023A808D0FA0E496ECF0E4A6E010EE6EC8C
:104C5000DAF007D0DFCFE6FF73EC04F0E552016E27
:104C6000DF2A2AA802D0019E2A980150006E009ED9
:104C70000FECE2F001AEE4D72398E552C2EFC9F0A1
:104C8000C4ECD6F003E2DFECD2F004D0FE0EDB5031
:104C9000410FF60F006EECECE1F0C2EFC9F0C4EC8E
:104CA000D6F003E2DFECD2F004D0FE0EDB50410F71
:104CB000F60F006E0FECE2F0C2EFC9F09BECD9F0FA
:104CC000DFDFE5526EECD0F0DBDFE552C2EFC9F07A
:104CD0009BECD9F0E4DFE5526EECD0F0E0DFE5527A
:104CE000C2EFC9F0C6ECC9F03AECD3F0020E0101F4
:104CF000002761ECE1F0DF50006E050E0101005F5E
:104D000061ECE1F0030E0101005FE552C2EFC9F072
:104D1000C6ECC9F03AECD3F0FE0EDB50020F0101F5
:104D2000016F7EECE1F0DF50006EFE0EDBCF01F193
:104D30007EECE1F0E552C2EFC9F000C059F26CEC34
:104D4000DBF0FF0E005C01E041DF0101B5891200DC
:104D500000C05AF27CECDBF0FF0E005C01E04BDFA0
:104D60000101B58B12006CECDBF0FF0E005C01E082
:104D70002DDF0101B58D640EAC6F249612007CEC22
:104D8000DBF0FF0E005C01E036DF0101B58F640E41
:104D9000AC6F24961200C6ECC9F016ECCFF0EEEC26
:104DA000CBF05DECCAF0C2EFC9F0C6ECC9F016EC6E
:104DB000CFF079ECD5F0010EE66E66EC08F0E55226
:104DC000E552C2EFC9F0C6ECC9F070EC6FF001011A
:104DD000190EAE6FFC0EDBCFB2F1FD0EDBCFB3F1DF
:104DE000FE0EDBCFB4F1C2EFC9F0830E096EE00E08
:104DF0004DECDBF0800E005C08E270EC6FF001011E
:104E0000190EAE6F0201E00EA96F12005CECDAF031
:104E1000DBCF4AF0800E4A1407E0B6ECCBF0496CC9
:104E20004A1E000E4A2202D0B6ECCBF08EECD9F02E
:104E3000C2EFC9F0C6ECC9F012A60FD0060150B5FA
:104E400003D00101C4ECCEF0288ABCBF289AFE0E24
:104E5000DB5001E0287AECEC40F0C2EFC9F05CECEA
:104E6000DAF0DBAE08D0DB50FF0DFE0EF3CFDBFF38
:104E700010ECD1F007D010ECD1F0DB50FF0DFE0E9E
:104E8000F3CFDBFFDB50C2EFC9F043ECD5F00701F5
:104E90005A5101E05DD11D50400B01E059D1325013
:104EA000040B01E154D10101D45104E18450020BFF
:104EB00001E14DD10B0E76ECCBF00601BC6F8DEC11
:104EC000CDF001E0A5D0140E0601E76EBC19E8AEE6
:104ED00002D0BC3503D0E750D880BC5502E2140E96
:104EE000BC6FEC0EE76EBC19E8AE02D0E73402D01E
:104EF000E750BC5D02E2EC0EBC6FBE51E76EBC1920
:104F0000E8AE02D0BC3503D0E750D880BC5502E2F1
:104F1000BE2B0BD0BE51E76EBC19E8AE02D0E73411
:104F200002D0E750BC5D03E2BE07BEC6BCF6200E51
:104F3000496E4A6AC1C63DF0C2C63EF041ECD3F0AC
:104F40003DC0C0F6C0C649F04A6A49BE4A684950E9
:104F50000601C15F4A50C25BBCC649F04A6A49BEFD
:104F60004A684950C1274A50C223C0C6E6FF77DFCE
:104F7000E552016E010EE66E0E0E01248CECCCF0B3
:104F800002011A5101E1E3D01BAA05D0BCC6E6FF1D
:104F900098EC75F0E55260ECCCF02AE01250080B6A
:104FA00003E1040E1A1528E0E4ECD5F001E0010E4F
:104FB000496ED45103E1D051400B07E0D45103E0D6
:104FC000CF51040B02E0000E01D0010E491809E098
:104FD00012A602D0E66A09D00601BC5101012427BD
:104FE0000BD012A605D0010EE66E24DFE55204D0E8
:104FF0000601BC510101245F0601BC5101E0A7D0AC
:1050000002011A51320801E3A2D0320E1A6F9FD06A
:105010001B0EE66EF2EC14F0E552F3CFBCF6F4CFC3
:10502000BDF6026A016A0601BC51E76EBD19E8AE21
:1050300002D0BD3503D0E750D880BD5505E2BC5144
:10504000BD5D8BECCFF0026E0601BD51E76EBC1961
:10505000E8AE02D0BC3503D0E750D880BC5505E29D
:10506000BD51BC5D8BECCFF0016E0601BF51D88005
:10507000025402E202C0BFF6BE51D880015402E2DF
:1050800001C0BEF6000EE76EBF19E8AE02D0BF3514
:1050900003D0E750D880BF5505E2010EE66E0D0E35
:1050A0008CECCCF0010E0601E76EBF19E8AE02D021
:1050B000BF3503D0E750D880BF5505E2010EE66E3C
:1050C0000C0E8CECCCF0020E0601E76EBF19E8AEB8
:1050D00002D0BF3503D0E750D880BF5505E2010E9E
:1050E000E66E0B0E8CECCCF0000E0601E76EBE19DE
:1050F000E8AE02D0BE3503D0E750D880BE5505E2F9
:10510000010EE66E0F0E8CECCCF0010E0601E76E80
:10511000BE19E8AE02D0BE3503D0E750D880BE55E8
:1051200005E2010EE66E100E8CECCCF0020E0601CC
:10513000E76EBE19E8AE02D0BE3503D0E750D88086
:10514000BE5505E2010EE66E110E8CECCCF03294E9
:10515000E552C2EFC9F047ECD5F0FC0EDB506AE136
:1051600002012A5167E10490FE0EDB50140804E2AC
:10517000140EFAECCEF00480FE0EDBCF49F056514F
:10518000D880495403E2FE0EDBCF56F201012A51CA
:10519000100B03E0050ED45D05E10450010B02E0A5
:1051A000FE0EDB2A010E67C1DBFF050ED45D02E1B6
:1051B000010EDB6A010EDB50280803E2DE52280EE6
:1051C000DD6E050EBDECD0F03EC0DBFFDF6A150ED4
:1051D000DF5C22E2006AFE0EDB5004E0FE0EDB50D4
:1051E000DF5C13E301012A51100B07E0050ED45DCB
:1051F00004E002015651DF5C08E001016751040838
:1052000006E2010EDB50DF5C02E1010E006E005091
:10521000CCECCEF0DF2ADBD71350010B69E00201A2
:10522000215166E10101D45103E0030ED45D60E138
:1052300032845ED0FC0EDB0430E102012A5106E02C
:10524000FD0EDB5003E12250400B55E107ECD5F099
:1052500003E2080EFAECCEF0FD0EDB500C0805E27E
:105260000C0EF36EFD0EF3CFDBFF70ECCEF0150EDF
:10527000DF5C3EE2FE0EDB5004E0FE0EDB50DF5C46
:1052800007E3090EDF5C07E3FD0EDB50DF5C03E2A2
:10529000010ECCECCEF0DF2AEAD7FC0EDB50020880
:1052A00027E107ECD5F003E2080EFAECCEF0FD0E94
:1052B000DB500C0805E20B0EF36EFD0EF3CFDBFFA7
:1052C00070ECCEF0150EDF5C13E2FE0EDB5004E056
:1052D000FE0EDB50DF5C07E3090EDF5C07E3FD0E2B
:1052E000DB50DF5C03E2010ECCECCEF0DF2AEAD724
:1052F000FE0EDBCF0AF2020EE15C02E2E16AE55249
:10530000E16EC2EFC9F00101D551D3ECCEF0A6ECAD
:10531000CCF00150080D4950F3240A01DF6F4A50C8
:10532000F420E06F12000101C951C45D0CE1CA51C3
:10533000C55D09E1CB51C65D06E1CC51C75D03E116
:10534000CD51C85D01E0000C010C0101D551D45DC7
:1053500001E0000CD4510BE1D051400B01E0010EF3
:10536000496EDD51400B01E0010E495C2DE0030E5A
:10537000D45D23E1DC5158ECCBF00A5C1EE18DECEE
:10538000CDF00CE00101D051040B01E0010E4A6E9A
:10539000DD51040B01E0010E4A5C16E08DECCDF00E
:1053A0000CE10101CF51040B01E0010E4B6EDC5109
:1053B000040B01E0010E4B5C07E00101D45103E056
:1053C000030ED45D01E1000C010CADDF000903E028
:1053D000BCDF000901E1000C010CF7DF000928E047
:1053E0009CECCAF001E1010CD551D3ECCEF0080ED3
:1053F000E66EE66AD551CFECD7F001507EECDAF0DC
:10540000D451100DF3CF4FF0F4CF50F02A0E4F26A9
:105410000A0E50220701B151080D93ECCFF074EC45
:10542000FAF0516E060EE15E5150000901E1010CE7
:10543000000C1AB202D09EECCFF0D4C1D5F134AA40
:1054400017D0010138A306D0DE93D1B3DE83DE95F9
:10545000D1B5DE85DD9DD0BDDD8DDD95D0B5DD8599
:10546000DC95CFB5DC85FFECD9F080ECD6F01AD016
:105470000101D55103E1DD9DD0BDDD8D030ED55D6C
:1054800011E1FFECD9F080ECD6F08DECCDF006E028
:105490000101DD95D0A506D0DD8504D00101DC95A4
:1054A000CFB5DC8534AA0DD0500EE66EE66A2A0E22
:1054B000E66E0A0EE66E7A0EE66E0A0E34ECCDF05B
:1054C0000FD0050ED45D0CE0100EE66EE66AEDEC32
:1054D000DAF0D551CFECD7F058ECD4F0E3ECCCF0C7
:1054E000050E0101D55D08E0D551EA6ACF0FE96EDE
:1054F0000A0EEA22B1C7EFFF1200C9C1C4F1CAC146
:10550000C5F1CBC1C6F1CCC1C7F1CDC1C8F1D5C180
:10551000D4F134AA08D063ECD2F02A0EE66E0A0E5B
:1055200034ECCDF014D09CECCAF011E0100EE66E15
:10553000E66AA6ECCCF032ECCBF0D451100D0CECBA
:10554000CDF02BECD4F058ECD4F0E3ECCCF09CECA8
:10555000CAF004E0D6ECCDF0B1C7EFFF1200C6EC04
:10556000C9F03BDF000916E1C2EC13F0FE0EDB5080
:1055700002E15FDF01D0C1DFF4ECD1F0248A1EAC80
:1055800004D002010983098102D0020106830501CA
:1055900047834781C2EFC9F0C2EC13F00101C45147
:1055A0000CE0C40503E13C0EC55D07E3C95105E00D
:1055B000C90514E13C0ECA5D11E207ECCDF0348A56
:1055C00010D8349A66EC13F01C8A07ECCDF01C9AC4
:1055D0001884FFECCEF0189474EFD1F002D866EF87
:1055E00013F00DC103F0C9C19AF2CAC19BF2CBC13D
:1055F0009CF2CCC19DF2CDC19EF2D5C100F05DEC14
:10560000D4F0DEC1E2F134AA08D063ECD2F0540E3B
:10561000E66E060E34ECCDF011D0050E005C0EE007
:10562000100EE66EE66A0101A6ECCCF032ECCBF08F
:10563000540EE66E060EE66E44ECD3F0016A050EDB
:10564000005C03E00050D3ECCEF0F3DE03C00DF1BC
:105650009AC2C4F19BC2C5F19CC2C6F19DC2C7F1FA
:105660009EC2C8F100C0D4F134AA1ED0010138A3F3
:105670000ED0D193E2B3D183D195E2B5D185129604
:10568000D1B312861294D1B5128481EC9AF0010143
:10569000D09DE1BDD08DD095E1B5D085CF95E0B559
:1056A000CF8547ECD6F018D00101D45103E1D09D4D
:1056B000E1BDD08D030ED45D0FE147ECD6F08DEC4B
:1056C000CDF006E00101D095E1A506D0D08504D04B
:1056D0000101CF95E0B5CF8534AA09D0500E4BEC2F
:1056E000D3F02A0EE66E0A0E34ECCDF00AD0050E89
:1056F000005C07E0100E4BECD3F0EDECDAF044EC7C
:10570000D3F001C0B1F79CECCAF004E0D6ECCDF0C8
:1057100001C0EFFF04903BB104803B913BB33B8160
:105720003B9304B03B83129C3BB1128C129E3BB363
:10573000128EF4ECD1F0248AB5DB1EAC06D0020147
:10574000098709850983098102D0020106830501C1
:105750004881BF0E476F1200C6ECC9F00101628597
:105760002AEC1EF0C2EFC9F0370E005C02E2370EE1
:10577000006E00509F0802E29F0E006E630E005CF8
:1057800008E2370E005CE824496E090EC0ECCAF04E
:1057900005D0630E005C10ECD8F0090F006E02011A
:1057A000D05102E0030E00260050150802E2150E4B
:1057B000006E12008CECD6F00201215110E1205055
:1057C000010B0DE124510BE13250100B08E1275081
:1057D000200B05E0D85103E130A003D03090000E3B
:1057E00070D0FE0EDB5002E0990E01D00A0E76EC6E
:1057F000CBF064ECD0F08C0E62ECD4F00201D0510E
:1058000003E0790E62ECD4F02C5129E1020EDB505A
:1058100044ECCCF024E30A0E76ECCBF0496E020E99
:10582000DB50495C1CE311AE0DD0119E83EC20F0DF
:105830000201068D090E7EECCAF052ECD3F00BEC9F
:10584000D5F00DD00201D05107E107010A939DEC7C
:10585000C4F028EC53F011840201FA0ED06F010E4F
:10586000DB50006E00509F0802E29F0E006E005059
:105870004B6E4C6A05011851070D58ECD3F0030E1E
:105880000F0B03E073ECD0F0FDE149C018F56CDFBD
:105890000050DF6E00C0A2F7090E016E01012AB9A7
:1058A00001061350010B06E00150D880005402E2BB
:1058B0000150006EE66AE66A0050E66E1BECCEF020
:1058C000DF50496E030EE15C02E2E16AE552E16EEF
:1058D0004950C2EFC9F069ECD5F0020B1CE00101A0
:1058E000E651400B18E00201685115E1080E155C05
:1058F00006E0290E155C03E00A0E155C0CE1080EAB
:10590000155C02E1010E20D0290E155C02E1020EA9
:105910001BD0030E19D0016A0A0E015C19E2FE0EBB
:10592000DB50010B06E0230E012457ECCCF0155C94
:105930000AE0FE0EDB50020B09E02D0E012457ECAD
:10594000CCF0155C03E101500C6E02D0012AE4D7C3
:10595000C2EFC9F0C6ECC9F0800E0C6E17AE17D0BE
:10596000179E1750010B03E11750100B10E0100E9B
:105970000C6E79ECD5F0AFDFE5522C0E155C02E130
:10598000200E0C6E0B0E155C02E1400E0C6EC2EF89
:10599000C9F0C6ECC9F0A9ECCFF079ECD5F031EC48
:1059A0000CF0E5521DECD8F00101A86FA851640D70
:1059B00097ECCAF018ECD8F05C0F7BECCBF0006EE3
:1059C00015ECD7F05FECD3F000504B6E4C6A010140
:1059D0004B50495CD86F4C504A58D96F29A60BD010
:1059E0009E515FECD3F00101D851495C0E6ED95144
:1059F0004A580F6E06D09E510F6AD8250E6ED951A7
:105A00000F22E4ECD4F03CECD6F03DC0A8F139C054
:105A10009EF1C2EFC9F0C6ECC9F0A9ECCFF0DB50A3
:105A2000F8ECCBF0030ECDECDAF00101A85D02E05A
:105A3000000E1BD0FE0EDB50F8ECCBF0020ECDECCE
:105A4000DAF09E5D006E00BE006C040E005C0AE39E
:105A500091ECD6F009E0945107E0A85105E0190E49
:105A6000005C02E2010E01D0000EC2EFC9F0010E8F
:105A7000E66E70DFE55200680A0E0C5C02E20C5024
:105A80001DD0200E0C5C02E10E0E18D0400E0C5CF6
:105A900002E10F0E13D0100E155C02E10A0E0ED0BB
:105AA000180E155C02E10B0E09D0110E155C02E117
:105AB0000C0E04D0190E155C02E10D0E006EFF0EE7
:105AC000005C1DE00050E66E8E0E0AECCAF0300E4F
:105AD000E66E8F0E0AECCAF0C80EF1ECC9F017A8FA
:105AE00008D07AECD1F0000904E0140EF1ECC9F012
:105AF000F8D7E66A8F0E0AECCAF0179E010C000C6C
:105B000052ECD8F0920E491810E14A500EE1006AAA
:105B10009DEC26F0B80E40ECD2F00101AC6B218672
:105B20000201776B696B289E072A52ECD8F0930E1E
:105B300049185CE14A505AE1010EE66E0BDFE5526E
:105B40000A0E0C5C32E202017751050833E3695119
:105B5000020830E3772B28BE692B010E016E070E79
:105B6000015C13E20128E3ECCAF0EF50006E060E70
:105B7000015C05E1800E010115150C10006E56EC5C
:105B8000D8F000C0EFFF012AEAD70101159F36AD1A
:105B90002DD00C5002E1540E02D0300E0C24006EB9
:105BA000800E001004ECCFF010D0200E0C5C12E13F
:105BB00028AE02D0258E1AD0288E0101158FD20E64
:105BC00004ECCFF0010136AD11D00501930E4B6FFF
:105BD0001E0E0BD0400E0C5C04E1980E076E1A8866
:105BE00005D0100E0C5C02E19A0E076E52ECD8F054
:105BF000980E491801E077D04A5075E1010E016E08
:105C0000070E015C0DE256ECD8F0EF9E56ECD8F092
:105C1000EF500E0803E156ECD8F0EF6A012AF0D7F6
:105C20000FC1A8F10A0E01011003F35011259E6F58
:105C30000A0E1203F35013259F6F0A0E1403F3CFBD
:105C4000A0F1A26BA2C1A1F1040E0201775D0DE2E9
:105C500069510BE112C1A8F10A0E01011303F350BF
:105C600014259E6FA06BA0C19FF10201690508E198
:105C700011C1A8F19FC19EF1A0C19FF10101A06BCC
:105C8000020E0201695D0EE110C1A8F10A0E0101C8
:105C90001103F35012259E6F0A0E1303F3501425BF
:105CA0009F6FA06B9A0E076EA1EC0CF0006E005077
:105CB00013E10101A85103E19E51380802E2258E4B
:105CC0001200BAECCDF00A0E005C06E10101E351CE
:105CD000010B02E010EF09F000C02BF12984FFEC6A
:105CE000CEF074EC21F052ECD8F09A0E491808E18D
:105CF0004A5006E10101B59BB59903D80C0E076E19
:105D0000120067ECD4F02582238A12003EC2A7F16C
:105D10003FC2A6F140C2A5F10101A46BA36B1FA471
:105D200002D09EEF31F0C2EF31F004902C50100BF6
:105D300001E004805EECC5F02C50100B01E0010E78
:105D4000496E0450010B495C02E009ECCFF01200EF
:105D5000D1ECDAF001018DA715D0FE0EDB5008E082
:105D6000FD0EDB5005E1DF68CFA102D0010EDF6E32
:105D7000FE0EDB5007E1FD0EDB5004E0010EDF6E8E
:105D8000CFB1DF68DF5021E0F4ECCAF0A76BA7C108
:105D9000A4F1A7C1A3F19FECD9F001E0010E496E77
:105DA000DF0402E0000E01D0010E491802E0C6DA5D
:105DB00001D0E8DA7CEC04F01EAC03D002010981CA
:105DC00002D00201068305014781E552C2EFC9F006
:105DD0000101A76BA66BA56B02018851E824496EEF
:105DE000640ED4ECD7F03CECFEF03AC0A4F1320ED5
:105DF00011ECD6F088C23EF03CECFEF03EC0A3F1C0
:105E0000020189A102D09EEF31F0C2EF31F095EC92
:105E1000D6F09AC23BF03C6A3D6A3E6ADBECCEF0BB
:105E2000FBECFBF037C0DEFF38C0DEFF39C0DEFF21
:105E30003AC0DDFFDD52DD529BC249F04A6A4B6A2F
:105E40004C6A100E406E270E416EB1ECCAF0AFECFA
:105E5000CCF09CC249F04A6A4B6A4C6A640E406EB0
:105E6000416AB1ECCAF0AFECCCF00A0E02019D031E
:105E7000F3509E25496E4A6A4B6A4C6AAFECCCF0EF
:105E8000DECF3BF0DECF3CF0DECF3DF0DDCF3EF0AD
:105E9000DD52DD52040EE15C02E2E16AE552E16EA0
:105EA000C2EFC9F007AE6ED02B50400B03E02C5070
:105EB000200B31E0800E0101C41505E1C4510CE155
:105EC0001F0EC55D09E2C46B1F0EC56FC86BC8C14C
:105ED000C7F1C8C1C6F11FD0100E2B5D1CE2360EF3
:105EE000006E0050C45D03E300C0C4F10DD0200E6D
:105EF000C45D11E32C0EC45D0EE2260EC45D02E209
:105F0000200E01D02C0EC46FC86BC8C1C7F1C8C128
:105F1000C6F1C8C1C5F12B50400B03E02C50200B3B
:105F200031E1800E0101C91505E1C9510CE11F0ED7
:105F3000CA5D09E2C96B1F0ECA6FCD6BCDC1CCF132
:105F4000CDC1CBF11FD0100E2B5D1CE2360E006EC2
:105F50000050C95D03E300C0C9F10DD0200EC95D3A
:105F600011E32C0EC95D0EE2260EC95D02E2200E81
:105F700001D02C0EC96FCD6BCDC1CCF1CDC1CBF111
:105F8000CDC1CAF12B50400B03E02C50200B1DE07B
:105F90002050400B03E11250080B0FE12050400B42
:105FA00012E01F50020B03E11250040B06E11F50D8
:105FB000020B09E01250080B06E0F4ECCAF0A6DE72
:105FC000B4ECCFF002D0BFECCFF02B50400B03E08D
:105FD0002C50200B16E11F50020B11E01250040B45
:105FE0000EE0BAECCCF092DE9EC1BFF19FC1C0F1D1
:105FF000A0C1C1F1A1C1C2F1A2C1C3F102D0CAECDA
:10600000CFF01F50020B18E102018951010B03E18F
:106010008951020B11E09CECCAF006E02050800B85
:106020000BE0050E9D5D08E12050400B05E0C5EC3E
:10603000CCF0CEDEB4ECCFF001013BA974D0BAC1F4
:106040009AF2BBC19BF2BCC19CF2BDC19DF2BEC124
:106050009EF2DDDE3BC0C8F73CC0C9F73DC0CAF7C1
:106060003EC0CBF7BFC19AF2C0C19BF2C1C19CF246
:10607000C2C19DF2C3C19EF2CADE3BC0CCF73CC098
:10608000CDF73DC0CEF73EC0CFF70701C851CC5F7A
:10609000C951CD5BCA51CE5BCB51CF5B0101D2A1BF
:1060A00008D0400E0701CC271F0ECD23000ECE23B3
:1060B000CF23049C1E50200B01E0048CD8800701E4
:1060C000CF51FF0A08E6680ECC5DC50ECD59FF0E14
:1060D000CE59FF0ECF5919E3CF35000ECF1909E67F
:1060E000D880980ECC553A0ECD55000ECE55000EE8
:1060F000CF550BE3CCC70EF0CDC70FF0E5ECCBF0DE
:10610000A50EECECC9F01E8A01D01E9A0450400B7B
:1061100001E0010E496E1E50200B01E0010E495CAA
:1061200002E052ECCCF02BAC96D0800E071401E1CB
:1061300092D0100E01012B5D01E38DD02CBA0DD051
:10614000D5ECCFF0C9C1A3F1CAC1A4F1CBC1A5F16F
:10615000CCC1A6F1CDC1A7F10CD0C5ECCCF0C4C127
:10616000A3F1C5C1A4F1C6C1A5F1C7C1A6F1C8C1BB
:10617000A7F1BAECCDF02C50200B2EE0005001011D
:106180002B5D2AE000C00DF100C02BF12BC1D3F133
:1061900066ECD3F0E3ECCEF0056E2CAA06D0050E2B
:1061A000E66E0524F8ECD1F005D0050EE66E05503C
:1061B0007CECD0F034ECCAF00E0E0524CBECCBF026
:1061C0000101D29B00BAD28B096AE2EC35F0208241
:1061D0000201010E246F01D0A8DD0701C2510101A7
:1061E000C45D04E07CEC0DF0C4C1C2F701012B5189
:1061F00032E12B50080B2FE0020E3A5D2CE13DEC12
:10620000D7F004E034ECD2F0E806FCE10701C65117
:106210000E1802E1C7510F181EE0006A5A0E0E1840
:1062200007E10F5005E1590EC61901E1C7510AE017
:10623000590E0E1808E10F5006E15A0EC61903E177
:10624000C75101E1002A0EC0C6F70FC0C7F70050C2
:10625000E66E02D8E5521200C6ECC9F001013951D0
:106260006BE12B5169E12B50080B66E0FE0EDB5011
:1062700003E1020E3A5D60E13DECD7F004E034EC5E
:10628000D2F0E806FCE10EC0C6F70FC0C7F7190E42
:10629000A0ECD0F003E2036802681DD0410EA0EC30
:1062A000D0F015E20CECD6F0190E495E000E4A5AF9
:1062B0004950016E15ECD6F00800F550026E15EC51
:1062C000D6F0F62A81ECD0F0F550036E04D069C305
:1062D00002F06AC303F0010196A904D069C302F079
:1062E0006AC303F0FE0EDB5007E10701C351025CF5
:1062F00003E1C451035C20E002C0C3F703C0C4F74C
:10630000410EA0ECD0F011E201019651100B0DE10D
:10631000010EE66EE66A0350E66E0250E66EE4ECAD
:10632000CDF00B0EFDECD1F005D0FE0EDB5002E0FF
:106330006CECD3F06EECD1F0C2EFC9F00101A751C3
:10634000A227A251090803E20A0EA25FA12BA651BF
:10635000A127A151090803E20A0EA15FA02BA551B4
:10636000A027A051630803E2640EA05F9F2BA451F5
:106370009F279F51630803E2640E9F5F9E2BA351EA
:106380009E2712000101A751A25FA2510A0803E251
:106390000A0EA227A107A651A15FA1510A0803E294
:1063A0000A0EA127A007A551A05FA051640803E22F
:1063B000640EA0279F07A4519F5F9F51640803E2CA
:1063C000640E9F279E07A3519E5F12000101E6A560
:1063D00036D0E5A902D0310E01D05E0E9E27E0EC4A
:1063E000CFF015DDC3ECCDF0030E22ECD8F008ECB5
:1063F000D9F00EECD9F03BC09EF119ECD1F0ADEC28
:10640000CBF0100E406E270E416E426A436A11ECCB
:10641000FDF03BC09FF137C00EF038C00FF0E4EC48
:10642000D4F03CECD6F03DC0A0F16BECCAF039C022
:106430003EF03CECFEF03EC0A1F13AC0A2F11200E9
:1064400047ECD5F02BBC03D01AD82F9E10D02CAA25
:1064500007D02050400B0AE01F50020B08E106D085
:106460002050400B04E01F50020B01E008D8020E40
:10647000E15C02E2E16AE552E16EC2EFC9F047EC8D
:10648000D5F00101E851010BDE6EDD6A1F50020BF1
:1064900006E02050400B03E0D5ECCFF002D0C5EC75
:1064A000CCF0A76BA7C1A6F1A7C1A5F1A7C1A4F124
:1064B000A7C1A3F120ACE8912050400B10E1D451CA
:1064C0000EE19FECD9F001E0010E74ECCDF002E09A
:1064D000000E01D0010E491801E081D07CD020507F
:1064E000400B12E03450400B0FE09FECD9F001E07C
:1064F000010E496E020ED45D02E0000E01D0010EC5
:10650000491801E189D06BD02050400B19E1D40526
:1065100003E0020ED45D14E16BECD4F011E2010152
:106520000F0EA56FE651040B01E0010E496E020E3D
:10653000D45D02E0000E01D0010E49184CE04FD0AE
:10654000EFECD2F014E00101090EA56F010EA66F69
:10655000050EA76FE651040B01E0010E74ECCDF0BF
:1065600002E0000E01D0010E491835E038D020506D
:10657000400B13E1A4ECD0F010E001010A0EA56F6E
:10658000E651040B01E0010E74ECCDF002E0000EC8
:1065900001D0010E49181FE022D02050400B21E10C
:1065A0009CECCAF003E0040ED45D1BE1010EA46F65
:1065B000140EA56F040ED45D03E1E6A510D00BD038
:1065C000E651040B01E0010E496EE551800B01E03C
:1065D000010E491804E0D6DE0101E8811ED0AEDECE
:1065E0001CD02050400B19E09CECCAF016E1A46BC3
:1065F000A4C1A3F1A56B5751080B0AE1E651040BA6
:1066000007E002018951040B03E00101140EA56F9C
:106610000101A76BA7C1A6F1B5DE0101E651010B8F
:106620002DE02050400B2AE1020114511DE0010130
:10663000E851010B496E4A6ADF50491813E1DE52F6
:10664000DD504A180FE10201A0510101A45D0AE1E9
:106650000201A1510101A55D05E10201A251010163
:10666000A65D02E005014785A3C19FF2A4C1A0F287
:10667000A5C1A1F2A6C1A2F2A7C1A3F228ECD2F053
:1066800015E02050400B12E1050ED45D0FE0040E22
:10669000D45D0CE0A36BA46B500EA56FA76BA7C1D4
:1066A000A6F1E6A502D04ADE01D06CDE0101E6B516
:1066B0008DDE52ECCEF01BE2100E2B5D0DECCFF018
:1066C0000101A46BA4C1A3F1A3ECD9F0A56FA8ECC0
:1066D000D9F0A66FA76BE651040B01E0010E496EDD
:1066E000ADECD9F0491802E04DDE01D027DE010102
:1066F00096B374D057A943D057AB70D0D2C70EF021
:10670000D3C70FF0260ED8800E54020E0F5406E2A7
:106710000480260E0E5E020E0F5A06D00490260E3E
:10672000D8800E56020E0F569F51496E4A6A9E51EE
:10673000640DF3504924D86FF4504A20D96FD8C162
:106740004DF0D9C14EF088ECCBF037C03BF038C0EB
:106750003CF039C03DF03AC03EF0880E406E130E5A
:10676000416E426A436A11ECFDF03BC00EF03CC042
:106770000FF022ECCDF004A030D004DE2FD09EC16B
:1067800000F0000405E19F51310802E2020E006EA4
:10679000030E005C05E19F51310802E2040E006E19
:1067A00098514F6E506A00504D6E4E6A0A0E4B6EF5
:1067B0004C6AB2C23DF0B3C23EF093ECDAF0E2ECC8
:1067C000FDF02CECDBF087ECCFF04FC042F050C076
:1067D00043F0EAECCCF022ECCDF0B0DD60ECCCF094
:1067E00003E1D7ECD2F019E00601F0510101A05D00
:1067F00014E10601EF5101019F5D0FE10601F15126
:106800000101A15D0AE10601F2510101A25D05E16C
:106810000601EE5101019E5D0CE09EC1EEF69FC1A6
:10682000EFF6A0C1F0F6A1C1F1F6A2C1F2F6D3ECE9
:10683000C5F0020EE15C02E2E16AE552E16EC2EFF0
:10684000C9F0D9CFE6FFE1CFD9FFBAC19EF1BBC1F4
:106850009FF1BCC1A0F1BDC1A1F1BEC1A2F1010176
:10686000A86BFE0EDB500A0807E22996FE0EDBCF6E
:10687000E6FFC9EC2CF0E5520101006B800E01012E
:106880001315036E800E01011015026E010EEA6EE3
:106890009E5105D89F5103D8A05101D814D0076B41
:1068A000066F0A0E065DD8A003D0066F072BF9D736
:1068B00000510E0FE96E0751EF6EE92A0651EF6E97
:1068C000002B002B000CA1C114F1A2C115F1010194
:1068D000A85107E10A0E01019E5D03E20101100EBD
:1068E0000E6F0701BEBB03D00101100E156F07012B
:1068F000BEAD05D00101100E146F14C115F11DBC01
:1069000003D00101108F03D00250010110130101C7
:10691000138F0101A85109081AE20201365117E04C
:106920006CECDBF00101020E006F9EC100F061EC27
:10693000E1F0A8C100F00101006B61ECE1F0010E93
:10694000E66EE66A33EC09F0E552E55223D0010128
:10695000A8511FE007010701BE51200B1AE1288C46
:1069600014C115F113C114F112C113F111C112F1C7
:1069700010C111F10FC110F10EC10FF10A0E496ED5
:1069800049C043F0A8C13EF03CECFEF03AC00EF125
:1069900001D0289CE552E7CFD9FF1200D9CFE6FFFE
:1069A000E1CFD9FF020EE126010EA8C1DBFF2BC10A
:1069B000DFFF0101D551EA6AB80FE96E070EEA223E
:1069C000EFCFBFF7BFC19EF1C0C19FF1C1C1A0F120
:1069D000C2C1A1F1C3C1A2F10101A86BDF500A0835
:1069E00006E22996DFCFE6FFC9EC2CF0E552010163
:1069F000016B800E01011B15026E010EEA6E9E51A5
:106A000005D89F5103D8A05101D816D0076B066F47
:106A10000A0E065DD8A003D0066F072BF9D70151E7
:106A2000160FE96E0751300FEF6EE92A0651300F4D
:106A3000EF6E012B012B000C300E0101A12501018D
:106A40001C6F0101A85107E10A0E01019E5D03E2DE
:106A50000101200E166F0701BFAD03D00101200E0A
:106A60001C6F0101188F01011B8F0101A8511DE04E
:106A700007010701BF51200B18E11BC11CF11AC10E
:106A80001BF119C11AF118C119F117C118F116C17A
:106A900017F10A0E496E49C043F0A8C13EF03CEC24
:106AA000FEF03A50300F0101166FA8C1A9F1010E96
:106AB000DBCFA8F1020EE15C02E2E16AE552E16E91
:106AC000E552E7CFD9FF120043ECD5F0830E096EF3
:106AD0000A0EE66E01010D03F350E66E5E0EE66EE1
:106AE000020E34ECCAF0DE0ECBECCBF00050DF6EC1
:106AF000FE0E4DECDBF00101E59D2E9EB90E005C13
:106B000016E1FF0E02015E5D12E02E8E020E010103
:106B10002B5D0DE1050E0201635D09E1210E5F5D54
:106B200001E1606B280E645D02E13C0E656FA30E0F
:106B3000DF5C02E10101E58DE552C2EFC9F08C0E88
:106B400002018D1909E10A0E8E1906E18C0E8F19CA
:106B500002E10A0E901917E00F0ED8808D55270E0E
:106B60008E5510E28DC249F08EC24AF04B6AD89021
:106B70004B50000A06E6F00E495CD80E4A58000E4B
:106B80004B5801E3000C010C0201915102E19251BA
:106B900007E0FF0E915D04E0FF0E925D01E0000C46
:106BA000010C2B50080B0DE0E4ECD5F00AE12B5161
:106BB00006E1010EE66E2CEC31F0E55212006CECB1
:106BC000D3F0120018B03DD00DC1E6FFBBEC5AF077
:106BD000E552B5DF000902E0C6ECD0F00DC1E6FFDA
:106BE000D5EC5AF0E552D0DF000903E00201916BC9
:106BF000926BB7EC15F068DF01015651080B03E109
:106C00002B51090809E2FF0E02018A5D02E1320EF2
:106C10008A6F8AC248F108D0FF0E8C5D03E1320E04
:106C20008C6F02D08CC148F1A2EC41F001015F8D64
:106C3000E6B55F9DE6ECC3F04DECCCF0E0ECD1F0B6
:106C4000B0DFF4EFD1F043ECD5F0FD0EDB50100DCA
:106C5000F350DF6E010E096E0201680E986FFD0E93
:106C6000DB500A080AE2020E096E690E986FFD0EEB
:106C7000DB50F00F100DF350DF6EFE0EDB50FF08FF
:106C800002E047ECD7F0DF50E552C2EFC9F0020155
:106C9000875103E08751330802E20D0E876F885158
:106CA00037ECCBF007E24950FA08000E4A5402E2F2
:106CB0001E0E886F89BF896B93510E0803E2936B98
:106CC0000101D09B120088ECD6F0FF081BE047ECD6
:106CD000D7F00F0E4FECD8F00A0E005C07E101016F
:106CE000E351010B03E0096A000EB9D100C02BF19A
:106CF00001018A51100B06E00A0E4CECCAF002E2C8
:106D0000FE0EDB682BC10DF10201756B0101E695EA
:106D1000E5992B510A0838E2100E2B5D006E0050E9
:106D2000F7ECD6F029E018ECD8F001010D6FFAEC81
:106D3000C9F0EF380F0B0201756F91ECD6F024E02B
:106D40001B50020B0EE02B50080B03E12250080BE6
:106D500008E00101E68515ECD7F0460815E1E58964
:106D600013D00701020E266F1BA202D0050E266F5C
:106D7000180EFFECCAF008D0FE0EDB680101090E08
:106D80000D6F0DC12BF1258E0101E6A50FD02BA6AD
:106D900005D007011397140E70ECD4F022A603D08F
:106DA000010E70ECD4F00701149F0FD02BA605D074
:106DB00007011387140EFDECD1F022A603D0010EBB
:106DC000FDECD1F00701148F14935BECD5F00101B9
:106DD00075ECD4F001E0098FBBECDAF007010B8908
:106DE0000101E6A502D007010B999BECC4F002015A
:106DF000D86B9AECCBF0100E80ECD7F029A403D01E
:106E00007CEC04F029940F0E0101CE15D46FCE391D
:106E10000F0BD56FD551060802E2D4C1D5F1D405C8
:106E200001E1CF91020ED45D01E1CF81FFECD9F0F9
:106E30000A6E040EE66E0B0EDF24E66EDC0EE66EC6
:106E4000010E34ECCAF09AECCBF0FE0EDB50FF08DA
:106E500003E198C209F002D0100EDF26100ED5EC27
:106E6000DAF07AECD8F0FE0EDB50FF0852E0E3ECEB
:106E7000CEF0DF6E0B0E4FECD8F019ECCCF008E042
:106E80001F0ECF17E00E0014CF13FFECD9F00A6EDF
:106E90000C0E4FECD8F0440E0101D017BB0E0014BD
:106EA000D01302ECDAF0470E0101D117B80E00142E
:106EB000D11302ECDAF09E0E0101D217610E00141C
:106EC000D21398C209F00A0EE66E030EDF24E66EB6
:106ED0008A0EE66E020E34ECCAF0E3ECCEF0DF6E02
:106EE0000C0E4FECD8F0440E0101DD17BB0E001460
:106EF000DD1302ECDAF0470E0101DE17B80E0014C4
:106F0000DE1302ECDAF09E0E0101DF17610E0014B1
:106F1000DF13096AC4C119F5C5C11AF5C6C11BF54D
:106F2000C7C11CF5C8C11DF5C9C11EF5CAC11FF5F1
:106F3000CBC120F5CCC121F5CDC122F518B41CD0B0
:106F400012941296129A1F92010138A30CD0D1A16B
:106F500002D0128A1F821296D1B312861294D1A542
:106F600009D0128407D01FECD3F00101DE95DE9327
:106F7000D195D19381EC9AF052ECCEF03DE25C0ECB
:106F80000D257BECCBF0006E00500101C45D016E5D
:106F900001AE03D0C451005C016EE651040B03E165
:106FA0000150030803E3015019080AE2050EF6EC4C
:106FB000D0F0C40EE66E010E92ECCAF000C0C4F12F
:106FC00000500101C95D016E01AE03D0C951005CE2
:106FD000016EE651040B03E10150030803E3015085
:106FE00014080AE2050EF6ECD0F0C90EE66E010EAA
:106FF00092ECCAF000C0C9F102ECD2F056EC25F0D8
:107000000EEC0DF0129C01013BB1128C129E3BB3B1
:10701000128E53EC64F0129801013BB912888BEC8C
:1070200020F00101D09F1190118271EC09F081ECE8
:107030004EF03CEC4EF0096A010137A702D01BEC80
:1070400048F0BFECCFF0CAECCFF0BCDD0101246BFF
:107050001DBC04D00701A16B66ECD3F0010EE55214
:10706000C2EFC9F043ECD5F00B0E01012B5D11E22C
:10707000C5C1E6FFC4C1E6FF3DEC21F0E552E55293
:10708000005001012B5D05E00701020E02ECD7F074
:107090006ED00A0E2B5D02E248C18CF19AECCBF067
:1070A00083EC20F00101D09F38A30DD0F80ED1174A
:1070B000D1911FB2D181D19312B6D183D19512B49F
:1070C000D185D4EC40F02BC1D3F150ECD7F0050EB4
:1070D0007CECD0F0D5ECDAF02FECCAF00A0EDF240D
:1070E000016E0101D539F00BD411ACECD0F0050ED6
:1070F000E66ECF0EE66E010EE66E0B0EDF2464EC3C
:10710000D6F0050EF8ECD1F0E66E050EDF2464EC47
:10711000D6F01CBA24D09AECCBF001015651080BE2
:1071200003E12B51090802E248C18AF239ECBCF0B4
:107130003AC18BF2FE0EDB50FF0803E198C209F062
:1071400002D0100EDF26100EE66E870EE66E020EDF
:10715000D5ECDAF02FECCAF0096AC2EC13F00101A9
:1071600037A702D055ECCFF0096A0201206BE55237
:10717000C2EFC9F043ECD5F00F0EDF6EF40E06013E
:107180000017F00E0517DF500617E552C2EFC9F0E1
:10719000060106910095019102990199149913999C
:1071A000049903911200C6ECC9F0E4ECD5F001E0BB
:1071B000010E496EFE0EDB5002E0000E01D0010E02
:1071C000491803E00601058502D006010587010183
:1071D0008AA102D00601068DC2EFC9F00050050A4F
:1071E0004FE0010A4AE0070A22E0010A1BE0030A15
:1071F00017E0010A01E0120006010583E4ECD5F076
:1072000001E0010E496ED051400B01E0010E49181A
:1072100002E0060105810601EA5146E0068B1200F4
:10722000E66A02D0010EE66EBEDFE55212000601EC
:107230000081E4ECD5F001E0010ED0ECD0F002E0EA
:10724000060105810A5003E0030E0A5C02E1060113
:10725000057103ECD5F002E00601068B32A024D0C4
:10726000E4ECD5F001E0010ED0ECD0F003E0060133
:107270000587120006010585120006010083120031
:107280000601008702018951040B04E03A5102E132
:107290000601068B020189A102D00601068D0201BA
:1072A00089A302D00601068F1200800E071406E0A3
:1072B0002050010B03E1D4C100F003D044EC20F0D6
:1072C000006E58DFEEEF38F01200C6ECC9F019EC92
:1072D000CCF00DE10A0403E0020E0A5C04E1D05197
:1072E000040B16E10BD0CF51040B08E011D0D405EC
:1072F00007E16BECD4F002E2420E21D0450E1FD024
:10730000020ED45D07E16BECD4F002E2400E17D020
:10731000440E15D0050ED45D07E1E551800B02E067
:10732000480E0DD0470E0BD0040ED45D02E1460E80
:1073300006D0D051400B02E1430E01D0410E2CEC9F
:10734000CAF091ECCDF0030E005C12E10A0403E0F8
:10735000020E0A5C05E10101D051040B05E106D0E3
:107360000101CF51040B02E0540E1CD0550E1AD06F
:10737000000402E1520E16D0020E005C02E1500E33
:1073800011D0050E005C02E1570E0CD0040E005C1B
:1073900002E1560E07D00101D051400B02E1530E1D
:1073A00001D0510E2CECCAF0C2EFC9F08CECD6F033
:1073B0009CECCAF00CE12A50020B01E0010EE66ED3
:1073C000D950010F2EECCCF02A9271EC16F033B8A4
:1073D00042D02050800B12E11450100B0FE01450DB
:1073E000200B0CE10101D45106E0030ED45D03E053
:1073F000050ED45D03E11498C4EC4FF02050800BCF
:107400000AE11450200B07E09CECCAF004E1149A46
:107410001498C4EC4FF019ECCCF003E0050ED45DE9
:1074200001E1D29D1390D45103E113908AB51380EA
:10743000030ED45D05E10A5003E013908EB513806E
:10744000139A13A0138A71EC0CF053EC64F0EAEC7D
:1074500018F056EC25F0258220EC32F0010EE66E95
:1074600034DFE552C1EC16F0FFEC1DF033B85FD00D
:10747000D5CAE6FFAB0E0AECCAF0FCEC18F0C4EC7F
:107480004FF059EC0FF08FEC1FF0B0EC1EF028B26B
:107490004ED01C9834902450010B05E12750200B4E
:1074A00002E0E7EC08F00E6A0F6A30ECD2F004E17B
:1074B000100E0E6E270E0CD0050ED45D04E1240EC6
:1074C0000E6E2C0E05D0D2A104D0400E0E6E1F0EF3
:1074D0000F6EE5ECCBF0A40EECECC9F09CECCAF01E
:1074E00003E0050ED55D02E155EC0CF0A5EC1EF0B5
:1074F0006F0E2CECCAF028EC53F01CEC1FF07CEC67
:107500001DF009EC19F05AEC15F083ECCAF002E01A
:1075100010EC1EF082EC15F0050E005C02E11DEC93
:1075200009F099EC23F0B6EC64F0D5ECC4F09CECD7
:10753000CAF00AE1010EDB502A92E8B02A822AB290
:1075400003D02A8278EC16F03398030EE15C02E255
:10755000E16AE552E16EC2EFC9F08C9800000000CC
:10756000030EE66E8DEC5CF0E552040E095CE66EEF
:107570008DEC5CF0E5520150E66E8DEC5CF0E5526E
:10758000B5ECFDF0006E00008C881200D9CFE6FF4C
:10759000E1CFD9FF8C9800000000060EE66E8DEC5E
:1075A0005CF0E5528C880000000000008C98000020
:1075B0000000020EE66E8DEC5CF0E552040E095CF4
:1075C000E66E8DEC5CF0E5520150E66E8DEC5CF001
:1075D000E552FE0EDBCFE6FF8DEC5CF0E5528C88C9
:1075E000020EE66E87ECFDF0E552E552E7CFD9FFDB
:1075F000120047ECD5F00050DF6E010EDB6A37D881
:10760000DF50005C2CE0040E095C16E2F29EA698A6
:107610000950636E0150626EDF50616E7F9E7F9CE9
:107620007F84550E7E6EAA0E7E6E7F82F28E040ED1
:1076300006ECD7F07F9413D0010EDB2ADFCFE6FFF4
:10764000A5DFE5528ADFDF50005C02E0FCEC0CF0C5
:10765000DF50005C04E0050E44ECCCF0EDE3020EDC
:10766000E15C02E2E16AE552E16EC2EFC9F047EC8B
:10767000D5F0010EDB6A040E095C0AE20950636E64
:107680000150626E7F9E7F9C7F806150006E12D0A1
:10769000010EDB2A62DF0050DF6E5FDF0050DF5C2F
:1076A00002E0FCEC0CF00050DF5C04E0050E44EC62
:1076B000CCF0EEE3020EE15C02E2E16AE552E16E3B
:1076C000C2EFC9F0C6ECC9F00CECD0F012E0FC0E31
:1076D000DBCFF3FFDB2AF350CBECCBF0FD0E05EC58
:1076E000DAF0FE0EDBCFEAFF01E3DB2A00C0EFFF9A
:1076F000EBD7C2EFC9F0C6ECC9F00CECD0F01AE041
:10770000D6ECD1F017E3CCECD8F005E24950A40850
:10771000000E4A540FE35DECD1F0016EFC0E05EC57
:10772000DAF0FD0EDBCFEAFF01E3DB2AEF50ACEC31
:10773000D0F0E3D7C2EFC9F0C6ECC9F01F0E0501C7
:10774000235D0DE2232B2551EA6A270FE96E050E12
:1077500006ECD8F0252B25511F0801E2256BC2EF5E
:10776000C9F0C6ECC9F0030E0A5C54E10E6A0F6A58
:10777000FE0EDB500D0803E11F0E0E6E0F6AFE0EAB
:10778000DB500A0803E11D0E0E6E0F6AFE0EDB5081
:10779000090803E1EF0E0E6E0F6A07ECD5F003E166
:1077A0000E68020E0F6EFE0EDB507F0804E1B50E70
:1077B0000E6E030E0F6EFE0EDB501F0821E27F0ED1
:1077C0004CECCAF01DE2410E4CECCAF00CE3FE0E8C
:1077D000DB505A0808E3200E496EFE0E27ECD8F065
:1077E000FE0EE7CFDBFF0C0E496ECD0E4A6E010E8A
:1077F0004B6EFE0EDB50E00F60ECDAF014ECD9F0CB
:107800000E500F1049E00FC0E6FF96DFE5520EC0A4
:10781000E6FF3DD0FE0EDB50090803E1200EFAEC36
:10782000CEF0016A400E015C37E2EB0E4A6EDA0ED2
:107830004B6E010E4C6E0150CEECCAF0FE0EDB50CA
:10784000495C28E1030E066E01B0068C01B2068A7F
:1078500001B4068801B6068601B806842350040BDD
:1078600009E1200E011406E06F0EE66E65DFE552B9
:1078700023840BD02350040B08E0200E011405E1F3
:107880007F0EE66E59DFE55223940650E66E54DF14
:10789000E55202D0012AC6D7C2EFC9F043ECD5F0B9
:1078A000800E4CECCAF003E3200EFAECCEF002019D
:1078B000050E2D6FFE0EDB50740810E1010E2D6FCA
:1078C000030E0A5C07E105012351CFECD8F0020F4B
:1078D00002012D6F0501106B1D822BD0FE0EDB50B7
:1078E00028E0DF6A150EDF5C11E21BECD9F00BE13A
:1078F000DF2A4AECCDF07AECD4F0DF2A4AECCDF066
:107900007AECD4F003D0030EDF26ECD7150EDF5C43
:1079100004E179ECD5F025DFE552200E4CECCAF0FD
:1079200003E2200EFAECCEF079ECD5F0C3EC6FF068
:10793000E552E552C2EFC9F047ECD5F023A01CD0C8
:107940001DB013D02750200B06E0E9ECCAF003E08D
:107950000201050E2D6F020E0201535D1FE30701A8
:10796000016B026B53C254F219D00201532B5351D5
:1079700080081EE2800E1BD01DA013D0070E070149
:10798000015D0AE2012B02910243020E0201535DE6
:1079900005E30701028F02D0070E016F0201010EFD
:1079A00006D00201532B5351800802E2800E536F20
:1079B0001D9023B01D802350010B03E1020E535D87
:1079C00004E01D50020B01E18AD01DA204D0070182
:1079D000CC0E026F0FD0070102910243028F070EF7
:1079E000D8800155016E01500106000903E00291A3
:1079F0000243F9D700C709F00101B5A7E88B0201DE
:107A0000545107081DE254513F0802E23F0E546FE3
:107A1000EFECD1F006E0200E11ECCDF0200E7AEC68
:107A2000D4F0AFECD0F00CE00701035109E0800E78
:107A300002015425006E03C701F007010307D9DDD9
:107A4000780E0701025D18E2298A02C7E6FF3CECC6
:107A500004F0E552DF6EDF500EE0EFECD1F00BE00A
:107A60002D5104E0DFCFE6FF19DF04D0DFCFE6FFC2
:107A7000C3EC6FF0E552299A0101E89BB5A72FD01E
:107A80000701035105E002C700F003C701F0B1DDB3
:107A90000701035106E01D50020B03E11C0E025DBD
:107AA0001BE103510AE01C0E025D07E1CC0E006EE3
:107AB000030703C701F09DDD1D820101B5974DEC61
:107AC00065F0230E155C03E1410E7EECCAF02492B2
:107AD00023AC03D0248201D003070701026B096A9B
:107AE000020EE15C02E2E16AE552E16EC2EFC9F02A
:107AF00060ECCCF00CE11C0E0101B95D08E11850FE
:107B0000400B05E084848C808D8A8D8C12000601E8
:107B10005051040B02E08D8C01D08D9C5051080B0C
:107B200002E08D8A01D08D9A5051010B02E08C80C9
:107B300001D08C905051020B02E084841200849496
:107B40001200000012000601D99D8850800B01E050
:107B5000D98DD99F8850400B01E0D98FD991885099
:107B6000100B01E0D981D9938850200B01E0D98313
:107B7000D9998850080B01E0D989D99B8850040B0A
:107B800001E0D98B1200C6ECC9F0FD0EDB504CECC5
:107B9000CAF008E3FE0EDBCFE6FFFD0E6BECD2F081
:107BA0000AE207D0FD0EDBCFE6FFFE0E6BECD2F053
:107BB00002E2010E01D0000EC2EFC9F08CECD6F04B
:107BC0002EB254D082B003D00701290E76D082B2F3
:107BD00003D007012C0E71D0DF6A060EDF5C43E292
:107BE000DF50040DF350830964ECD0F0050EDF5C28
:107BF00003E1DE52BB0EDD6EB2ECD9F000C047F7F8
:107C000000501A082EE2F00E005C2BE2FE0EDB5054
:107C100002E1010E56D0B2ECD9F000C048F7005096
:107C20001A081FE2F00E005C1CE2B2ECD9F000C0B2
:107C300049F700501A0815E2F00E005C12E2080E37
:107C4000E66E48C7E6FF47C7E6FFE9ECCDF009E07E
:107C5000080EE66E49C7E6FF48C7E6FFE9ECCDF03F
:107C600002E1DF2ABAD7060EDF5C02E1000E29D05E
:107C7000010E62ECD4F073ECD2F010E20C0EE66E62
:107C8000020EDB50370F57ECCCF0E66E48C7E6FF2C
:107C9000E9ECCDF003E1020EDB2AEDD773ECD2F074
:107CA0000FE247C74AF748C74BF749C74CF7020EE0
:107CB000DB50080DF350DF1007014D6F4D5101D01F
:107CC000800E496E030EE15C02E2E16AE552E16E6C
:107CD0004950C2EFC9F016ECCFF0BBECD2F006E190
:107CE0009CECD0F003E001011E0EAC6F01012D0EE3
:107CF000176F1FA402D02B0E176F0201405107E12E
:107D00003F5105E13E5103E10101200E176F6BEC7D
:107D1000CAF040C23EF092ECCCF00101186F300E78
:107D20003A24196F300E02013F2501011A6F070135
:107D3000BEAB05D0300E02013E2501011B6F0101D3
:107D4000198F120088ECD6F02CECCBF0EFCFDFFFD0
:107D50000101A36BA46BA56BA66BA76B1DAE03D033
:107D6000050EA56F32D035ECCEF0EF50400B03E19D
:107D70002750040B1DE079ECD5F015EC0DF0E55221
:107D800000C0A5F1005063081BE20101A56BA42B04
:107D90007D0E005C02E1190EA56F4FECDAF0FA0ED1
:107DA00049180EE14A500CE1A42B320EA56F08D001
:107DB00035ECCEF0EF50200B02E0A72B01D0A62B24
:107DC0002AAE03D0020EF1ECC9F0E552C2EFC9F0C1
:107DD000AC0E006E005098ECCEF035C100F00FEC08
:107DE000D5F001011A5D05E12CECD8F002E1200E7E
:107DF0001B6F0201060E3D6F56EF25F0C6ECC9F071
:107E0000960E496EDD0E4A6E010E4B6E050E4F6EDC
:107E10004FC043F0FE0EDBCF3EF03CECFEF03EC028
:107E20004CF031ECDBF0006E6CECDBF00101020E8B
:107E300008ECD4F0128F0C0E4CECCAF003E20E0EDC
:107E40000F6F0ED00E0E106FFE0EDB50630802E2B5
:107E5000100E106F0F0E4CECCAF002E2090E116FFB
:107E6000140E146F120E156FC2EFC9F0C6ECC9F0F4
:107E70007CECDBF00101012BFE0EDB50006E7EEC92
:107E8000E1F02B50100B07E1640E4CECCAF003E25A
:107E90000101200E176F2BA807D001014D0E1B6F9B
:107EA000570E1C6F188F16D0FD0EDB5003E1010139
:107EB000198F07D00A0E4CECCAF003E20101200E24
:107EC000186F0101570E1B6F33B602D02A0E1C6FBC
:107ED0005FB31C8FC2EFC9F0C6ECC9F056EC25F0B9
:107EE000FE0EDB5003E0E8ECD4F003D00068BFECFA
:107EF00026F064ECCBF01AE0020E0101395D0FE1CF
:107F0000A50E485D0CE17CECDBF0090EE66EE40E9C
:107F1000E66E010EE66E25ECE2F0E5520BD0010EA6
:107F2000E66E79EC05F0A60FE66E03D0E66A48C16E
:107F3000E6FF9CDFE552E5522BA807D00068B3ECC2
:107F400026F048C1E6FF5ADFE552C2EFC9F043EC24
:107F5000D5F056EC25F0B40E40ECD2F034C1DFFF82
:107F6000CFECD2F003E0C3ECD2F001E1DF6ADF50E6
:107F7000006E7EECE1F0640EDF5C03E20101200E96
:107F80001A6F0A0EDF5C03E20101200E1B6FE5523F
:107F9000C2EFC9F016ECCFF0BBECD2F008E19CECDC
:107FA000D0F005E00101D45102E0AC91AC4349C1ED
:107FB00000F07EECE1F0640E0101495D02E2200E6A
:107FC000166F0A0E495D02E2200E176F8F0E006ECB
:107FD000FBEF25F0270E7EECCAF00101500EAC6FCE
:107FE0003B51200B06E19CECD0F003E001011E0E9A
:107FF000AC6F1200EB0E006E83ECCAF002E0EE0EE6
:10800000006EA8EC26F032C100F083ECCAF002E06A
:1080100053C100F00101040E016F7EECE1F001019B
:108020001B8F1200C6ECC9F083ECCAF003E0E9EC48
:10803000CAF003E028C100F008D0FFECD4F003E060
:1080400058C100F002D054C100F0C2EFC9F0CD0E0B
:1080500040ECD2F0010EE66EE5DFE5520FECD5F014
:1080600001011A5D05E12CECD8F002E1200E1B6F36
:108070001200C6ECC9F0BDECCBF0EF50400B03E1B1
:108080002750040B04E001018E51020B6BE0BDECA4
:10809000CBF0EF50200B03E02750040B02E001016E
:1080A000A26BBDECCBF0EF50400B03E12750040B6B
:1080B00059E00101A4510EE0A5510CE1FE0EDB5088
:1080C00005E1A05102E1A15101E0A46BA06BA0C1A8
:1080D000A1F148D05A0EA55D16E16BECCAF0A0C123
:1080E0003EF0EFECD4F0006EFE0EDB5007E10050E6
:1080F00003E10101A15102E00101A56B0101A16BA6
:108100000050A05F2FD0A05102E1A1512BE0A1515E
:10811000496E4A6AA0510A0DF1ECCCF0A5510A0D46
:108120003AECD4F0C1ECCBF0D8C142F0D9C143F065
:10813000E2ECFDF039C0D6F13AC0D7F10101D651D9
:10814000D71110E0D6510E5ED7510F5AFE0EDB50FC
:1081500001E1A56B24ECD2F03CECD6F03DC0A0F1DF
:1081600039C0A1F1C2EFC9F0C6ECC9F079ECD5F085
:10817000E66A7FDFE552E552E0ECCFF0C2EC31F089
:1081800001019E510DE11F0E9F5D0AE29AC29EF110
:108190009BC29FF19CC2A0F19DC2A1F19EC2A2F11F
:1081A00002016F2BC2EFC9F00101DE93D1B3DE8370
:1081B000DE95D1B5DE851200010138A306D0D1933A
:1081C00012B6D183D19512B4D185EEDF04B083DD30
:1081D00081EC9AF081EF2EF00A0E02013F03F3507A
:1081E0004B6E4C6A4051640D58ECD3F03E51010186
:1081F0004924DA6F000E4A20DB6F0A0E006E070179
:10820000BEAB02D0010E006E1FB403D0010106EC1C
:10821000D2F028AA1AD04FECDAF0100ED8804956C6
:10822000270E4A560101DB514A18E8AE02D04A3403
:1082300004D04950DA5D4A50DB591FE20050E9ECA6
:10824000D6F0DA274A50DB2318D000504A6AF00FE4
:10825000496ED80E4A2201014A50DB19E8AE02D01D
:10826000DB3504D0DA51495CDB514A5806E2005054
:10827000E9ECD6F0DA5F4A50DB5B1F84800EDB1539
:1082800003E01F9406ECD2F04FECDAF0DAC13DF0D7
:10829000DBC13EF041ECD3F04AAE04D0396C3A1E5B
:1082A000000E3A2239500101DA5F3A50DB5BE4EC10
:1082B000D4F022ECD9F03DC040F239500101DA6F20
:1082C000DB6B24ECD2F022ECD9F03DC03FF239C098
:1082D0003EF26BEF41F02F8E0480DCEF40F00A019C
:1082E000DA9F71EC0CF0016A0101D4510EE1070133
:1082F000BEBF11D00A0E016EB3ECCDF03E50006E41
:108300000150005C18E2005015D0030ED45D11E15D
:108310000701BEAF02D0160E0DD0030E0A5C02E1BB
:10832000140E08D00A5002E11E0E04D0C5ECD7F09E
:1083300001D0160E016E0150160802E2160E016EF3
:108340001200000CFEDF000903E00101500E486F2F
:108350001200C6ECC9F000AE14D0FF0E0002F3CF3D
:108360006FF26F0EE96E020EEA6EEFCF3EF0FE0E78
:10837000DBCF43F03CECFEF03EC0EFFF02016F6D3F
:1083800009D000C03EF0FE0EDBCF43F03CECFEF027
:108390003EC06FF2C2EFC9F043ECD5F02F50200B76
:1083A00056E12350800B53E13050400B50E12450F4
:1083B000010B4DE11FA618D078ECD2F001012699EF
:1083C00002016F5102E0010126890101269B020191
:1083D0006FAF02D00101268B010126A938D01DAC58
:1083E00036D028EC0CF033D024C100F001012699DE
:1083F000005001E02689269B00BE268B26BB006C20
:1084000060ECCCF016E12E50100B0DE01E50040B6A
:108410000AE11B50080B07E1005002E0FFEC08F0F6
:10842000006A0101246BD7ECD2F006E0450EB95D7D
:1084300003E000380F0B006E005007E00101268DAD
:10844000269F26BB268F246B02D0010126990101AD
:1084500026A902D08CEC04F001012651100B06E095
:108460002B50200B40E01D50400B3DE11F50080BEE
:1084700016E03B51200B13E13BB332D080ECD2F03D
:108480000101279902016F5102E0010127890101D1
:10849000279B02016FAF27D00101278B24D025C174
:1084A00000F02799005001E02789279B00BE278B09
:1084B000279927BB006C32A005D00038E8461F0B77
:1084C000006E04D0D8900032D890003200500AE0FC
:1084D0000701460EA66F0101278D279F27BB278F17
:1084E000256B01D027992B50200B03E01D50400B2A
:1084F00010E001012651100B02E0C5EF46F02751B4
:10850000100B02E0C5EF46F02050200B02E1C5EF52
:1085100046F0D7CADCFAD6CADDFA0601D551D595A0
:10852000010B01E0D585D551D597020B01E0D58728
:10853000D5918650040B01E0D581D5938650020B6E
:1085400001E0D5830F0ED51500ECCCF000A019D0BA
:108550008CEC04F006015051040B0CE03250010B7E
:1085600009E13050040B06E100AE02D0DA0709D071
:10857000DA2B07D000AE03D00101250702D001019C
:10858000252BDAC600F00601D599005001E0D58907
:10859000D59B00BED58BD5A930D0D5BB006C009043
:1085A000004200502AE0DA6B50A527D00101375174
:1085B000010B06E01250080B03E11250040B0FE010
:1085C000288A0601D5BB289A07DE1EAC03D002011B
:1085D000098702D0020106810501478D0ED03BB10B
:1085E0000CD0AAC224F10601D5AB04D0AAC224F152
:1085F0000101246D0101268927840601D651D695F3
:10860000010B01E0D685D651D697020B01E0D68743
:10861000D951D691020B01E0D681D951D693010BE5
:1086200001E0D6830F0ED61500ECCCF000A009D0E7
:1086300080ECD1F000AE03D00601DB0702D00601CA
:10864000DB2BDBC600F0D699005001E0D689D69B23
:1086500000BED68BD6A9CBD0D6BB006C30BC02D026
:1086600000900042005001E1C2D0DB6B010E0D6EA4
:10867000D6BB0D6880ECCBF001E1B0D00BECD5F0AF
:108680009CECCAF003E1E3EC0BF0A8D031BCA6D01F
:1086900030AC0ED0D00EE66E0F0EE66E840EE66E97
:1086A000070E04ECCAF0FFEC04F0F9EC4FF096D0A2
:1086B000D4510BE0030ED45D08E08D51100B3EE069
:1086C000020ED45D02E0D40539E114BC1CD0348420
:1086D000ABEC0FF040ECD6F007E249501408000E66
:1086E0004A5402E2ABEC0FF040ECD6F009E24950FC
:1086F0003D08000E4A5404E2ABEC0FF0ABEC0FF077
:10870000B4EC0FF06BD034842CECD2F008E0C80E3F
:10871000E66E280EE66EB80EE66E030E0AD0DFDDBA
:10872000190E0124E66ED3ECD2F0E66ED70EE66E9B
:108730000A0E04ECCAF00A01030E49D014BC25D07D
:108740003484CDDD0D040BE172ECD3F008E2190E98
:108750000124D75D04E2020ED65FD72B11D0800E24
:108760000D140EE09BEC0FF0FF0F0A01D65D08E23E
:10877000D3ECD2F0D880D75503E2020ED627D70724
:108780000A01010ED46F338825D03484A8DD800E11
:108790000D140CE072ECD3F009E2D3ECD2F0D880E7
:1087A000D75504E2020ED65FD7070FD00D040DE1B6
:1087B0009BEC0FF0FF0F0A01D65D07E2190E0124B2
:1087C000D75D03E2020ED627D72B0A01020ED46F23
:1087D0003388010EE66E51EC1BF0E5521EAC03D05F
:1087E0000201098902D00201068B050147850601B5
:1087F000D751D795010B01E0D785D751D797020BF9
:1088000001E0D787D951D791200B01E0D781D95109
:10881000D793100B01E0D7830F0ED71500ECCCF0E7
:1088200000A009D080ECD1F000AE03D00601DD0736
:1088300002D00601DD2BDDC600F0D799005001E023
:10884000D789D79B00BED78BD7A9C8D1D7BB006C1F
:1088500000900042005001E1C1D1DD6B010E0D6EB0
:10886000D7BB0D681950100B04E12050800B01E1BB
:10887000E6D001018DB595D133B637D020BE04D0F6
:10888000740E006EB3EC26F0FF0E0D5C0CE10201DD
:10889000050ED8800055000E015524E2060E005F3B
:1088A000000E015B1FD071C201F02B50100B0DE1C7
:1088B0000201715137ECCBF008E249509608000EE6
:1088C0004A5403E25A0E015C016E01500B5C0AE24D
:1088D0000201880E005D130E015904E2060E002706
:1088E000000E0123F1EC0BF075D102011D6B960E09
:1088F000016E026A13ECD5F002E0C80E016E2BA8DF
:1089000004D0960E016E0A0E026E0150E66E025001
:10891000E66E480EE66E010E04ECCAF064ECCBF095
:108920000CE1010148510A0808E2010E481505E072
:108930000D0402E1482B01D048072A840901ED6BA0
:10894000EE6BF3EC04F099EC23F07FECD4F0E552FD
:108950000201320E046F48C15BF243ECD2F002E236
:1089600048C18CF1E783E795E79748C102F064ECD2
:10897000CBF004E00101E7935A0E025E0250E66E6E
:10898000F3ECD2F013ECD5F015E02B50100B12E104
:108990000D0404E1650E0101485D07E0800E0D1431
:1089A00009E0640E0101485D05E1318E80ECCBF0F9
:1089B00001E01C9491ECCDF03150800B11E120507E
:1089C000800B0EE180ECCBF00BE100500BE0050ECC
:1089D000005C08E0030E005C03E1020E0A5C02E0AA
:1089E0000D5001D0020E0BECD2F031AE25D0319EED
:1089F000049819A006D004884DEC0BF0050EF1EC9C
:108A0000C9F00101395111E064ECCBF006E0030E2E
:108A1000E66EE40EE66E010E02D086ECD1F05AEC62
:108A2000D7F003E1FA0EF1ECC9F004A802D048EC4B
:108A30000BF00D500BECD2F00201078BCBD00101F3
:108A4000E6AF28D08DB5ADD034C1A8F2FFEC18F058
:108A50001E0EE66E340EE66E010EFFECC9F0A7ECBA
:108A60003FF083ECD4F034C1E6FFF3ECD2F07CECC1
:108A70001DF00201A85103E00101345106E002019A
:108A8000A85105E10101345102E0BAEC17F00201EE
:108A900008859FD02CA425D0E785E793E79783EC42
:108AA000CAF00EE1C80EE66E320EE66E010EFFEC65
:108AB000C9F032C1E6FFF3ECD2F053EC64F00ED013
:108AC000C80E57ECDBF0530EE66E010E04ECCAF054
:108AD00053C1E6FFF3ECD2F0EAEC18F0FAEC3FF009
:108AE00079D024A034D0D45111E1460EE66E280E80
:108AF000E66E290EE66E010E04ECCAF00101295162
:108B0000E8240301B86FF7ECCEF015D08DECCDF072
:108B100007E0E66A2E0EE66E010EFFECC9F00DD0FE
:108B20009CECCAF00AE1330E57ECDBF0870EE66EE0
:108B3000020E04ECCAF0FFEC04F02EEC4FF052EC05
:108B4000CCF0BAEC17F005014785478F43D083EC92
:108B5000CAF006E0E9ECCAF003E12750020B1CE082
:108B6000320E006E0050E66E080EE66E490EE66E9E
:108B7000010E04ECCAF0CAEC3FF00101E793E7955F
:108B8000E78749C1E6FFF3ECD2F049C113F5F0ECF9
:108B900064F0020106871ED091ECCDF001018DA595
:108BA00003D0F8EC08F016D0FFEC18F0500EE66E8B
:108BB000350EE66E010EFFECC9F05AEC15F0E8EC4C
:108BC0003EF083ECD4F035C1E6FFF3ECD2F00201C5
:108BD00008832A842D8E02011E0E206F0601D851B3
:108BE000D895010B01E0D885D851D897020B01E048
:108BF000D887D951D891800B01E0D881D951D89329
:108C0000400B01E0D8830F0ED81500ECCCF000A08B
:108C100009D080ECD1F000AE03D00601DC0702D011
:108C20000601DC2BDCC600F0D899005001E0D889A1
:108C3000D89B00BED88BD8A9A8D0D8BB006C009018
:108C40000042005001E1A1D0DC6B010E0D6ED8BBDB
:108C50000D682CA631D083ECCAF003E0E9ECCAF031
:108C60000AE0320EE66E280EE66E010EFFECC9F049
:108C700086ECCCF01ED0CFECD2F00BE11E0EE66EEF
:108C8000580EE66E010EE66E20EC7AF0E552E552E3
:108C90000DD01E0EE66E540EE66E010EFFECC9F00E
:108CA00083ECD4F054C1E6FF4FEC0AF0E55209EC36
:108CB00019F027EC40F065D023AE23D021B661D067
:108CC000016A0101D45102E0010E016E55ECD6F0AB
:108CD0000AE1E2ECD6F004E6E20E495C000E4A58E6
:108CE00002E2190E0026FF0E0D5C05E10050180887
:108CF00002E2190E005E015066ECCAF000C0EFFF00
:108D00000BD02FAA0DD021B63CD00E0EE66E930EDE
:108D1000E66E020EFFECC9F0FFEC04F0238A31D0BE
:108D200021B00ED021B62DD03C0EE66E660EE66E5A
:108D3000010EFFECC9F007EC53F025EC05F021D053
:108D400021B61FD09CECCAF00CE1280EE66E680E2E
:108D5000E66E010EFFECC9F055EC0CF063EC05F08B
:108D600010D0800E0D1404E03C0E675D01E2672B0D
:108D70000D0403E1675101E0670728EC53F03FEC75
:108D800005F02D8E02011E0E206F1DAC66D007016E
:108D9000BE8388EC09F001013B91129C3B51010B11
:108DA00001E0128CE66ADAEC2BF0E552006E00501E
:108DB0000F0802E20F0E006E100E0002F3CF0EF24B
:108DC00045EC27F01D9A050E0701A1250201D88068
:108DD0000E5501E21D8A2A50800B13E10D5111E05E
:108DE000050E0701A15D02010E5D03E2E7EC08F04C
:108DF0001D881D50100B31E01D50200B2EE002018C
:108E000009D02A50800B0AE11D50800B07E11D504C
:108E1000200B04E0FA0E0D6F1D981FD02ABE02D061
:108E2000E4EC08F02BBA17D01E0EE66E050E7CECB3
:108E3000D0F0E66E3CECCDF00AE019C5C4F11AC5DD
:108E4000C5F11BC5C6F11CC5C7F11DC5C8F1AAC235
:108E500024F10101269B010126891D50800B0DE1A3
:108E600001012651100B01E17ED01F50080B01E1DA
:108E70007AD02050200B01E176D002011E0E206F27
:108E80001DAC02D0140E206F2BAA2FD01DBC16D003
:108E900001014451630801E2446B800E241506E091
:108EA000FB0E245D03E2246B000E12D0800E24150D
:108EB00059E12451030856E2246B09D00101246BC7
:108EC0002AAE09D0050116514DE1320E166F010E82
:108ED00079ECD3F047D0AD51030844E3010E79ECAF
:108EE000D3F00101140EAD6F3DD01E50400B03E0D6
:108EF0000951010B37E11EAC02D0098101D0068374
:108F0000050147812B8C2C8AF4ECCAF0D4C1E6FF12
:108F1000A2EC3EF0E55278ECD2F01D50800B06E05A
:108F20000101245103E19EEC31F016D002016FAF34
:108F30000AD0BEC7E6FFB4EC40F0E5520201AA51E8
:108F40000101242709D06F5107E0BEC7E6FFEBEC13
:108F5000CFF0AA510101245F02016F51DCE12D82A3
:108F60007CEC04F01D9E01012751100B4BE01F50BB
:108F7000080B48E02050200B45E002011E0E206F38
:108F80001DAC02D0140E206F1EAC02D0098301D09C
:108F90000683050147832B8CD5C1DFFF2C9ABAECE1
:108FA000CCF0DFCFE6FFA2EC3EF0E55280ECD2F051
:108FB00002016FAF0DD0DF502CECCBF0EF50E66E1E
:108FC000B4EC40F0E5520201AB51010125270CD071
:108FD0006F510AE0DF502CECCBF0EF50E66EEBEC7B
:108FE000CFF0AB510101255F02016F51DFE12D820E
:108FF000D0ECCCF024A606D00101010EAC6F070125
:10900000140E556F2BAC06D067ECD4F02B9C258248
:109010002CAA238A0101279926992794E552C2EFA9
:10902000C9F03B0EDFECCAF00101320EAC6F2F88A5
:1090300033C119F21200010137A70AD04D0E096E93
:109040000F0EE66E100E0D03F35010ECD2F010D0A0
:10905000030E096E0F0EE66E140E10ECD2F034EC17
:10906000CAF0030EE66E230EE66E230EE66E0A0EBF
:1090700034ECCAF0096A1200C6ECC9F0030E096E9E
:10908000140EE66E000EE66E0A0E93ECD9F0040E96
:10909000E66E260EE66E0A0EE66E260E64ECD6F03E
:1090A000FE0EDB501EE0010137A70AD04D0E096EFF
:1090B0000F0E10ECD2F0E66E100E0D03F3500ED032
:1090C0000F0E10ECD2F0E66E140E64ECD6F0030E28
:1090D000E66E230EE66E0A0EE66E230EE66E2FECAB
:1090E000CAF0096AC2EFC9F0030E096EAA0EE66E55
:1090F0002A0EE66E0A0EE66E300E36EFDBF053EF08
:10910000DAF0E4ECD5F003E10201D8511CE00101F2
:1091100075ECD4F001E0098FBBECDAF00601EE6BE0
:109120003FEC32F007010B999BECC4F08BEC20F084
:109130000701149F5BECD5F00701158162ECD5F0B7
:1091400078EC16F02D860201D96BD9C2D8F2120044
:10915000010121A15EEF4DF0219102010F070F5196
:1091600001E01AD1640E0F6F9CECCAF016E120509A
:10917000400B13E1080E76ECCBF0046E04AC0DD07E
:109180000101E5BF02D0E58F02D0E5BFE59FE66AA9
:1091900065EC39F0E55220EC32F002013D510CE073
:1091A0003D51010803E380ECCBF006E002013D07EE
:1091B0003D5102E156EC25F03196150E0101555D49
:1091C0000BE002011651171103E01607000E175BA2
:1091D0001651171101E12F8C0201145101E01407FF
:1091E00001018B5104E08B078B5101E131960201A3
:1091F00020510CE01F50080B09E02007205106E128
:109200001DAC02D01D8E02D02DBE2D9E300E04014D
:10921000F75D06E10201066B076B086B096B05D071
:10922000340EF75D02E281ECA1F0020119511BE05E
:109230000501105118E12750400B15E138ECD2F030
:1092400012E1190719510FE10C50006E555106E05B
:109250007F0E5515006E189A55BF188A010EE66EDE
:1092600000505BECD2F00201580758510BE10101AC
:10927000515102010B5D06E2410EDFECCAF0010123
:10928000AC69258E80ECCBF008E00101835105E04C
:10929000765103E14AECE3F002D016ECE4F028EC5E
:1092A000D2F008E060ECCCF005E117ECD5F002E17B
:1092B00006011D79E7ECD2F011E01B50100B0EE116
:1092C0002150020B09E0050ED45D06E0040ED45DCA
:1092D00003E01E50200B02E1060104790101385120
:1092E000100B06E11350020B05E01950200B02E1B0
:1092F00006010D752850400B01E0010E020F016EB2
:109300002850400B01E0010E050F026E03681DACF2
:1093100008D056ECD8F0EF7E56ECD8F0EF50800B2A
:10932000036E010183512BE0BBECE3F0000903E184
:109330002E50200B24E02E9A71EC16F0016A030ED9
:10934000015C12E2026A040E025C08E2020EA4EC66
:10935000D6F0320EF1ECC9F0022AF5D7E66895ECAA
:1093600021F0E552012AEBD778EC16F001015F9964
:109370002582DFEC78F0A5ECE3F04AECE3F00201A3
:109380002D5101E02D077A5104E02250100B01E12C
:109390007A07325101E03207D35109E0D307D351A4
:1093A00006E1D45102E1010ED46F41ECC2F01EACD3
:1093B00009D00201D107D15105E181ECA1F00201F0
:1093C000030ED16F38ECD2F040E02050400B3DE06E
:1093D0001950400B3AE0AFECD0F003E11950200BEC
:1093E00034E002013707000E385B1950200B0AE009
:1093F000EEECD0F009E11EECCDF004E10101E45106
:10940000100B02E1000E01D0010E0490E8B00480C0
:1094100038ECD2F003E00450010B17E0376B386BE7
:109420000101E49904A006D00201196B19C255F29A
:109430004DEC65F017EC0BF00101B5A705D02492B7
:1094400023BC2482DAECD0F0209402013C5101E0EC
:109450003C07335101E03307315101E0310730510E
:109460000AE03007305107E11FECCEF001E14A502D
:1094700002E00EEC0DF00201185109E01807185136
:1094800006E109ECCFF00201D05101E1119410077F
:1094900010513FE1280E106F1AAC0FD0BAEC38F023
:1094A000D4C100F0EEEC38F00601017901A931D009
:1094B000D5C100F0EEEC38F02CD01BA803D006018B
:1094C000047927D01CA206D00101E6B522D00601FE
:1094D00014711FD01950200B06E001013851100BF8
:1094E00002E106010D752450020B03E1BFECD2F03E
:1094F00010E0020130510DE11FECCEF001E14A50C5
:1095000008E02C50800B05E12C50400B02E10601D5
:10951000017102012B5101E02B070701A65105E063
:10952000A607A65102E1DBECD1F002012A5116E0B8
:109530002A072A5113E183ECCAF003E175ECE2F04B
:109540000DD00701A351A41109E0A35101E0A30725
:10955000A45101E0A4070201020E2A6F0201295161
:109560000CE02907295109E1178E17901788080E7A
:10957000156E2CAC02D0290E156E0101AE5169E0BA
:10958000AE07AE5166E122ECD1F0006E0201A951A6
:1095900007E0830E096EA9C201F037EC3BF0096ABF
:1095A000FF0E0201845D28E084C24FF0506A516AC8
:1095B000C70E496ED80E4A6E010E4B6EB9C14CF003
:1095C0004D6A4E6A2FECD5F00900F5504F24F36E2A
:1095D0000900F5505020F46E0900F550512036EC8A
:1095E000D6F00800F550006E0201842B005004E113
:1095F0008469010128ECD9F0005013E00101190E33
:10960000AE6F0050E66ECEEC6FF0E5520201A9514C
:1096100002E0A92B1ED00101B22B000EB323B4230C
:1096200018D02850080B03E13050080B04E02896AE
:109630000101E8970ED00201A95105E0A96B0101D3
:10964000FA0EAC6F05D00101D890AC33D890AC3392
:10965000E8970201285104E02807285101E1259EDE
:10966000275107E02707275104E10601416941C658
:1096700040F60101AA510DE0AA07AA510AE1090E1C
:10968000155C07E160ECCCF004E10101FA0EAB6F70
:109690001A8A0101AB5101E0AB070701555101E006
:1096A000550702012F5123E02F072F5120E1000E13
:1096B0000601E76EBE19E8AE02D0BE3503D0E75012
:1096C000D880BE5502E2BE0701D0BE2B000EE76E69
:1096D000BF19E8AE02D0BF3503D0E750D880BF55E0
:1096E00002E2BF0701D0BF2B0201050E2F6F1551FB
:1096F00005E01507155102E1DDEC69F00201215189
:1097000024E0210727AA21D020BC1AD01A50800BB0
:1097100017E0800E071414E02050010B11E1216BBB
:109720001A9E0A01DA8F71EC0CF00BEC75F01EAC8E
:1097300003D00201098902D00201068B0501478589
:109740000201215102E1238A25820D5107E01D50BB
:10975000400B04E00D070D5101E11D8E050116516E
:1097600001E016070201355105E03507355102E1E8
:10977000D0EC0AF00201B05101E0B007D0510DE089
:10978000D007D0510AE107010A839DECC4F028EC10
:1097900053F00201185101E111942C5101E02C0702
:1097A0000101AC5101E1A3D0AC07AC5101E09FD065
:1097B000B59DB59F2F98E4951C921B9830AC02D0B4
:1097C00018EC50F02FBA07DB23BE98DA24B05CDB2C
:1097D0002582238A279820BA02D0F5EC26F0208A29
:1097E0000C0E155C29E12150200B26E00101AA5145
:1097F00023E1156860ECCCF002E11E8417D0010172
:109800003B71129C3B51010B01E0128C4AEC99F028
:10981000540E7EECCAF001013BA108D04B0EE66E5F
:10982000CC0EE66E30EC0AF0E55204D0550EE66E32
:10983000D5EC26F0E5521A861D50400B11E02A5057
:10984000800B0EE12150200B0BE02A8E130E98ECBA
:10985000CEF0460EE66E410E8CECD1F0E7EC08F04F
:109860000101E8A909D0E899E887330EE66ED40E25
:10987000E66E010ED1ECCDF02550040B38E00B0E56
:10988000155C35E12150200B32E00101AA512FE196
:1098900020982594B59BB599E67DE6AD1AD0E8A34E
:1098A0000AD0F50EE66EE30EE66E010EF6ECC9F098
:1098B0000101198F09D0420EE66ED40EE66E010E3C
:1098C000D1ECCDF00101E887E883500EE66EC60EBC
:1098D0000CD0ED0EE66EE30EE66E010EF6ECC9F06E
:1098E0000101198F500EE66E4E0E57ECCAF00201C0
:1098F0001D5101E01D07045101E004071E5101E064
:109900001E071F5101E01F07345101E03407010118
:10991000AD5101E0AD070201235101E023073951A8
:1099200001E03907D85108E0D807D85105E181ECAA
:1099300048F002010E0ED96FD95101E0D9073A5112
:109940001CE02150200B0AE1110E11ECD6F03AC2B6
:109950003EF0EFECD4F002E10601067B02013A078B
:109960002150200B05E02050400B02E08FEC05F069
:1099700002013A5102E1B5EC04F0060143510AE05C
:109980004307435102E15A0E436F25860F0E435D94
:1099900001E225960201225108E02207225102E14C
:1099A00073EC69F002011E0E216F3B5110E00101C2
:1099B0002651400B0CE102013B073B5108E144C139
:1099C00000F01886A6EC96F00201010E246F020149
:1099D000245141E0240724513EE10101395103E0C3
:1099E0000901010EEB6F0901ED6B0BECD5F00101E4
:1099F000E78F5EECC5F00201186BD05101E11194C4
:109A000009ECCFF020A204D0209281EC2EF014D0EB
:109A100088ECD4F078EC16F0640EF1ECC9F04AEC66
:109A2000E3F0EAECD0F008E02050200B05E0010E56
:109A3000E66EDFEC99F0E55218B002D02FECD9F0C9
:109A40001890020106891EAC02D00987098505011C
:109A5000BF0E476F48810201365104E03607365188
:109A600001E12582255101E02507D25109E00501D8
:109A7000105106E10201D207D25102E15CEC0AF07A
:109A800002011B5106E01B071B5103E1630E2CEC86
:109A9000CAF002011C5106E01C071C5103E1B10E83
:109AA0002CECCAF002011A5105E01A071A0502E16E
:109AB000F1EC0FF002012E5101E02E071200060119
:109AC0004F6B4FC64EF64FC64DF64FC64CF64FC6BF
:109AD0004BF6120047ECD5F0DE52010EDD6EFE0EA5
:109AE000DB501AE1FCECD8F0050EE66E200EDF2408
:109AF000E66E4B0EE66E060E34ECCAF0050ED5ECA3
:109B0000DAF0BA0EE66E010E34ECCAF00F0E4FEC2E
:109B1000D8F00050DF6E096A0101BA51630805E30D
:109B2000BA5110E11F0EBB5D0DE2360E006E9DECCA
:109B300026F0FE0EDB5001E1C2DF010EDB6A81EC94
:109B40002EF022D0FE0EDB501FE12C50800B07E0E0
:109B5000DF500A0804E20701BE9B88EC09F0DFCF62
:109B6000E6FF21EC34F0E55201018A51100B0CE0C4
:109B70000A0E445D09E26CECDBF059ECD8F0DFCF63
:109B8000E6FF4FEC80F0E5520201295115E1640E29
:109B90000101445D0BE26BECCAF044C13EF092EC73
:109BA000CCF00101166F300E3A2405D04D0E166F21
:109BB000030E4415310F176F016A050E015C2EE28A
:109BC000630E496EDB0E4A6E010E4B6E0150EA6A5F
:109BD0004B0FE96E060EEA22EFCF4CF031ECDBF0D2
:109BE000026E2D0E025C05E10101B65102E1200E6C
:109BF000026E0201295110E1020E012468ECCBF043
:109C000002C0EFFF015008E12B9A2A0E025C04E12A
:109C10002C50800B01E02B8A012ACFD70201295159
:109C200002E10101188F010EDB50DBECD2F002E201
:109C3000E16AE552E16E4950C2EFC9F04EECD4F052
:109C4000016E44510AECCCF0050EE66E4B0EE66E4A
:109C5000060EE66E200E012436EFDBF00201050E43
:109C6000B86FF00EB96FFA0EBA6F140EBB6FF00E2C
:109C7000BC6FFA0EBD6F1200016A0101D45102E0FF
:109C8000010E016E0150F8ECD5F0EF50006ED2AD30
:109C9000006A015066ECCAF0EF50E66E0150F8EC35
:109CA000D5F0010ECDECDAF0E66E0050E66E250E32
:109CB00028ECCCF001011496D251400B01E014863F
:109CC0001200026A0101D45102E0010E026E02503C
:109CD00066ECCAF0EFCF49F0190EC0ECCAF07CEC8C
:109CE000CEF002E1200E1B6F4E0E186F520E196F50
:109CF0003CEF4EF0238E1F9661EF4EF0239E2BEF2C
:109D0000D1F0020EE66EBD0E0AECCAF00101D0BB26
:109D10000FD0BB0E2CECCAF0010EE66E200EE66EE4
:109D2000E66A2F0EE66E3BEC16F03DECDAF03AD028
:109D3000070E0201935D18E29351E824496E4A6AC6
:109D4000FF0EBFECD7F0E66E060ED8809355070DD8
:109D5000F3500A0FE66EBC0EECECC9F0010EE66E95
:109D6000200EE66EE66A17D0F30EE66E0A0EE66E79
:109D7000BC0EECECC9F0020193510A0802E2030E9A
:109D800001D0010EE66E0F0ED88093550C0DF350E6
:109D9000E66E800EE66E2F0E28ECCCF0B90EE66E65
:109DA000FCEC15F0E55201011494D051200B01E0B8
:109DB00014841200020193297CECCEF002E1200E03
:109DC0001B6F4E0E186F420E196F81EF4EF02F8AE7
:109DD0001F96DAEF4EF02F9A2BEFD1F07CECDBF0F0
:109DE0009CECCAF017E1020E016F02018729F0EC2A
:109DF000D3F014ECD8F0030EE66E020EE66E48ECDB
:109E000009F0E552E55201011C8F500E166F4C0E01
:109E1000176F1200030ED45D10E18DECCDF006E05B
:109E2000E50EE66EE30EE66E010E05D0DD0EE66E83
:109E3000E30EE66E010E72EFD7F0016B29C100F060
:109E40000FECD5F00101165D02E1200E166F300E09
:109E5000196F480E1B6F5A0E1C6F12002450010B15
:109E600009E19CECCAF006E071EC16F0030E006EFE
:109E70003DEC75F024809CECCAF003E00068A8EC8F
:109E800026F01F96EEEF4EF09CECCAF005E11DECBB
:109E900009F01CEC1FF004D0D0EC0AF078EC16F0BE
:109EA00024901A940101AC6BB59F2398CEEC0CF072
:109EB000FAEF0DF06CECDBF00A5018E01F0E006EAC
:109EC000010196BB02D03F0E006E030E0A5C02E059
:109ED0002D0E006E61ECE1F001010E5102E1100E59
:109EE0000E6F002B8B0E006EE6EC25F07CECDBF0A9
:109EF000F20E496ECD0E4A6E010E4B6E0A50F3EC17
:109F0000DAF017C1E6FF16C1E6FF18EC0AF0E552D9
:109F1000E552010136AD02D06EECDFF01200328066
:109F200000689DEC26F0E8ECD4F01F96C3DF55EFF7
:109F300039F03290CEEC0CF001DA2F98120069EC77
:109F4000D5F0140D97ECCAF0FBECD4F005E0E5EC8D
:109F5000CBF0230EECECC9F00EEC15F0140EF1EC86
:109F6000C9F0C2EFC9F0C6ECC9F0B6C200F0FE0EEF
:109F7000DB5001E1006AB7C2E6FF0050E66E240E36
:109F8000ECECC9F0C2EFC9F007018B51845D15E11B
:109F90001450100B01E0010E496E3350010B495C67
:109FA0000CE11450200B01E0010E4A6E3350020BFD
:109FB00001E0010E4A5C01E1120084C78BF7339087
:109FC00014B83380339214BA338214A80BD014AA75
:109FD00003D084C7E6FF07D0E66AB1DFE552010E81
:109FE000E66E04D0E66AABDFE552E66ABCDFE55216
:109FF000120007018451140D14ECD8F019C116F1A8
:10A000001AC117F11BC118F11CC119F10101200E71
:10A010001A6F480E1B6F5A0E1C6F300E165D02E150
:10A02000200E166FC4EF4FF0308C1F96F9EF4FF0F3
:10A03000309C2F980101AC6B2398B59FCEEF0CF0AC
:10A040000101AC5103E02450080B03E0B551200B93
:10A0500001E02F88005011ECCDF00101AC5106E079
:10A060002F50100B03E1FA0EAC6F24861200010E84
:10A070000701D89056375737E806FBE121AC02D0EC
:10A08000070156810D0E0701585D01E2582B1200A1
:10A09000219C8450020B01E0218C07014E5111E1FB
:10A0A00021AC78D04E2B010E566F576B586F3098FD
:10A0B000596F5151FE0BE8425125506F0101219318
:10A0C0001200010121A366D0219307014E0562E130
:10A0D00021BC52D030A84DD00C0E585D47E2D8902C
:10A0E00057335633006A5F0E005C1BE20C0E4B6E5A
:10A0F000CD0E4C6E010E4D6E00504E6ECEECCBF080
:10A10000565149180CE157514A1809E1200E002612
:10A11000610E005C02E3200E005E92DF02D0002A96
:10A12000E2D75F0E005C22E107011F0E561901E124
:10A1300057510AE01D0E561901E1575105E0EF0E87
:10A14000561905E1575103E1200E006E79DFFF0E2D
:10A150000701561902E1020E571906E0B50E56190D
:10A1600005E1030E571902E18BEC6FF007014E6B0E
:10A170001200308837EF50F07ADF30A804D00701A2
:10A18000010E596F06D00701592B59510C0801E2F5
:10A190004E6B3098120007AE06D08450020B02E0DE
:10A1A000219C01D0218C07014E5110E121BC75D0BA
:10A1B0000101219307014F6B07AE6FD0020E4E27AE
:10A1C0005151FE0BE8425125506F12004E050BE134
:10A1D0004E2B51C750F70101219321AC5ED00701EE
:10A1E000080E4E6F1200010121A357D02193070ED4
:10A1F00007014E5D46E14E6B21AC40D00101AC51F0
:10A2000003E02450080B03E0B551200B01E02F8838
:10A21000EB0E496EDA0E4A6E010E4B6E07014F517E
:10A22000522554ECD5F0006E810E005C02E1526BB9
:10A230001BD0800E005C03E1200E526F15D00D0E76
:10A24000005C03E00A0E005C02E1200E0BD00B0E56
:10A25000005C02E12A0E06D00A0E005C05E0005008
:10A2600003E0005011ECCDF00101AC5109E02F509A
:10A27000100B06E1FA0EAC6F24861200080E4E6F2A
:10A280001200080E4E5D04E121AC07D04E6B1200A7
:10A290004F914F4321BC4F894E2B12007CECDBF0D9
:10A2A00019ECCCF013E103ECD5F006E0D60E496EC4
:10A2B000E30E4A6E010E05D0620E496EF20E4A6E32
:10A2C000010EDAECD7F05DECCAF018D0EAC600F067
:10A2D0000050020802E2020E006ECA0E496ECD0E58
:10A2E0004A6E010E4B6E0050F3ECDAF00601EA51B3
:10A2F000020804E2EA05300F01011C6F8FEC1FF029
:10A3000083EC0FF0006E00500A01D65D04E200C03D
:10A31000D6FA52ECCCF012000101D45105E13084A0
:10A32000E8ECD4F01F9603D00068BFEC26F04EEFA7
:10A3300051F03094CEEC0CF09EEF51F0040EE66E2E
:10A34000EA0EE66E060EE66EA00E64ECD6F0140E73
:10A35000016E3CC100F0F9EF3AF043ECD5F0E0C6F5
:10A3600049F0E1C64AF0D89049364A3606018CECED
:10A37000D4F00CE3DEC64BF0DFC64CF0D8904B3681
:10A380004C36E0514B5CE1514C5820E2DE51E02567
:10A390000E6EDF51E1210F6E34ECD2F0E2C649F0CF
:10A3A000E3C64AF0030E5BECD0F0FDE14950060134
:10A3B000E25F4A50E35B0CECD6F0030E5BECD0F0AE
:10A3C000FDE149500601E2274A50E323DEC6E0F6EC
:10A3D000DFC6E1F692ECD1F049364A36D8904936DC
:10A3E0004A368CECD4F00BE392ECD1F04A3249328D
:10A3F00009ECDAF04950DE5D4A50DF5902E2DF6ACB
:10A4000009D0E251DE5DE351DF5902E2010E01D0D5
:10A41000020EDF6E92ECD1F049364A364950E22501
:10A42000E46F4A50E321E56FDF50E552C2EFC9F017
:10A430001DBC1200219C8450020B01E0218C21AC38
:10A4400003D002016C2B02D002016D2B1F9E06016E
:10A45000E65109E121AC4BD0010EE66FDE6BDF6BFC
:10A46000E76BE86B44D0E60515E121BC40D0020E55
:10A47000E66F73DF006E00500BE0070E0601E85D2B
:10A4800007E2E82BE791E7430050010801E2E78F7C
:10A4900006011FD0020EE65D2AE121AC1DD0E2C606
:10A4A0004BF0E3C64CF0030E0F0B05E0D8904C3296
:10A4B0004B32E806FBE106014B50E25D496E4C5021
:10A4C000E3594A6E4950DE5D4A50DF590EE2010EF3
:10A4D000E66FDE6BDF6B0BD0E451E425496EE5518E
:10A4E000E5214A6E8CECD4F002E2030EE66F030E17
:10A4F000E65D43E1E791E743E78F070ED880E85533
:10A50000016E01500106000903E0E791E743F9D726
:10A51000780EE75D30E20101AC5103E02450080BF6
:10A5200003E0B551200B01E02F88E7C6E6FF3CECC5
:10A5300004F0E552006E200E005C03E300506E084C
:10A5400002E22A0E0BD0298A005011ECCDF0060150
:10A55000DE51E45DDF51E55903E2200E11ECCDF050
:10A56000299A0101AC5107E02F50100B04E1248619
:10A57000FA0EAC6F30860601E66B1F8E12000101E9
:10A58000E583D45102E154DF07D01F9EA4ECD0F044
:10A5900002E07EDD01D0FFDD0101E5931200800EB7
:10A5A000071420E02A50020B1DE12050200B1AE076
:10A5B0000201A95117E10101D45104E10601EA5158
:10A5C000010806E319ECCCF00DE103ECD5F00AE04C
:10A5D0002A0E0101B51506E10C0E155C10E12150A3
:10A5E000200B0DE0800E071409E1E9ECCAF006E04B
:10A5F0000601EC5103E002012D5101E0000C010CB9
:10A600000201395103E1120E7EECCAF0120043EC54
:10A61000D5F066C1DFFF01016651140804E26651FE
:10A62000E824EC0FDF6E21A204D06651CFECD8F005
:10A63000DF5E1EBCDF6ADFCFE6FF720E0AECCAF0F7
:10A6400030800201078334B0DBDFE552C2EFC9F08E
:10A6500043ECD5F067C1DFFF9CECCAF002E1DF6A92
:10A6600005D007010AB302D00F0EDF5EDFCFE6FF91
:10A67000710E0AECCAF002010787E552C2EFC9F079
:10A6800047ECD5F0D00EDE6E070EDD6E01014851AD
:10A69000320804E28C0EDE6E0A0EDD6EE6A510D0E6
:10A6A000D00EDE6E070EDD6E44EC20F0010804E0F3
:10A6B00044EC20F0020820E1340EDE6E080E1BD0C0
:10A6C000090E2B5D0DE25F51020B0AE02250100BC8
:10A6D00007E13450800B04E102010B517D080CE2CC
:10A6E000B80EDE6E0B0EDD6E01014851780804E2F3
:10A6F000800EDE6E0C0EDD6E3BECCBF002E3000E46
:10A7000001D0010EDBECD2F002E2E16AE552E16E2B
:10A710004950C2EFC9F047ECD5F0F8EC10F0A8ECC6
:10A7200048F09CECD0F002E02ADF02D01FBE1F9E52
:10A730002450200B06E00201245103E1D5ECC4F0C3
:10A74000249A02012B5102E0A3EC3DF00101B75124
:10A7500011E1E66ADAEC2BF0E552006E1DAC8EEFEB
:10A760005AF00701A151F00BE83AA15D0024A16F56
:10A770008EEF5AF0B7050DE11BEC71F045EC27F0B8
:10A780003CEC18F01E92E8A08EEF5AF01E828EEF7D
:10A790005AF0020EB75D04E1A2ECDBF08EEF5AF046
:10A7A000030EB75D07E12EB48EEF5AF0D0ECE0F067
:10A7B0008EEF5AF0040EB75D01E0B4D002012551CE
:10A7C00002E08EEF5AF01750100B06E11750010B04
:10A7D00003E11750200B02E0000E01D0010E229081
:10A7E000E8B0228021AA45D07AECD1F0166E22A0E2
:10A7F00036D00101AA512AE1090E155C17E160EC7F
:10A80000CCF014E10101AB510BE1A00E176EA3ECEB
:10A8100009F000093CE0EAECD0F039E11A8637D0C3
:10A82000165035E1AB6B900E176E1FD0165002E13B
:10A83000010E01D0100E8009176EA3EC09F000097B
:10A8400026E0EAECD0F023E11A8421D016501FE173
:10A85000AB6BABC1AAF1810E176E219A06D01650D0
:10A8600016E12250010B13E1219A0201020E256F1D
:10A870000ED031B40CD0E66ADEEC3DF0E5520009B2
:10A8800006E031840201020E256F07AE256B3150C0
:10A89000040B02E18EEF5AF00201255102E08EEF27
:10A8A0005AF031947AECD1F0166E165002E18EEF28
:10A8B0005AF08CEC04F00201A96B0101280EAA6F7A
:10A8C000150E165C05E12050400B02E01E0EAA6F2B
:10A8D000080E165C06E0290E165C03E0100E165CEE
:10A8E00002E12D0EAA6F0201020E256F218A176A5E
:10A8F0001650156EA3EC09F000090BE0010136516A
:10A90000800B07E00201355104E1040E006E3DECBE
:10A9100075F028B602D00101AE6B7BEC0CF02A84F6
:10A920008EEF5AF0050EB75D21E180ECCBF00FE021
:10A930001B50080B0CE187ECCEF009E287ECCEF05F
:10A9400006E202011E0E186F09ECCFF0118401011E
:10A950002651100B02E08EEF5AF02751100B02E047
:10A960008EEF5AF0A3EC3DF08EEF5AF0060EB75D75
:10A9700007E120AA8EEF5AF0E2EC07F08EEF5AF0D2
:10A98000070EB75D5FE11F50080B59E080ECCBF07C
:10A9900056E0FFECD4F053E1AFECD0F050E156A517
:10A9A0004ED0D70E1BECCDF02ABC30D0E2ECD6F066
:10A9B00004E68F0E495C000E4A5802E38EEF5AF00F
:10A9C0001E0E036E27A002D0010E036E0350F1ECA1
:10A9D000C9F0D70EF5ECD9F0016E050EF1ECC9F017
:10A9E000D70E1BECCDF0040E4EECCEF00050E66E10
:10A9F000E9ECCDF002E18EEF5AF02A8C3FEC0CF03E
:10AA000027900201080E336F8EEF5AF0CCECD8F08D
:10AA100004E249508F08000E4A5405E30201335105
:10AA200002E08EEF5AF02A9C0201335103E12780A5
:10AA30008EEF5AF0190EF1ECC9F08EEF5AF02A9C05
:10AA40008EEF5AF0080EB75D01E089D32550800BD8
:10AA50000AE00201285107E1020EA4ECD6F002013F
:10AA60001E0E286F259E25AC03D0F7ECCEF0259C5A
:10AA700025AA03D0D0EC0AF0259A01013651800BAB
:10AA80001BE00201355118E11AA404D0040EA4EC15
:10AA9000D6F01A941AA604D0070EA4ECD6F01A9693
:10AAA0001AA804D0060EA4ECD6F01A981AAA04D05C
:10AAB000050EA4ECD6F01A9A0101B5BDA7D0B5A930
:10AAC00067D020AE0FD0AD5101E07BD02BA805D0D0
:10AAD0000B50E66EFEEC3EF003D0E66AC2ECBDF031
:10AAE000E5526FD024A003D02EEC4FF06AD032A0F4
:10AAF00012D026AD0DD0A4ECD0F002E00101967B7F
:10AB00007BEC0CF01CEC1FF08FEC1FF05AEC4FF0BC
:10AB10000101269D34D02C50400B03E12C50800BBA
:10AB200030E026AD4ED0D8EC08F00101B6511AE164
:10AB3000630EE66E440EE66E010EF8ECCCF044C1F6
:10AB40000CF202013B6B86ECD0F0000917E02C50B0
:10AB5000800B14E001018E51100B10E10201100E68
:10AB60003B6F0CD0290EE66EB6054A6A4B0F496E54
:10AB7000060E86ECD7F091ECD4F0E5520101AD6BF6
:10AB800020D021B61ED059C200F09DEC26F019D07D
:10AB9000B5A305D025A215D02592228212D0B5A149
:10ABA00010D025A206D025922BC1E6FF21EC34F06F
:10ABB000E5520201215105E11A50400B02E155EC2A
:10ABC00039F0A4EC14F0006EFF0820E0570E005C92
:10ABD00007E16CECDBF0220E006E9DEC26F016D047
:10ABE0001B0E005C03E174ECC3F010D0FF0E015C9F
:10ABF0000DE06CECDBF00101140E116F0D0E126F05
:10AC0000050E006F0150006E61ECE1F00101B5BF6F
:10AC10008ED2B5ABF6D02CA603D027EC40F071D283
:10AC200030AC03D0F9EC4FF06CD22FAA05D023AA98
:10AC300068D2DAEC4EF006D023AE06D023AA61D259
:10AC400061EC4EF0239AA8D024A003D0EEEC4EF095
:10AC500058D22CA403D0FAEC3FF053D2E6AF03D085
:10AC6000A7EC3FF04ED219A803D07FECD4F0B1D0BE
:10AC70003050040B1BE0D45119E127AD0DD0010E6B
:10AC80000D6E27BF0D680A0EE66EEA0EE66E060E22
:10AC9000FFECC9F052ECCCF02350200B04E1010191
:10ACA0002751400B3FE04EEC51F03CD032A03ED05B
:10ACB00027AD16D0010E0D6E27BF0D680AC006F134
:10ACC000030EC9ECD5F0F8ECCCF006C10AF050EC5C
:10ACD000D7F00A5080ECD6F09EEC51F00501478584
:10ACE0002350200B03E0EAECD0F004E001012751EF
:10ACF000400B18E07BEC0CF035ECD9F05AEC4FF03F
:10AD000002010881050147871EAC02D002010985B6
:10AD10001F50020B05E0A4ECD0F002E098ECD1F05B
:10AD2000D6EC39F00101279D239A37D02C50400BE7
:10AD300003E12C50800B33E023AA04D0239A91EC3A
:10AD4000D4F047D027ADDDD1279D010E0D6E27BF72
:10AD50000D68006A050EE66E0050E66EB60EE66EF1
:10AD6000010E04ECCAF00601030E426F0101B65158
:10AD70000EE0B629496E010E495204E0E846FE0B8A
:10AD80004906FCE10601426F1E0E436F02D01EEC25
:10AD90004EF091ECD4F0E5520101AD6BB2D120AE92
:10ADA0001AD0AD5101E0ADD164ECCBF001E0A9D1F6
:10ADB0000B50016E2250100B03E13450800B02E067
:10ADC000E0EC67F0006A00504EECCEF036EC3FF05D
:10ADD000E552E55296D121B694D15AC200F0A8ECC2
:10ADE00026F0A30E02015A5D01E08BD183ECCAF07C
:10ADF00001E187D1E9ECCAF001E083D10101320E13
:10AE000020D0B5B37ED1B5A71ED01950400B04E0B9
:10AE10001950040B01E075D17CECDBF00A0E006EDA
:10AE2000FBEC25F00101040E016F03C700F019AC23
:10AE300002D09EEC04F07EECE1F019AC62D101018D
:10AE4000200E1A6F5ED13BAB46D1070E006E00504C
:10AE5000D880765501E2766B27AD10D0279D010E84
:10AE60000D6E27BF0D680050E66E760EE66E010E81
:10AE7000FFECC9F00601426B0101AD6BAD5101E081
:10AE800040D12050200B01E13CD10201A95101E049
:10AE900038D1070E0101765D40E17CECDBF06AEC15
:10AEA00016F001012B0E166F00010FAE0BD0010141
:10AEB0002D0E166FFF0ED8800E560F56010E0E2661
:10AEC000000E0F22E70E5FECD0F002E295ECD4F01A
:10AED0000E500F1003E10101200E166F0CECD6F09E
:10AEE000640E2CECD6F039C049F03AC04AF0495013
:10AEF000006E0101012B7EECE1F082EC04F0300FDA
:10AF00000101176F300E175D02E1200E176F198FC8
:10AF1000640E1A6F420E1B6FD0D0060E765D1EE1D6
:10AF20007CECDBF067EC16F080ECCCF00101410E1C
:10AF3000166F460E176F560E186F300E195D01E032
:10AF4000E0D0200E196F300E1A5D01E0DAD02CEC43
:10AF5000D8F001E0D6D0200E1B6FD3D0040E765D62
:10AF600003E0050E765D6CE17CECDBF00498050EE9
:10AF70000101765D09E14F0E166F530E176F430EF8
:10AF8000186F3BECD9F026D0500E166F410E176F9C
:10AF9000048864ECCBF006E00101580E186FEAC992
:10AFA00000F01AD00101E6A50DD0320E186FE5A908
:10AFB00002D0340E186F24ECD2F0ABC73DF0ACC712
:10AFC0003EF008D0490E186F24ECD2F0A9C73DF02E
:10AFD000AAC73EF08EECDAF0049000AE02D0006C0E
:10AFE00004800101030E016F3DECCFF004A002D0FC
:10AFF0002D0E196F430E1C6F04B8188F050E765D69
:10B000000FE196A302D0230E09D05751100B01E196
:10B0100078D05751200B01E174D02A0E196F71D0EE
:10B02000E651040B6EE08A51400B6BE080ECCBF0F4
:10B0300068E101014E0E1A6F2F0E1B6F410E3ED0BC
:10B04000760514E17CECDBF0D20EE66EE30EE66EE4
:10B05000010E72ECD7F00BC200F00FECD5F001013D
:10B06000195D02E1200E196F1B8F27D0020E765D4D
:10B0700027E17CECDBF0CA0EE66EE30EE66E010E15
:10B0800072ECD7F0010183513CE033AC02D02A0EC0
:10B09000186F060EE66E820E80ECD3F000500201AF
:10B0A0000B5D006E0101030E016F0FECD5F0010185
:10B0B000195D02E1200E196F1B8F560E1C6F21D0F7
:10B0C000030E765D03E165EC10F01BD0765119E1BB
:10B0D000EAECE3F016D0020119510BE02750400BC7
:10B0E00010E1140E0101AC5D0CE23B0EDFECCAF086
:10B0F00008D00101B5A105D023AA03D0239ACEEC34
:10B1000034F0A4EC14F0006EFF0811E0570E005C60
:10B110000AE1E8ECD4F0C20EE66EE30EE66E010E34
:10B1200072ECD7F004D00050006EA8EC26F00101BC
:10B13000AD5101E0F3D1140EAD6F0201565101E0A3
:10B140005607020E685D01E0E9D1330E0101B95DD9
:10B1500004E00E0EB95D01E0E1D12582DFD1090ED8
:10B16000B75D0AE106015051515D01E1D7D150C6EA
:10B1700051F678EC3DF0D2D10A0EB75D05E1A7ECAF
:10B18000DFF072ECDFF0CAD10B0EB75D01E0C6D183
:10B19000B85124E1A4EC11F0E4ECD5F001E1B8D110
:10B1A0008A51400B09E080ECCBF001E1B1D1040EF3
:10B1B0000101765D01E0ACD112EC13F00701BC0E89
:10B1C000D880AB55020EAC5501E3A2D101018A51E2
:10B1D000400B01E09DD1EDECD6F007D1B8053EE182
:10B1E00033ECD1F001E394D133ECD1F001E390D111
:10B1F0001B50080B01E08CD10101485132080FE2CD
:10B20000770EDFECCAF06EECDFF09AECD4F00DECC8
:10B21000DAF0A50EE66EE30EE66E010EDED0C80E85
:10B2200098ECDAF0F3EC12F00701A80EB6ECD9F0C6
:10B230000DE2940EE66EE30EE66E010EC4ECCAF06B
:10B240008C0EE66EE30EE66E010E9BD0760EB6EC2B
:10B25000D9F001E35DD1EDECD6F0EBD0020EB85D94
:10B2600001E0EDD01BEC10F080ECCBF001E195D0CB
:10B270002050040B01E091D02050400B01E08DD014
:10B280005E0EDE6E010EDD6E01012B51090804E237
:10B29000900EDE6E010EDD6EE6A504D0F40EDE6EBD
:10B2A000010EDD6E21B204D0640EDE26000EDD221A
:10B2B0003BECCBF001E32CD11B50080B01E028D173
:10B2C0001BEC10F0C9ECD8F03BECCBF001E320D143
:10B2D0001BEC10F0050EF1ECC9F03BECCBF001E3F8
:10B2E00017D12CA609D083ECCAF003E0E9ECCAF030
:10B2F0000AE081ECD8F007D0010166518BECD0F068
:10B30000665F07EC53F0460E98ECDAF03BECCBF0BE
:10B3100001E3FED0170E7EECCAF02CA609D083EC18
:10B32000CAF003E0E9ECCAF011E081ECD8F00ED0ED
:10B33000740EE66EE30EE66E010EC4ECCAF0010177
:10B340006651CFECD8F0665F07EC53F0960E98ECA0
:10B35000DAF001ECD8F0320EFBECD2F00201CD5164
:10B36000495CCE514A5801E3D3D0610EE66EE30E3C
:10B37000E66E010EC4ECCAF0590EE66EE30EE66E00
:10B38000010E26ECD3F08BEC10F0010EE66EA0EC73
:10B3900010F0E552D1EC10F0BBD040EC53F00009B6
:10B3A00001E1B6D01B50080B01E0B2D01BEC10F04D
:10B3B00040EC53F0000901E1ABD0170EBBECD9F023
:10B3C0000101E6A514D048510EE0480516ECCDF079
:10B3D0004B0EE66EE30EE66E010EE66E50EC14F0D8
:10B3E000E552E55294D088ECD8F0209425D048510D
:10B3F000320809E22A0EE66EE30EE66E010EC4EC98
:10B40000CAF0320E0BD048511E0811E21C0EE66E37
:10B41000E30EE66E010EC4ECCAF01E0E16ECCDF083
:10B420009AECD4F0640EE66E95EC21F070D088ECC6
:10B43000D8F020949AECD4F030ECCEF069D0030E22
:10B44000B85D2EE1060150932450020B12E11F500B
:10B45000020B04E0E5EC29F0000909E01250080BAA
:10B4600003E11250040B05E003ECD4F002E0060106
:10B4700050832450020B4CE1BFECD2F049E10201B1
:10B48000305146E11FECCEF001E14A5041E02C5032
:10B49000800B3EE12C50400B3BE10601018138D08E
:10B4A000040EB85D35E1A30E1BECCDF00101E5A162
:10B4B00005D00050E66E98EC75F0E55204902150EE
:10B4C000020B01E00480C00E005C02E2219204D075
:10B4D0000050F00801E221822150020B02E08F901F
:10B4E00001D08F800450010B496E2150020B01E006
:10B4F000010E495C0DE08CEC04F0C1EC16F007EC99
:10B5000053F052ECCCF0010EE66EA9EC1DF0E552C2
:10B510000101B82BB851040801E2B86B0101B72B47
:10B52000B7510B0801E2B76B020EE15C02E2E16A7F
:10B53000E552E16EC2EFC9F0016A750E015C0DE2E1
:10B54000A80E496ED90E4A6E010E4B6E015054EC96
:10B55000D5F0ACECD0F0012AF0D71200026A400E10
:10B56000025C08E2B00E0224016E320EACECD0F0A8
:10B57000022AF5D7120031ECD8F0060F016E040E46
:10B580004EECCEF08D0EE66E020E34ECCAF0096A77
:10B59000C2EFC9F031ECD8F0060F016E040EE66E72
:10B5A0008D0EE66E020E42EFD9F031ECD8F00A0FA4
:10B5B000016E020E4EECCEF0910EE66E020E34ECF1
:10B5C000CAF0096AC2EFC9F031ECD8F00A0F016E77
:10B5D000020EE66E910EE66E020E42EFD9F043ECDB
:10B5E000D5F0340E87ECD3F0010E096EDF6A100E31
:10B5F000DF5C42E2026A100E025C3CE2A7ECD6F08D
:10B6000003E0050E025C06E1DF50E824820F57ECF0
:10B61000CCF0006E020403E0060E025C07E1DF508E
:10B62000E824820F010F57ECCCF0006E020EDF5CB5
:10B6300003E3030EDF5C0AE10A0E025C02E1110E75
:10B64000006E0B0E025C02E1240E006E0C0E025C1A
:10B6500005E10A0EDF5C02E11B0E006E0D0E025CBE
:10B6600005E10A0EDF5C02E1200E006EF9EC3AF013
:10B67000022AC1D7DF2ABBD7020E096EDF6A090E84
:10B68000DF5C12E2026A100E025C0CE2A7ECD6F05C
:10B6900003E0050E025C02E11C0E006EF9EC3AF0CC
:10B6A000022AF1D7DF2AEBD7096A46DFDF6A200ECC
:10B6B000DF5C09E2100E006E800EDF24016EF9ECF3
:10B6C0003AF0DF2AF4D7DF6A0B0EDF5C03E246DFD5
:10B6D000DF2AFAD7DF6A090EDF5C35E2DF28006E69
:10B6E0000038F00B006E090E0012DFCFE6FF31ECE0
:10B6F0000CF0E55249ECD9F0EE52090EEF6EFAEC7F
:10B70000C9F0020E60ECD6F02C0EEF6EFAECC9F028
:10B71000030E60ECD6F0010EEF6EFAECC9F0040EE9
:10B720001AECD7F0050E1AECD7F0070E1AECD7F08A
:10B73000080E1AECD7F0060E1AECD7F0090E12EC30
:10B74000CFF0DF2AC8D71FD829D8DF6A060EDF5C02
:10B750000DE2DF5002E1030E01D0010EE66EDF5074
:10B760002CECCBF05CECCCF0DF2AF0D753ECDAF029
:10B77000FD0E016EDB0EACECD0F00101010EB56FD9
:10B78000E552C2EFC9F0020E096E5A0EE66E000EC7
:10B79000E66E030EE66EA20E36EFDBF0D1ECDAF0C9
:10B7A000030E096EFE0E4DECDBF0850E005C02E030
:10B7B000010EDF6E2D0E87ECD3F0140EF6ECD0F0F8
:10B7C000000EE66E0A0E92ECCAF00A0EF6ECD0F00D
:10B7D000CA0EE66E0A0E92ECCAF0040EF6ECD0F039
:10B7E000260EE66E0A0E92ECCAF0DF501DE00F0E38
:10B7F000F6ECD0F0140EE66E0A0E92ECCAF0030ED0
:10B80000F6ECD0F0230EE66E0A0E92ECCAF00A01B6
:10B810002D0E1B6F1BCA1AFA1BCA19FA410E206F94
:10B8200020CA1FFA20CA1EFA0A01D46BDA6BDA8129
:10B83000D56B380ED66F040ED86F3C0ED96F190E2B
:10B84000D76F016A020E015C0CE20150050D3AEC63
:10B85000DBF0000EE9260A0EEA22360EEF6E012A10
:10B86000F1D70101D46B050ED45D18E20701010E7A
:10B87000B16FFF0EB15D0FE0C2EC13F0ABECDAF08C
:10B88000CFECD7F00701B1517EECDAF0E3ECCCF06D
:10B890000701B107EED70101D42BE5D70701B16B42
:10B8A0000101D46BDFCFE6FF3CEC48F0E55274ECCD
:10B8B00048F0030E096EFE0E016E850EACECD0F062
:10B8C000096AE552C2EFC9F00490049201013EB149
:10B8D00004803EB304820450010B02E08E8E01D03E
:10B8E0008E9E0450020B02E08F8801D08F98405149
:10B8F000E8240A0FE66EE66A68ECFCF0E552E552D1
:10B900000C0EBB6E006A01013E5104E1100E3F03B4
:10B91000F350006E0050BC6E1200C6ECC9F079EC1A
:10B92000D5F035ECFDF0E552000902E0C69EF7D7F0
:10B93000C2EFC9F0C79EC698C78C1200C78EC688D2
:10B94000C78C1200F29E8EECD0F0480EBFECD9F0FE
:10B95000480E1EECD7F0480ED5ECC9F00701800E5A
:10B96000146FF90E156F5BECD5F062ECD5F0F28E2A
:10B970001200D9CFE6FFE1CFD9FF030EE126D2ECCA
:10B980000FF0E668930EE66EC1ECFCF0E552E5526E
:10B99000AA9EC26A000000000000000000008A8A1F
:10B9A000209A3386278AD9EC13F00601B66BB76B61
:10B9B000FCEC0CF036ECC4F0D5ECC4F092688F0EC1
:10B9C000E66EE668E2ECFAF0E552E552CF0EE66E7E
:10B9D000E66833ECFCF0E552E552050EE66E53ECFA
:10B9E000FDF0E5520101010E3E6F0101030E3F6FB4
:10B9F0000101020E406F68DFE668870EE66E97EC85
:10BA0000FCF0E552E552B09E0201320E116F000EBD
:10BA1000A56EA26E9F6EA282D08E010EC26EC16A0A
:10BA20000A0EC06E0F01DF0E256F0F01F70E246F97
:10BA30000F01E00E236FDB0E006EB5EC25F000C0A9
:10BA40004AF5010EDB6A100EF36E010EDBCFF4FF38
:10BA5000F350F45C28E28E0E496EDB0E4A6E010E46
:10BA60004B6E010EDBCF4CF04D6A4E6A49504C24B0
:10BA7000F36E4A504D20F46E4B504E20F86EF4CFCA
:10BA8000F7FFF3CFF6FF0800F550E66E010EDB502E
:10BA9000EA6AC50FE96E060EEA22E552E750EF6E3C
:10BAA000010EDB2AD0D70101266B010126918850B7
:10BAB000010B01E02681010126938850020B01E071
:10BAC0002683F28E0601506978EC3DF030ECE1F00F
:10BAD00001018E0EB26FD30EB36F010EB46F02016F
:10BAE00084690601506B78EC3DF00101010EB56FE1
:10BAF0006CECDBF07CECDBF070EC6FF00601178196
:10BB00000601416941C640F60601426B138A128064
:10BB100011881182138613880A01380ED66F0A0124
:10BB2000010ED76F56EC19F072ECDFF01FEC20F02D
:10BB3000010EE66EDEEC3DF0E552166E200E165C50
:10BB400002E101013889010EE66EDEEC3DF0E552BE
:10BB5000000901E0F8D7640EE66E87ECFDF0E552CF
:10BB60001C9ED5ECC4F0096AFC0E016E37EC3BF06C
:10BB7000001CDF6EFC0E016EDF50006EF9EC3AF037
:10BB8000FC0E016E37EC3BF0DF50005C06E0210E4E
:10BB9000E66E65EC14F0E5524ED0830E096EFC0E95
:10BBA000016E37EC3BF0001CDF6EFC0E016EDF50C7
:10BBB000006EF9EC3AF0FC0E016E37EC3BF0096ACE
:10BBC000DF50005C06E0240EE66E65EC14F0E552F2
:10BBD00032D0FD0E016E37EC3BF0DB0E005C03E172
:10BBE000210E165C02E1FBDC1ED0020E016E37EC6A
:10BBF0003BF000C02AF1370E016E37EC3BF000C07D
:10BC00005FF1110E016E37EC3BF000C039F1120EFE
:10BC1000016E37EC3BF000C03AF10F0E016E37ECCD
:10BC20003BF000C037F1E00E016E37EC3BF0005006
:10BC3000800801E293DC0701580E626F020E636F09
:10BC400007018B697BEC0CF0D5ECC4F0A3EC3DF064
:10BC50001F860001116A126A136A146A800E076E49
:10BC6000176A219A750EE66EE66A280EE66E010ED8
:10BC7000E66E62EC3BF0E552E552E552E552020E0B
:10BC8000096E5A0EE66EA20EE66E000EE66E030E0A
:10BC9000E66E62EC3BF0E552E552E552E552030EEA
:10BCA000096E2A0EE66EE66A000EE66E0A0EE66E73
:10BCB00062EC3BF0E552E552E552E552AA0EE66E23
:10BCC000300EE66E2A0EE66E0A0EE66E62EC3BF071
:10BCD000E552E552E552E552FE0E016E37EC3BF0BF
:10BCE000096A850E005C01E059DD060EE66EF00E75
:10BCF000E66EB80EE66E070EE66E62EC3BF0E552BD
:10BD0000E552E552E552040EE66EA00EE66EEA0E2E
:10BD1000E66E060EE66E62EC3BF0E552E552E55249
:10BD2000E5520601EA510A0802E20601EA6B060141
:10BD3000EC51010802E20601EC6B200EE66E800E6B
:10BD4000E66E640EE66E070EE66E62EC3BF0E552C0
:10BD5000E552E552E552830E096EF90E016E37EC9D
:10BD60003BF000C071F202017151C80803E2020108
:10BD7000C80E716FF80E016E37EC3BF0339A6E0E01
:10BD8000005C01E1338ADF0E016E37EC3BF001010C
:10BD9000E391720E005C02E10101E3817E0E096E07
:10BDA000080EE66EE66AB60EE66E020EE66E62EC0F
:10BDB0003BF0E552E552E552E552096A01019C511A
:10BDC000040802E201019C6B1C0E165C10E10101EB
:10BDD000368F0101368D0101369136833695010E7D
:10BDE000E66EDEEC3DF0E552000901E0F8D7090E01
:10BDF000165C09E11B86010EE66EDEEC3DF0E552B5
:10BE0000000901E0F8D701018051060802E20101B2
:10BE1000806BD9EC04F0A0EC0CF001018DAB06D0E6
:10BE200001013C9F01013C9D01013B9F0A0E010164
:10BE3000985D04E301019851640803E201011E0EBC
:10BE4000986F010101015751200B07E00101010129
:10BE50005751100B02E10101579BB6C201F0BDC260
:10BE600002F0FF0E015C07E0015005E0FF0E025CEE
:10BE700002E0025008E102017C0EB66F0201FA0EE8
:10BE8000B76F2EEC4EF001018351050802E201016B
:10BE9000836B01018451020802E20101846B0101FC
:10BEA000425104E001014251020803E20101020E85
:10BEB000426F01016D51230803E201010A0E6D6F0B
:10BEC00001015F8D0101505104E0010150510D0845
:10BED00003E20101010E506F0601EA510A0804E273
:10BEE0000601EA6B0601EB6B01018E9D0101578390
:10BEF00001012E6B460E0101525D04E30101525116
:10BF0000730803E20101540E526F640E01014A5D91
:10BF10000BE301014A51496E4A6A4A3404E249502E
:10BF2000B408000E4A5403E201018C0E4A6F01016D
:10BF30005551150804E3010E0101555D03E20101AD
:10BF4000150E556F040E0101475D04E301014751D1
:10BF5000080803E20101050E476F01017D51496E9A
:10BF60004A6AD8904A5004E6C80E495C000E4A5806
:10BF700003E20101CF0E7D6F01014D51496E4A6A06
:10BF80004A3404E249509608000E4A5403E2010183
:10BF90008C0E4D6F01014C51320803E20101280E55
:10BFA0004C6F01014B51496E4A6A4A3404E24950D0
:10BFB000C808000E4A5402E201014B6B0A0E01014F
:10BFC000415D04E3010141510F0803E201010F0E3D
:10BFD000416F01013551500803E20101010E356F37
:10BFE00001012851320803E20101320E286F550E7B
:10BFF00001014E5D07E0680E01014E5D03E00101A5
:10C00000680E4E6FFF0E0101695D03E00101695189
:10C0100009E10101C80E696FD90E6A6FCF0E6B6F0F
:10C02000060E6C6F01017751010802E20101776B86
:10C03000010166513C0802E20101666B0101675192
:10C040003C0802E20101676B01016851280802E225
:10C050000101686B010101018D51020B05E1010134
:10C060003A5102E001018D8301016151030802E2AE
:10C070000101616BFF0E01015F5D02E101015F6B78
:10C0800001017551496E4A6A4A3404E24950C808B0
:10C09000000E4A5403E201011E0E756F0101315179
:10C0A000020803E20101010E316F3C0E0101E76E4F
:10C0B0007C19E8AE02D07C3503D0E750D8807C559F
:10C0C0000BE3C40E0101E76E7C19E8AE02D0E73441
:10C0D00002D0E7507C5D02E201017C6B01018651D8
:10C0E0000F0802E20101866B01017B510F0802E299
:10C0F00001017B6B01016E513C0802E201016E6B94
:10C1000001016F513C0802E201016F6B0601EB5126
:10C110001E0802E20601EB6B0601ED511E0802E269
:10C120000601ED6B01017F51640803E201011E0E5F
:10C130007F6F01012951496E4A6AD8904A5004E63E
:10C14000280E495C000E4A580BE3010129514B6E41
:10C150004C6A4C3404E24B504608000E4C5403E247
:10C160000101370E296F01018551C80802E2010162
:10C17000856B01018551496E4A6A4A3404E249508F
:10C180009608000E4A5403E20101960E856F0201E3
:10C19000875104E002018751330803E202010D0ECA
:10C1A000876F01018751780803E20101640E876FF0
:10C1B000010193510C0803E20101060E936F010186
:10C1C00095510C0803E20101060E956F010188519B
:10C1D0001E0802E20101886B01018AAF02D0010151
:10C1E0008A6B01018DAF02D001018D6B01018EAF11
:10C1F00003D001010A0E8E6F010196AF03D0010139
:10C20000600E966F1E0E0101895D04E301018951E4
:10C21000280805E201011E0E896F01018A910101C2
:10C220008B510A0802E201018B6B01017A51190856
:10C2300004E201017A6B01018A930101705104E06B
:10C24000010170511E0803E201011E0E706F010111
:10C250003E51010803E20101010E3E6F210EE66E20
:10C26000E6EC13F0E552000909E00101010E3E6F12
:10C270000101030E3F6F0101020E406F64EC5CF0A0
:10C28000318805014B69D0EC0AF00101E38301011B
:10C290002951E8240301B86F5DEC21F0300E010153
:10C2A00084250401F76F020E0101845D03E104019E
:10C2B000340EF76FA5ECA7F004013B0EFE6F0501ED
:10C2C000106B10C512F510C511F50501800E156F24
:10C2D00074ECC7F092ECC7F09BECC7F0000905E1E5
:10C2E0002D0EE66E65EC14F0E55207013C0E846FEE
:10C2F0000101D56BD5C1D4F10701B16B0BEC75F021
:10C300000701BE817BEC0CF048EC1EF007EC53F00B
:10C3100028EC53F00101010138510701099F040B7A
:10C3200001E0098F8BEC20F0E6ECC3F01FDBD5ECCD
:10C33000C4F0A4EC11F0F3CF0EF0F4CF0FF0430EE5
:10C340000E5C010E0F5806E3D30ED8800E54020E79
:10C350000F5411E20EC049F00FC04AF0040ED890FD
:10C360004A324932E804FBE149C026F75A0EE66E2C
:10C3700065EC14F0E552F3EC12F0F3CF0EF0F4CFCD
:10C380000FF01F0E0E5C010E0F5806E3D30ED8807F
:10C390000E54020E0F5411E20EC049F00FC04AF0C5
:10C3A000040ED8904A324932E804FBE149C026F72E
:10C3B0005D0EE66E65EC14F0E552550EE66E020E6B
:10C3C000E66E400EE66E0CECC4F0E552E552E55226
:10C3D000020EE66E400EE66E58ECC4F0E552E552F1
:10C3E000006E550E005C07E000C026F7600EE66E9A
:10C3F00065EC14F0E552E66A020EE66E400EE66E5B
:10C400000CECC4F0E552E552E552AA0EE66E020EBF
:10C41000E66E420EE66E0CECC4F0E552E552E552D3
:10C42000020EE66E420EE66E58ECC4F0E552E5529E
:10C43000006EAA0E005C07E000C026F7630EE66EF1
:10C4400065EC14F0E552E66A020EE66E420EE66E08
:10C450000CECC4F0E552E552E5520201440E976F30
:10C46000120EE66E420EE66E58ECC4F0E552E5524E
:10C47000046E026E0450800B01E0010E496E045000
:10C48000400B01E0010E495C23E1047C0450E66EA0
:10C49000120EE66E420EE66E0CECC4F0E552E5526A
:10C4A000E552120EE66E420EE66E58ECC4F0E5520E
:10C4B000E552046E0450800B01E0010E496E0450F9
:10C4C000400B01E0010E495C03E10201450E976F4C
:10C4D0000250E66E120EE66E420EE66E0CECC4F0F2
:10C4E000E552E552E5520101835116E05EECE4F0BD
:10C4F00000090AE0EBECE2F04AECE3F001018351C1
:10C50000010801E2338C08D00701050E266F1E0ECC
:10C51000E66E65EC14F0E5525CECBDF02B962296CD
:10C5200001013A510101941101E17CD0150EE66E32
:10C53000020EE66E440EE66E0CECC4F0E552E552D7
:10C54000E5522A0EE66E020EE66E460EE66E0CEC24
:10C55000C4F0E552E552E552020EE66E440EE66E78
:10C5600058ECC4F0E552E552150802E1000E01D086
:10C57000010E006E005014E001013A5108E000C0C5
:10C5800026F7660EE66E65EC14F0E55208D007015A
:10C59000030E266F180EE66E65EC14F0E55242D0DD
:10C5A00001013A5118E0020EE66E460EE66E58ECB6
:10C5B000C4F0E552E5522A0802E1000E01D0010E56
:10C5C000006E005008E000C026F7690EE66E65ECCC
:10C5D00014F0E55227D0120EE66E440EE66E58ECCB
:10C5E000C4F0E552E552006EC00E001601013A514A
:10C5F0000CE0005008E000C026F7840EE66E65EC03
:10C6000014F0E55201D02B860DD0C00E005C09E07D
:10C610000701040E266F180EE66E65EC14F0E55265
:10C6200001D02286A2EC5CF01B92010194511FE024
:10C63000370EE66E020EE66E480EE66E0CECC4F0A7
:10C64000E552E552E552020EE66E480EE66E58ECF3
:10C65000C4F0E552E552370809E00701010E266FE4
:10C66000180EE66E65EC14F0E55201D01B822580B1
:10C67000E66863EC36F0E55239C1E6FF21ECC3F021
:10C68000E5520101B581219401013BBB06D00601B1
:10C6900050950601508778EC3DF00101D45104E03B
:10C6A000030E0101D45D04E10A01D46B149C04D093
:10C6B0000A01020ED46F148C93D901012ABD0CD04B
:10C6C000B5ECC8F0C6C269F1C7C26AF1C8C26BF165
:10C6D000C9C26CF101012A8D81EC2EF00201320EEB
:10C6E000246F0101100EB96F0501010E176F0901CA
:10C6F000020EE56F0201582B0201320E226F85EC0B
:10C7000096F08CEC04F00201CF5108080AE2D9EC53
:10C7100013F0CFC226F72A0EE66E65EC14F0E55250
:10C720001B860D0EE66EE0EC14F0E552870B006EF2
:10C73000005008E000C026F73C0EE66E65EC14F0F1
:10C74000E55214D04CEC20F03B0E0E5C000E0F585E
:10C7500006E3E60ED8800E54030E0F5407E20EC017
:10C7600026F7570EE66E65EC14F0E552030EE15C19
:10C7700002E2E16AE552E16EE552E7CFD9FF12002D
:10C78000440E0101B95D03E3B951490801E2000C0F
:10C79000010C01013B7B279D256B1DD8238A258237
:10C7A00001013BBB13D009014F0EE66F460EE76F48
:10C7B000060150A707D00901560EE66F420EE76F3B
:10C7C000010136890601436B43C642F601013BBBBA
:10C7D0000480DBEF09F006015097509501013BBB47
:10C7E00007D021B403D006015085120006015087FE
:10C7F00012000A01D65151EFDBF0D4C100F0005015
:10C8000003E0030E005C33E100500EE10101D07D36
:10C810000901430EE66F0101D0AD02D09DECD1F0CD
:10C820000101D0AD20D010D08DECCDF00FE0010192
:10C83000D0750901440EE66F0101D0A502D09DEC30
:10C84000D1F00101D0A50FD004800DD00101CF752A
:10C850000901440EE66F0101CFA502D09DECD1F095
:10C860000101CFB50480DBEC09F0FFEFD3F0000449
:10C8700003E0020E005C16E1C2EC13F0000402E1DA
:10C88000020E01D0010E006E09014C0EE66F020E81
:10C89000005C03E10480550EE66FDBEC09F000C09C
:10C8A000D4F166D812000101325103E183ECCAF0E1
:10C8B00002E0000E01D0010E1492E8B0148283EC65
:10C8C000CAF003E11BECD5F00CE183ECCAF007E001
:10C8D000E9ECCAF004E101013B51800B02E1000EDA
:10C8E00001D0010E1490E8B01480120083ECCAF05D
:10C8F0000AE0EFECD2F007E1C3ECD2F004E0E4ECA4
:10C90000D5F001E1000C010CEBECD2F003E00101E9
:10C9100081511200010178511200EBECD2F003E0DA
:10C92000010182511200010179511200C6ECC9F0D7
:10C93000EBECD2F005E0FE0EDB500101816F04D07C
:10C94000FE0EDB500101786FC2EFC9F0C6ECC9F0F2
:10C95000EBECD2F005E0FE0EDB500101826F04D05B
:10C96000FE0EDB500101796FC2EFC9F08DEFD7F0F9
:10C9700021902792D4C100F00050800802E2050EF9
:10C98000006E060E005C01E3006A000402E1010192
:10C99000CF91020E005C02E10101CF8100C0D4F111
:10C9A000248A20BE03D088ECD4F002D0D6EC39F033
:10C9B00056EF25F043ECD5F0030EDF6E010149512F
:10C9C000496E4A6AB00E3D6E040E3E6E48ECCAF0E7
:10C9D0003D50D880DF540201506FE552C2EFC9F0DC
:10C9E00043ECD5F026B00ED0320EDF6E080E0101FA
:10C9F000495D02E2080E496FDF50D880495502E2D6
:10CA0000DFCF49F1D7DFE552C2EFC9F050C2B0F134
:10CA100022AE34D0006A01013D510C0803E3070E39
:10CA20003D5D02E20C0E3D6F070E3D5D4D6E4E6AA0
:10CA3000020150516EECCBF0006E4FECDAF00101C8
:10CA4000B0514B6E4C6AFF0ED8804B56000E4C56C0
:10CA50004A504C18E8AE02D04C3404D04B50495CDC
:10CA60004C504A580BE20050D880B05507E223A042
:10CA700003D00050B02702D00050B05FAFECD0F030
:10CA800008E102012D510601EA1106E02750400B92
:10CA900003E11D929CEC3CF01200050E98ECCEF0E8
:10CAA000580E04EFCFF0F9DF258E1200180E7EEC41
:10CAB000CAF0010136AD03D0580E04EFCFF0258E39
:10CAC0001200C6ECC9F0050EE1261FA20FD0BFC1AF
:10CAD000DFFF010EC0C1DBFF020EC1C1DBFF030E91
:10CAE000C2C1DBFF040EC3C1DBFF0ED0BAC1DFFF42
:10CAF000010EBBC1DBFF020EBCC1DBFF030EBDC1DB
:10CB0000DBFF040EBEC1DBFFE4ECD5F022E0E55113
:10CB1000100B1FE13851010B03E19651040B06E0A5
:10CB2000320EDF5C62E3DF5033085FE32E50800B90
:10CB300006E0320EDF5C59E3DF50350856E32E5035
:10CB4000800B3BE12F0EDF5C50E3DF50380835E20D
:10CB50004CD0DF504AE0DF0404E1460E44ECCCF058
:10CB600044E3DF50180806E21C0EDF5C03E2965136
:10CB7000010B23E1E5BD07D0DF50180815E21C0EBC
:10CB8000DF5C12E232D0190EDF5C2FE01A0EDF5CA0
:10CB900004E1010EDB505F0828E31B0EDF5C04E1BB
:10CBA000290E44ECCCF021E32B50100B06E12E5063
:10CBB000800B03E02B510A0802E2F36A1BD0630EDC
:10CBC000E66E020EE66ED9CFE6FFDACFE6FF3CEC6A
:10CBD000CDF00BE1D9CFE6FFDACFE6FF5E0EE66ED1
:10CBE000020EE66E3CECCDF004E060DF010EF36E69
:10CBF00001D0F36AF46A050EE15C02E2E16AE552F3
:10CC0000E16EC2EFC9F065C301F022A802D078C37B
:10CC100001F00E0E015C01E2010C100E015C01E25C
:10CC2000020C120E015C01E2030C140E015C01E225
:10CC3000040C160E015C01E2050C1B0E015C01E206
:10CC4000060C220E015C01E2070C080C69ECD5F021
:10CC5000F5ECD9F0F00801E2006A0050C2EFC9F02B
:10CC6000C6ECC9F079ECD5F0F1DFE552FE0EDB50F1
:10CC70009B0805E1030E11ECD6F0F6ECCDF0E2ECEA
:10CC8000D6F004E6DC0E495C000E4A580AE20F0EAC
:10CC9000496ED50E4A6E010E4B6E005054ECD5F025
:10CCA00001D0D20E0E6E0F6AE2ECD6F004E6AA0EA8
:10CCB000495C000E4A580CE2650E496ED40E4A6E6D
:10CCC000010E4B6E005054ECD5F00101D86F02D02C
:10CCD0000101D869D96BC2EFC9F043ECD5F00490DB
:10CCE00034B80480B30E016E0101E6A539D01BB63D
:10CCF0002AD0B30E22ECD7F0D8C1D7F244EC20F002
:10CD0000026E300EDF6E020403E0020E025C02E1EE
:10CD1000380EDF6EDF500201D880D75509E229ECCA
:10CD20000EF0150EE66EE30EE66E010EF6ECC9F09F
:10CD3000DF50496E4A6A0101D851495CD9514A58BD
:10CD400002E24851D6E1070114B108D014815BEC2E
:10CD5000D5F07D0E976E080E64ECD8F09B0E016E38
:10CD6000015022ECD7F064ECCBF012E00E50010140
:10CD7000D66FD76BB30E22ECD7F00E50E9ECD6F09D
:10CD80000101D6274A50D723D6C10EF0D7C10FF0E4
:10CD90000101E6A502D0D86BD96BD8C161F3D9C126
:10CDA00062F334B80AD113A64DD00B50016E225055
:10CDB000100B03E13450800B02E002D913D064EC75
:10CDC000CBF010E00701C1514D6E4E6A0B506EEC76
:10CDD000CBF0016E2050800B05E00901EC5102E020
:10CDE000ECC901F0050E0124496E0A0EC0ECCAF030
:10CDF000016E015005E12250400B02E0010E016E70
:10CE000083ECCAF003E03450400B05E001C0A3F707
:10CE100002010A0E08D00701A351015C05E301C01D
:10CE2000A3F702010C0E2A6FEEDE0701A46F2B5050
:10CE3000100B03E1040E0B5C01E2A46B13ECD0F0C9
:10CE40001BECCEF091ECCDF00480005009E03450A2
:10CE5000400B06E1030E005C04E1020E0A5C01E1F6
:10CE60000490070E016E04A004D0090E76ECCBF0FE
:10CE7000016E0F0E01140201736F070E7317013854
:10CE80000F0B016E04A0016A13A408D0020EE66E17
:10CE900073C2E6FF0150E66E1BECCEF052C100F00B
:10CEA0000101E6A502D04AC100F04FECDAF0C1EC76
:10CEB000CBF09AECD6F0FBECD6F0640E4FECD9F048
:10CEC0000E500B6E91ECCDF0040E005C0BE00004F4
:10CED00009E0020E005C06E0030E005C0AE1020EAF
:10CEE0000A5C07E00201AF51D8800B5402E20BC08C
:10CEF000AFF20101E6A507D00301636B646B676BBA
:10CF0000686B656B5AD0B70E22ECD7F0D8C163F3CB
:10CF1000D9C164F303016151635D6251645906E351
:10CF2000010E6325616F000E6421626F61516325FC
:10CF3000676F62516421686F67516725496E685158
:10CF400068214A6E67C34BF068C34CF0030ED8905B
:10CF50004B364C36E804FBE149504B240301676F24
:10CF60004A504C20686F6351615D496E625164554F
:10CF70004A6E9AECD6F067C33DF068C33EF0E2EC2F
:10CF8000FDF03DC067F33EC068F367C365F367C358
:10CF900049F068C34AF04B6A4C6A4C34000E4C1896
:10CFA00009E6D880FF0E4954000E4A54000E4B5437
:10CFB000000E4C5402E203016569E552C2EFC9F06C
:10CFC00048C101F02B50100B05E164ECCBF002E0FE
:10CFD000D5C201F0120091ECCDF000500DE03450BC
:10CFE000400B0AE1050E005C07E0030E005C03E164
:10CFF000020E0A5C01E0000C010C0482ECDF000967
:10D0000001E00492348604A23496349866DE34B883
:10D01000120091ECCDF004980496030E005C01E13F
:10D020000486000403E0020E005C01E10488225043
:10D03000400B01E1F8D02250100B01E0F4D0345045
:10D04000800B01E0F0D03350080B01E1ECD002017D
:10D050001D5101E0E8D01950010B01E1E4D0048238
:10D060000494B9DF000901E00492040E005C01E1C0
:10D070000484A6DF0150CFECD8F0026E6BECCAF04E
:10D0800001C03EF03CECFEF03EC007F1020E010193
:10D09000075D02E2020E076F07510A0802E20A0E5C
:10D0A000076F0450040B07E00201735104E1D890AC
:10D0B0000132D890013204902050800B33E00901F6
:10D0C000ED5130E064ECCBF02DE00901EE510208A7
:10D0D00029E2030E006EEE51190802E2020E006E04
:10D0E000EE51280802E2010E006EEDA104D00050BE
:10D0F00088ECD2F00480020E0901ED150FE04FEC30
:10D10000DAF002010051495C01514A5807E200502F
:10D11000E9ECD6F0005F4A50015B0480040E09017F
:10D12000ED1772D001500B5C42E20201880E005DE7
:10D13000130E015969E203016C0E635D000E645920
:10D1400063E204B20AD00B50015C0E6E0F6A0E50FF
:10D15000020100270F50012356D002011E5154E155
:10D160000A0E1E6F0150AF5D20E2AF5103E1735113
:10D1700001081BE204A802D0020E1E6F0450080B27
:10D180000FE0030E0A5C03E07351010809E201019C
:10D19000075188ECD2F01F5107E01E911E4304D0C6
:10D1A000020E0027000E01230480AF6B2DD001502A
:10D1B000D8800B5429E2010E036E04A208D007C1E7
:10D1C00003F004A804D0030E0302F3CF03F00350CE
:10D1D0000E6E0F6A0450020B06E00450080B09E0C3
:10D1E00002011F5106E001500B5CF9ECDAF0FBEC98
:10D1F000D6F0020100510E5C01510F5805E20E50AD
:10D20000005F0F50015B048004A00DD002010251A9
:10D21000001902E10351011906E0F1EC0BF000C224
:10D2200002F201C203F20201205102E00F0E206F50
:10D230001200D1ECDAF01750100B0CE0200E155C48
:10D240004CE0210E155C49E0150E155C03E1C3ECC2
:10D25000D2F043E01750010B09E0150E155C3DE0DC
:10D26000220E155C3AE01D0E155C37E00A0E155CC7
:10D2700003E19CECCAF031E01950200B12E10201ED
:10D2800019510FE1230E155C28E00B0E155C25E00B
:10D29000090E155C22E0090E155C1FE0220E155CDC
:10D2A0001CE01FECD5F004E08EEC96F0000915E1CF
:10D2B0001D0E155C07E11750100B04E0DEEC18F0B2
:10D2C00000090BE12050800B06E10201685103E0E8
:10D2D0003250200B02E0000E01D0010EDF6EDF5055
:10D2E000E552C2EFC9F00101E6A509D00701158199
:10D2F00062ECD5F00701149F14935BECD5F0030E9C
:10D30000E66E8DEC16F0E5528A8607010B919BECD8
:10D31000C4F0FCEC18F083ECCAF003E03450400B8E
:10D3200011E06DEC0BF000090DE0E4EC08F086EC88
:10D3300016F06F0E2CECCAF0C80E88ECCDF0E7ECBE
:10D3400008F002D086EC16F00601509178EF3DF01F
:10D350005BC248F15CC200F25DC201F2F1EC0BF07D
:10D3600099EC23F0E0ECD1F0239612000101B051CA
:10D3700003E12B820850076E2050010B12E083EC72
:10D38000CAF00FE11750800B03E03CECD2F006E04E
:10D390002050040B06E11EECCDF003E06AD97FECCF
:10D3A00071F012000101050EAF6F2050010B04E077
:10D3B0001950020B01E0AF6B120095ECD6F00101A1
:10D3C00039512BE105C2DFFF2FECBEF0DF50020127
:10D3D000055D23E0010E69C3DBFF020E6AC3DBFFBC
:10D3E000030E6BC3DBFF010EE66ED4ECBEF0E5521C
:10D3F000010EDB500301695D08E1020EDB506A5D3E
:10D4000004E1030EDB506B5D08E07EECBDF0D5EC73
:10D41000C4F01C820101960EAC6F040EE15C02E2C6
:10D42000E16AE552E16EC2EFC9F00201185107E06E
:10D43000186B09ECCFF00201D05101E1119483EC9B
:10D44000CAF009E12050010B06E11BECD5F003E125
:10D450002050800B0FE0AFECD0F00CE11E50400BE1
:10D4600009E160ECCCF004E1020E0101B95D02E0DB
:10D47000228CD18022BC06D0E66AE66A740EECECFF
:10D48000C9F017D0C3ECD2F012E13350080B0FE013
:10D4900000C249F001C24AF0030E0F0B03E073EC27
:10D4A000D0F0FDE149500201005F4A50015BF1EC10
:10D4B0000BF002010A0E1E6FAF6B20AE1C84C80E6B
:10D4C0001F6F7FEC16F0780E006E005088ECCDF0E8
:10D4D00039EC18F00201226B0101E6A509D0070121
:10D4E000148F01012AA102D0070114835BECD5F04F
:10D4F0008A96320E88ECCDF013ECCBF014E12B5071
:10D50000080B11E02250100B0EE101013A050BE06F
:10D5100083ECCAF007E12050800B04E102011E0EEB
:10D52000156F01D04ADF2050800B0EE12050010B17
:10D530000BE183ECCAF008E03450400B05E1020136
:10D540002D5102E0050110511DAC02D028EC0CF069
:10D55000208C3182D5CA85F291ECCDF0360E026E68
:10D56000380E036EBAC17DF255ECD9F03EC07EF2A2
:10D5700052EC2FF0BAC17BF255ECD9F03EC07CF2F0
:10D580001FA20AD0BFC17BF26BECCAF0C0C13EF053
:10D590003CECFEF03EC07CF222AC26D007010B8FA3
:10D5A0000B819BECC4F043ECD2F008E15751010B26
:10D5B00005E00701088F089DADECD5F0030E0101D1
:10D5C0002B5D04E102017B51070808E3040E010111
:10D5D0002B5D0AE10A0E02017B5D06E20701088F5E
:10D5E00008970895ADECD5F02F8E20EC32F00201B3
:10D5F000FA0E236F238A2582319222AC02D09FEC4F
:10D60000D4F055EC39F021AE12D0219E24EC0BF071
:10D6100063ECD7F07DECD5F00AE07DECD5F007E0C7
:10D620007DECD5F004E017EC0BF039EF6BF0020164
:10D63000145109E00101E551080B05E1140E72ECEB
:10D64000CAF00101E587120043ECD5F0050123077C
:10D650002451EA6A270FE96E050EEA22EFCFDFFFB9
:10D66000242B24511F0801E2246BDF50E552C2EF46
:10D67000C9F0C7EC21F00201196B19C255F2EFECA9
:10D68000D1F007E0200E01011C5D03E0200E11EC3B
:10D69000CDF00101B06B006A3DEF75F04B0E026EEC
:10D6A000140E0301655D07E343ECD2F01EE11E0E8C
:10D6B0000301655D1AE2100E01012B5D16E22B508D
:10D6C000100B03E0640E485D11E02B50100B0DE1D0
:10D6D000280E485D0BE03C0E485D08E0020E395D07
:10D6E00004E15A0E0224485D01E0000C010CD1EC6B
:10D6F000DAF01B50080B0AE160ECCCF009E13C0EBB
:10D700000101B95D03E0430EB95D02E1000E36D0C0
:10D710000101815102E0825104E1480EFFECCAF0A0
:10D72000DF2A0101785102E0795104E14B0EFFEC50
:10D73000CAF0DF2AB3DF00091CE19FEC35F00009D5
:10D7400006E03F0EFFECCAF0C6ECD0F0DF2AC4ECD6
:10D7500035F0000907E0420EFFECCAF00201916BC0
:10D76000926BDF2A0701C05104E1450EFFECCAF0BD
:10D77000DF2ADF5002E07DDF2094DF50E552C2EF68
:10D78000C9F052ECCEF002E27B5112008651120039
:10D7900043ECD5F00750DF6E27AA03D002011E0E1E
:10D7A000216F050110510201191103E137513811A0
:10D7B00009E01D50040B0FE01D50080B0CE01E503B
:10D7C000010B09E01750800B08E02750200B05E102
:10D7D0000501105102E04DDFB4D2075049E127BAEC
:10D7E00004D0F7ECCEF0020E87D081DF000901E013
:10D7F000A8D20201245101E0A4D220B002D015DE4B
:10D800000AD02D5108E00501105105E1BFECD2F01E
:10D8100002E1F7ECCEF0C3ECD2F019E1020189A5E8
:10D8200014D0330E875D0EE10101E451800B03E15A
:10D830002D50080B0CE02D96B1EC04F00201330ED4
:10D840003A6F05D0B1EC04F002D0B5EC04F099DFEA
:10D85000050DF3CFAFF10101E6A512D10A0EAF5DC0
:10D8600002E20A0EAF6F0701159162ECD5F008D104
:10D87000070420E10101AF5101E05FD21F9C13ECCE
:10D88000CBF002E01F8C05D0BFECD2F002E148ECF7
:10D890000BF00101280EAF6FE6A505D00701158535
:10D8A000158362ECD5F020AE03D00101050EB06FF8
:10D8B000072A17D0020E075C16E10201155102E09B
:10D8C0001E0E156F27BA06D00101B05101E035D206
:10D8D00008505DD10101AF5102E1FDEC67F052EC5F
:10D8E0000BF044DD2AD2030E075C3CE127BA06D0D8
:10D8F000006A3DEC75F0070E076E23D22BA218D0FC
:10D900005BC1AFF10101B05105E03BDF050DF35004
:10D910000101AF272B922050010B04E01950020B9C
:10D9200001E0AF6B02012D5103E0006A3DEC75F0A0
:10D930000101AF5106E083ECCAF00FE03450400B18
:10D940000CE11F50400B05E102012D5102E14DECAD
:10D950000BF00101280EAF6F19D126B8EED1FDEC06
:10D9600067F0EBD1050E075C62E10101AF5101E008
:10D97000E4D1072A269820B0E0D11C0E016E01DF09
:10D98000E8240124006E0201765107E00050765D24
:10D9900004E2090E076E2688D0D1318207010B9F61
:10D9A0009BECC4F043ECD2F008E15751010B05E0C9
:10D9B0000701089F088DADECD5F0030E01012B5D2A
:10D9C00004E102017B51070808E3040E01012B5D0D
:10D9D00011E10A0E02017B5D0DE20701089F030EB3
:10D9E00001012B5D03E10701088502D007010887CB
:10D9F000ADECD5F00101E6A508D00701159515930A
:10DA000062ECD5F001010A0EAF6F209C85C2D5FAF9
:10DA100086ECC4F067ECD4F083ECCAF003E0345039
:10DA2000400B03E00101050EAF6F319286D1060E67
:10DA3000075C28E10101AF5101E07FD120B01ED089
:10DA40002650100B0DE1325109E083ECCAF003E0DF
:10DA50003450400B03E01BECD5F002E144DC0ED067
:10DA600032C122F226A80AD08CDE10ECD8F0006E6B
:10DA700000500201225D02E200C022F20201566B58
:10DA8000072A5BD1070E075C24E10101B0510FE1C9
:10DA900017AE0BD03CECD2F003E04BEC97F005D086
:10DAA0009DEC0BF0000901E0179E0850076E020183
:10DAB0002D5101E042D12A5106E03450400B03E1E0
:10DAC00013ECD0F003D0E66AE66AE66AABEC28F025
:10DAD00047D0080E075C4BE10101B05106E01D5034
:10DAE000040B03E01D50080B02E10850076E020111
:10DAF0002D5101E122D1FDEC67F052EC0BF0020157
:10DB00002E5101E01AD141EC0EF0000901E115D1CE
:10DB10000501020E266F235111E096DD006E020E04
:10DB20000A5C02E1005010D0016A0501235102E0B5
:10DB30008BDD016E00504EECCEF00ED0105114E192
:10DB4000020E0A5C07E1030EE66E150EE66E2CEC83
:10DB500016F007D0E66AE66A160EE66E32EC16F0AC
:10DB6000E552E552E552E9D002012D6BE6D0090EEF
:10DB7000075C28E1020176417F0B76250101D88000
:10DB8000B15507E20201766B76C2B1F1050E076E60
:10DB9000D4D01EB0D2D0010EB16F320EAF6F010ED5
:10DBA000076E83ECCAF003E002012D5108E0BFECE0
:10DBB000D2F005E12750200B02E1F7ECCEF00B0E7E
:10DBC000086EBBD00A0E075C06E121BAA9D0179EE9
:10DBD0000B0E076EA7D00B0E075C01E0A6D0175006
:10DBE000800B39E12050010B06E02050040B03E1CB
:10DBF0001EECCDF030E183ECCAF003E03450400B72
:10DC00000CE02050800B09E11E50010B06E01D5076
:10DC1000040B03E01D50080B1EE183ECCAF00CE07E
:10DC20003450400B09E12050040B06E11EECCDF00E
:10DC300003E0EEECD0F00FE02050800B09E01D5027
:10DC4000040B09E01D50080B06E01EECCDF003E0CC
:10DC500013ECCBF05BE017AE18D01950800B07E047
:10DC60000A0E155C04E037EC2DF000096AD03CEC9C
:10DC7000D2F005E04BEC97F0000907E162D09DEC93
:10DC80000BF0000902E0179E5CD083ECCAF023E0A1
:10DC90003450400B20E1E9ECCAF01DE119AA06D08E
:10DCA00017EC0BF0C0EC08F07CEC1DF0AFECD0F002
:10DCB0000AE01950400B07E0249223BC248217ECA1
:10DCC0000BF0DAECD0F00101885105E088C1E6FFE5
:10DCD00095EC21F0E552B1C176F20101B15102E0BB
:10DCE000010EB16F26A802D0FDEC67F00701A16B11
:10DCF000030E076E800E086E2050800B03E1175054
:10DD0000800B08E020940C0E086E04D022A802D0EC
:10DD10009BECBFF00101AF5105E12650100B02E171
:10DD2000FDEC67F052EC0BF008D00C0E075C05E13F
:10DD300021BA03D0FBEC98F007D8DF50075C01E074
:10DD40001C8CE552C2EFC9F020AEABD01D50040BC5
:10DD5000FDE01D50080BFAE02A840101B59B238ADF
:10DD6000B59925829D510BE01FA203D09DC1D5F12D
:10DD700002D09DC1D4F152EC2FF0B8EC64F02250E7
:10DD8000100B03E13450800B04E0A8EC69F0349EE2
:10DD900063D084DC000950E064ECCBF04DE13FEC53
:10DDA000D4F000C20EF001C20FF00EC04DF00FC053
:10DDB0004EF088ECCBF019ECD1F06BECCAF00BC252
:10DDC0003EF04BECD8F0006E00503AECCAF0C40EB6
:10DDD000406E160E416E020E426E436A08ECD9F098
:10DDE00000503AECCAF048C149F097ECD5F011EC7C
:10DDF000FDF03EC0EDFF3DC0EDFF3CC0EDFF3BC080
:10DE0000EFFF070130513111321133110CE0DC0EFC
:10DE1000305D000E3159000E3259000E335903E2C5
:10DE200030C700F007D030C726F74E0EFFECCAF01F
:10DE3000DC0E006EF9EC3AF018A804D0A8EC69F0FA
:10DE400018980AD00901EC5107E064ECCBF004E02B
:10DE50000BC0D5F20901ED6B209E33A403D0D6ECA4
:10DE600039F005D0010EE66E65EC39F0E5522298E6
:10DE700086ECCCF056EC25F0010136BF04D0050E3F
:10DE8000A4ECD6F00ED036AD0CD0E385E783E79551
:10DE9000E7970601FB29FC6F65C3E6FF4FEC0AF02C
:10DEA000E552800E076E12002F50100B04E00101A6
:10DEB000E851080B13E00701555110E10101B5517C
:10DEC000200B0CE13B51200B0AE060ECCCF007E0AA
:10DED000A95105E10101E851080B01E1000C010C19
:10DEE000070EE66EE66A200EE66E440EE66E060E3D
:10DEF000E66EC8ECFAF0050EE15E120045C644F687
:10DF000046C645F647C646F648C647F649C648F6E9
:10DF10004AC649F6120049C64AF648C649F647C6F7
:10DF200048F646C647F645C646F644C645F60601D7
:10DF3000200E446F1200C6ECC9F031AA02D02AECC0
:10DF4000D3F00101E551020B0CE0280E0901BB5D85
:10DF500008E2BB51BB2BEA6A930FE96E090E06EC8F
:10DF6000D8F00101E851200B0CE0280E0901E45D16
:10DF700008E2E451E42BEA6ABC0FE96E090E06ECF4
:10DF8000D8F0C2EFC9F0C6ECC9F00101E8B704D07F
:10DF900079ECD5F003D8E552C2EFC9F047ECD5F0E3
:10DFA000010EDB6A1A50010B0AE0800E4CECCAF03D
:10DFB00004E2FE0EDB50200802E11A905CD09EDFE6
:10DFC000FE0EDBCF4AF6DB50800804E0850E4CECF9
:10DFD000CAF003E30601200E21D0FE0EDB5030080C
:10DFE00003E10601630E1AD02950200B1CE02850D3
:10DFF000080B19E1DF6A150EDF5C15E21BECD9F0A6
:10E000000FE1DE52010EDD6EDF2A4AECCDF0060193
:10E010004A6F74DFDF2A4AECCDF006014A6F03D065
:10E02000030EDF26E8D760ECCCF012E0010EDB50E7
:10E0300004E049C6E6FF7FDFE5524AC600F0630E02
:10E04000005C02E1300E006E0050E66E74DFE552B7
:10E050002BDF000910E016ECCFF044C616F145C6E0
:10E0600017F146C618F147C619F148C61AF149C654
:10E070001BF14AC61CF1020EE15C02E2E16AE552C4
:10E08000E16EC2EFC9F043ECD5F00750DF6E23928A
:10E09000100E075C13E11C0E076E02015151010BBB
:10E0A00003E11D50040B02E1110E92D05151040BFB
:10E0B00027E11D50080B01E0B3D022D0110E075C00
:10E0C00009E12380228E0201080E516F2382076A24
:10E0D000120EA5D0120E075C06E123902382030ED8
:10E0E000076E130E9CD0130E075C0CE11C0E076E1E
:10E0F00002015151040B04E11D50080B01E090D0C6
:10E10000140E66D0140E075C10E12380228E180EC8
:10E11000076E1D50040B01E083D01D50080B01E079
:10E120007FD02382076A150E7AD0150E075C0CE1AA
:10E1300001012AAF03D00201020E516F229E2382F9
:10E14000020E076E160E6BD0160E075C05E12382D9
:10E15000020E076E170E63D0180E075C07E102016E
:10E16000020E516F2382076A190E59D0190E075CEF
:10E1700006E1229E2382020E076E1A0E50D01A0E5E
:10E18000075C05E12382020E076E1B0E48D0170EB6
:10E19000075C08E101012ABF03D00201020E516FA2
:10E1A0001B0E16D01B0E075C05E12390228E2382E6
:10E1B000030E33D01C0E075C33E12390800E076EF4
:10E1C00002015151010B03E11D50040B03E1110E3B
:10E1D000076E26D034AC0BD044EC20F0010802E1ED
:10E1E000520E01D0500E2CECCAF0349C19D01750AE
:10E1F000800B16E1AFECD0F004E0090E0201535D94
:10E200000AE30601EA5104E0080E0201535D03E34C
:10E2100002012D5105E02382080E076E100E086ED4
:10E2200023A202D006EC65F0DF50075C01E01C8CF5
:10E23000E552C2EFC9F01C9612000201566BE66A65
:10E24000E66AE66A1BECCEF002012A6B0701A36BBB
:10E250000B6A20B003D0208015EC6AF0120043EC6A
:10E26000D5F00201050E2D6F280E2E6FE6DF020E8F
:10E270000A5C05E168ECD1F0140EECECC9F0050184
:10E28000040E266FE552C2EFC9F0348C0101D05163
:10E29000400B02E1530E01D0510E2CEFCAF00101E8
:10E2A000E351020B18E03C51800B15E12050010BAB
:10E2B00012E12550040B0FE12450020B0CE1E39313
:10E2C0002F882A0EE66EF20EE66E010EF6ECC9F00D
:10E2D0000101AA0EAC6F12001BECD5F004E1205036
:10E2E000010B01E1000C010C01015651800B05E00E
:10E2F000020E005C03E0000401E0000C010C43ECA2
:10E30000D5F0EFECD2F005E068ECD1F0140EECECB7
:10E31000C9F0209020940701A16B30ECCEF0E552BB
:10E32000C2EFC9F052ECD8F0800E491843E14A50D0
:10E3300041E10101E39B199ED190FF0E05014B5D68
:10E3400004E04BC507F04B6912000101E5A503D0BD
:10E35000E59509EC19F00101E551080B08E02050A2
:10E36000400B05E1120E72ECCAF00101E59734ACE6
:10E370000AD044EC20F0010802E1520E01D0500E08
:10E380002CECCAF0349C20B013D0EFECD2F002E0B9
:10E39000006A73DB2196020168510AE13250010BD9
:10E3A00007E12C50800B04E12C50400B01E11F864B
:10E3B000072A120063ECD1F001E00FD24A5001E0CD
:10E3C0000CD220A0229CA4EC14F0FF0801E005D19F
:10E3D0002050200B01E101D11850800B01E0FDD04D
:10E3E0000201766B76C2B1F1199291ECCDF0349CBA
:10E3F0001C901E50010B06E01D50040B03E01D5045
:10E40000080B0DE100500BE01F50020B08E06CDF21
:10E41000000905E0258E1F0E7EECCAF0DED01E50EE
:10E42000010B18E1005006E01F50020B13E15CDF06
:10E43000000910E00101010EB16F1982076A0B0E8D
:10E44000086E005003E148DF000901E01C80005025
:10E450002CE12DD01D50040B03E01D50080B29E1C9
:10E4600000500CE0EFECD2F009E11F50020B21E16B
:10E47000E9ECCAF003E138DF00091BE01DB402D06B
:10E48000110E05D01DB604D00201516B140E076E9B
:10E49000005003E121DF000901E01C80005007E08B
:10E4A00019ECCCF002E1DBDE98D0EFDE96D0F7DE9F
:10E4B00094D0050110511EE027AA12D0005003E0AD
:10E4C000E9ECCAF010E0005003E106DF000901E0CA
:10E4D0001C80005001E1E3DEE9ECCAF001E0BFDEA0
:10E4E0001E0E076E7AD0258E8A0E98ECCEF0AAEC1E
:10E4F00021F073D020AE05D0076A0A0E086E1C808A
:10E500006CD0005051E01EECCDF006E02050040B22
:10E5100003E11E50020B48E00201195114E01E50A5
:10E52000020B07E1EAEC08F000090DE11EECCDF06A
:10E530000AE10201376B386B196B19C255F217ECFF
:10E540000BF04DEC65F013ECCBF00AE01EECCDF0D7
:10E55000FDE0EEECD0F0FAE120941E928CEF04F096
:10E560001C80AFECD0F013E01950400B10E01950B4
:10E57000040B0DE020A40AD01994050EE66ED00E0F
:10E58000E66EE80E0C24ECECC9F001D01C901CA047
:10E5900024D0000E02012A6F0701A36F0B6E1E929A
:10E5A000076A0B0E086E19D0005017E12050010BBE
:10E5B00014E11EECCDF003E02050040B0EE001014D
:10E5C000E3938CEC04F013ECCBF005E01EECCDF003
:10E5D000FDE0209412001C8030DE2050200B04E16E
:10E5E000BAEC0BF0000903E1020134514DE060EC9C
:10E5F000CCF04AE00501106B20902094810E076E4C
:10E6000005EC05F0000906E10D0EE66EE30EE66E80
:10E61000010E0DD01EECCDF002E11B0E12D0EEEC7F
:10E62000D0F00AE0050EE66EE30EE66E010E10EC89
:10E63000DAF0E552E55208D0BAEC0BF0000905E03B
:10E640001A0EE66ED5EC26F0E552BAEC0BF0000996
:10E6500019E0ACC134F205EC05F0000905E1010157
:10E66000806BD9EC04F00ED0EEECD0F00BE0FFECB8
:10E67000D4F003E001013C9D02D001013B9FEAEC94
:10E6800018F01490E2EC07F063ECD1F001E14A508D
:10E6900042E08CEC04F00201D95102E0E7EC08F012
:10E6A0000201D85102E081EC48F027AA28D075EC8D
:10E6B000E2F002012A6B2FAA02D0EBEC4EF030A45C
:10E6C00002D099EC51F030AC02D018EC50F024A0FC
:10E6D00002D044EC4FF032A002D099EC4FF023AEC0
:10E6E00002D07EEC4EF01FA802D0F1EC0FF02C50BF
:10E6F000800B03E12C50400B02E04CEC0EF0259A0D
:10E700001AAC02D0D0EC09F028A203D02892D6ECA3
:10E7100039F01C8C12002050010B14E002012D5125
:10E7200011E11750800B06E03CECD2F009E00B0E33
:10E73000155C06E02050040B05E11EECCDF002E074
:10E740007FEF71F002012A5104E013ECD0F01BECD2
:10E75000CEF017AE5BD04BEC97F080ECCBF017E02F
:10E760002F50200B14E13050040B11E12350800B8B
:10E770000EE13050400B0BE12450010B08E1325008
:10E78000010B05E13250020B02E181EC2EF03292D6
:10E790001FAA3CD01F9A01013BAB38D016ECCFF03A
:10E7A0000201315110E1CEEC34F0190E155C14E188
:10E7B0001750010B11E00101D451D55D0DE10201AB
:10E7C000C80E316F1200316B1C0EE66E2BECE2F0BE
:10E7D000E5520101960EAC6F12001FECCEF016E16F
:10E7E0004A5014E121BA12D0D3EC07F0000902E13B
:10E7F000A8ECD4F00EEC0DF0238A810E076ED3EC5A
:10E8000007F0000903E081EC2EF0258212000C04D1
:10E81000040F0701006F12000101B59B19AC27D04E
:10E8200017EC0BF0138225A41CD07CECDBF0FD0E62
:10E83000E66EE20EE66E010E72ECD7F06EECDFF0E3
:10E84000E30E0C242CECCAF024EC0BF07CECDBF097
:10E85000F50EE66EE20EE66E010E72ECD7F06EEC8F
:10E86000DFF002010E0E376F060E386F1200CFDF99
:10E870000701FA0E036F016B026B0201536B546BBD
:10E880001D90120000C709F00201555104E0800EEE
:10E89000C9ECCAF01A800701035117E003510307BE
:10E8A000CBECCBF0CC0E005C10E0FF0E005C0DE07A
:10E8B000800E005C06E20050E66E3CEC04F0E5528F
:10E8C000006E0050C9ECCAF0E6D7096A12005CEC91
:10E8D000DAF0DBCF55F22F88006A2388BFEC26F0F0
:10E8E0000101320EAC6F17A802D00201558F020150
:10E8F000195102E0010E196F179EC2EFC9F017A857
:10E9000002D011EC48F019AC24D017EC0BF01392A4
:10E9100063ECD7F0D00ED8800E54050E0F5405E2EC
:10E9200053EC65F00201196B120013820101E683BA
:10E93000218EF9EC0AF0198AEAEC08F000090FE1DF
:10E9400020840101E4991EECCDF009E00101E48985
:10E950001200278A02012D5102E0010E2D6F1200D4
:10E96000C6ECC9F0198C83ECCAF003E0E9ECCAF0FC
:10E9700001E0199C25A410D0FE0EDB500C6E4CDF7C
:10E9800025940101B587239C24B2238C248219ACE1
:10E9900032D0198428802FD01950400B0EE0EAECB9
:10E9A00008F000090AE01EECCDF007E02050040B4F
:10E9B00004E11D0E7EECCAF01ED0FD0EDB500DE111
:10E9C0000201195103E12750400B07E079ECD5F023
:10E9D0007EDFE5520201196B0ED0FE0EDB500C6E8D
:10E9E0001BDF19BC07D04EDF0501105103E153ECCA
:10E9F00065F001D084DFC2EFC9F00601060E406F5A
:10EA000052ECCEF004E2A85102E00601402B0201D4
:10EA10001E0E276F120001012951E8240301B86F6F
:10EA20000A01190ED76F360ED66F0101D45103E0DB
:10EA3000030ED45D03E10A01080ED66F30ECD2F06C
:10EA400003E10A013C0ED66F0A01DA8FD46B3484DD
:10EA500052EFCCF0C6ECC9F064EC39F056EC19F08A
:10EA6000338879ECD5F051EC1BF0E552C2EFC9F0D8
:10EA7000010EE66EEFDFE5521200000403E1CAEC7E
:10EA8000D7F01BD0005045E0030E005C18E1CAEC43
:10EA9000D7F0A4ECD0F004E0E80E0E6E030E0F6E7B
:10EAA0008DECCDF004E06AEC04F097ECCAF09CEC3D
:10EAB000CAF003E1640E0E6E0F6A5BEFD9F00EEC44
:10EAC00015F0930E0E6E020E0F6E0050030819E241
:10EAD000700E0E6E030E0F6E050E005C04E1930EB9
:10EAE0000E6E020E0F6E060E005C04E1970E0E6EA7
:10EAF000040E0F6E070E005C04E1200E0E6E060E73
:10EB00000F6E5BECD9F0020E005C05E1500EF1ECEB
:10EB1000C9F0D0EF0AF00050030803E20201040E2E
:10EB2000356F070E005C03E10201080E356F12001D
:10EB3000C6ECC9F0280EE8ECD5F0290E72ECCAF04C
:10EB4000C2EFC9F0D9CFE6FFE1CFD9FFE6528C9EE4
:10EB500000000000000000008C9600000000060E7F
:10EB6000E66E8DEC5CF0E5528C8600000000000043
:10EB70008C9600000000D80EE66E8DEC5CF0E5523D
:10EB8000A5C7E6FF8DEC5CF0E552E66A8DEC5CF023
:10EB9000E552E66A8DEC5CF0E5528C868C8EDF6A7D
:10EBA0001E0EDF5C07E2640EE66E95EC21F0E55286
:10EBB000DF2AF6D7E552E552E7CFD9FF1200D9CFC9
:10EBC000E6FFE1CFD9FF8C9E0000000000000000AE
:10EBD0008C9600000000030EE66E8DEC5CF0E552B2
:10EBE000A5C7E6FF8DEC5CF0E552FC0EDBCFE6FF3F
:10EBF0008DEC5CF0E552FB0EDBCFE6FF8DEC5CF0BC
:10EC0000E552FA0EDBCFF3FFDB06F35000090FE00D
:10EC1000B5ECFDF0006EFD0EDBCFE9FFDB2AFE0E4A
:10EC2000DBCFEAFF01E3DB2A00C0EFFFEAD70000F9
:10EC30008C86C69E8C8EE552E7CFD9FF120047EC3A
:10EC4000D5F0DF6ADF2AFA0EDBCFE6FF1AECD0F050
:10EC5000FDECCDF021ECD0F0FA0EDBCFE6FF1AECA4
:10EC6000D0F0A80EE66E030EE66E21ECD0F0010E99
:10EC7000DB6AFA0EDB5044ECCCF017E2010EDB50FD
:10EC8000E76E25ECD0F0E75060ECD6F0EFCF49F01E
:10EC9000010EDB50EA6AA80FE96E030EEA22EF507C
:10ECA000495C03E1010EDB2AE4D78DECD3F002E0EE
:10ECB000FCEC0CF08DECD3F003E00A0EDF5CC2E359
:10ECC0000A0EDF5C02E3000E01D0010EDBECD2F095
:10ECD00002E2E16AE552E16E4950C2EFC9F0D9CFD4
:10ECE000E6FFE1CFD9FF8C9E00000000000000008D
:10ECF0008C9600000000060EE66E8DEC5CF0E5528E
:10ED00008C860000000000008C9600000000020EBF
:10ED1000E66E8DEC5CF0E552A5C7E6FF8DEC5CF08D
:10ED2000E552FE0EDBCFE6FF8DEC5CF0E552FD0E0A
:10ED3000DBCFE6FF8DEC5CF0E552FA0EDBCFF3FFA4
:10ED4000DB06F350000911E0FB0EDBCFE9FFDB2A05
:10ED5000FC0EDBCFEAFF01E3DB2AEF50006E005030
:10ED6000E66E8DEC5CF0E552E8D700008C86C69E1E
:10ED70008C8E050EE66E95EC21F0E552E552E7CF5C
:10ED8000D9FF1200D9CFE6FFE1CFD9FFE652B9ECA7
:10ED90005CF00101640EAC6F0400CCEC41F0020E9B
:10EDA00007015A5D0FE00701945109E0B3EC05F04B
:10EDB0000401FD6FFDC4E6FFD6EC05F0E552E0EC82
:10EDC000A7F071D0070194516EE007019451496E8C
:10EDD0004A6A4A3404E24950C008000E4A5408E224
:10EDE0000701040E266F270EE66E65EC14F0E5525F
:10EDF000B3EC05F00401FD6F3B0E0401FD5D0CE179
:10EE000004013B0EFE6F0601C46B309A0101379B73
:10EE10007BEC0CF007015A6B610E0401FD5D07E30A
:10EE20000401FD51660803E3200E0401FD5F300E6E
:10EE30000401FD5D22E30401FD5146081EE30601C5
:10EE4000C42B410E0401FD5D04E2300E0401FD5FA0
:10EE500006D0410E0401FD5D0A0F0401FD6F020E94
:10EE60000601C45D08E10601C339F00B0401FD256C
:10EE70000401FD6F02D0FDC4C3F6020E0601C45D9D
:10EE800011E1FDC4E6FFD6EC0CF0E552006E010E78
:10EE9000E66E95EC21F0E5520601C46B0050E66E7B
:10EEA00047DEE5528FD70201685102E054EC8EF044
:10EEB0001C9C100E075C03E2C8EC6BF024D01E0E05
:10EEC000075C03E243EC70F01ED00750496E4A6ABB
:10EED000D8904A5004E6800E495C000E4A5803E27E
:10EEE000D5EC21F010D00750496E4A6AD8904A50AC
:10EEF00004E6920E495C000E4A5803E292EC71F06F
:10EF000002D080EC2DF01CBCD3D78BEC53F0095011
:10EF100008E00701070E266F270EE66E65EC14F079
:10EF2000E55222A228D022922E98329A9CEC80F0B0
:10EF3000DF682E50100B15E0010101012A51040B6E
:10EF400010E12950020B0DE1DF500BE00D5002E102
:10EF5000010E0D6E2E980FEC8EF09CEC80F0DF060B
:10EF6000E8D7DF5008E10701050E266F270EE66E91
:10EF700065EC14F0E55210D7E552E552E7CFD9FF22
:10EF800012000101E6A507D0D40501E1020C020E32
:10EF9000D45D01E1010CD4511200080E016E010193
:10EFA000D45102E1180E016E380EB95D09E1016A13
:10EFB00095EC0BF0000902E0100E016EFFEC18F06A
:10EFC0001200200EE66E640EE66E070EE66E800EF0
:10EFD00064EFD6F088ECD6F05BECCFF0EFCFDFFF3C
:10EFE000FF0EDF5C02E1100EDF6EDF50E552C2EF74
:10EFF000C9F0D3DF03015E510126015049ECD4F082
:10F00000046E120016ECCFF00101040E016F0450E3
:10F01000006E00500F0803E2100E005E04D0100EC8
:10F02000D8800054006E7EECE1F00101200E1A6FD2
:10F03000050E006E300E1B5D02E0040E006E0450E3
:10F040000F0805E2005068ECCBF02B0E04D0005006
:10F0500068ECCBF02D0EEF6E010E016F300E496E95
:10F06000F40E4A6E010E4B6E5EC34CF04D6A4E6A52
:10F070002FECD5F000ECD6F00101188F12001D0E18
:10F080000101B95D01E1010C000C43ECD5F0005029
:10F09000EF085CE2F00E005CDF6EDF50080862E310
:10F0A0002950010B05E10401F95102E1FA5108E090
:10F0B0000101E4910201246B3C6BE0ECA7F0F0D776
:10F0C00016ECCFF0A8ECD0F0DF50FE0BE842750F45
:10F0D000096E016ADFA002D0800E016E026A070E7F
:10F0E000025C0CE237EC3BF0005008E0FF0E005CE5
:10F0F00005E00FECE2F0012A022AF1D76EECDFF016
:10F100000101E485080E016EDFA002D0800E012609
:10F11000026A780E025C10E237EC3BF000500CE023
:10F12000FF0E005C09E00050036EE66ED6EC05F0C1
:10F13000E552012A022AEDD73B0E035C05E03B0EA7
:10F14000E66ED6EC05F0E552096A16D094ECD3F0E1
:10F15000005054ECD5F0056EFF0E055C05E16C0E19
:10F16000DFECCAF0258E08D0B9C157F205C0B9F15D
:10F1700029820201010E686FE552C2EFC9F01D0E2F
:10F180000101B95D04E1F00E03015D2513D00068B3
:10F19000016A015061ECCAF004E6960E495C000E6B
:10F1A0004A580CE294ECD3F0015054ECD5F0B95D20
:10F1B00003E10150006E1200012AEBD71200020E8B
:10F1C000016E2AC100F0F9EC3AF02F0E016E57C122
:10F1D00000F0F9EC3AF0370E016E5FC100F0F9EC87
:10F1E0003AF00F0E016E37C100F0F9EC3AF0100E54
:10F1F000016E38C100F0F9EC3AF02E0E016E56C1E6
:10F2000000F0F9EC3AF0620E016E8AC100F0F9EC00
:10F210003AF0650E016E8DC100F0F9EC3AF0660E21
:10F22000016E8EC100F0F9EC3AF06E0E016E96C1DF
:10F2300000F0F9EC3AF06E0E016E97C100F0F9EFB4
:10F240003AF0130E016E3BC100F0F9EF3AF03F0EB9
:10F250000101B95D02E119A6D17B0A0EB95D05E194
:10F2600019B603D05F77E2EC35F0170E0101B95DF6
:10F2700014E119A63B79B0EC1EF081EC2EF0E7EC1E
:10F28000D2F004E02150020B01E1E8893BB903D040
:10F290001E9A52ECCCF0050147873E0E0101B95D84
:10F2A00009E119B607D0020E425D02E1010E01D05C
:10F2B000020E426F050EB95D03E0060EB95D11E165
:10F2C00019B608D0050EB95D03E10701BE7102D081
:10F2D0000701BE7302ECD2F088EC09F0020107814D
:10F2E0002D84290E0101B95D04E119A677718BEC1B
:10F2F00020F0220E0101B95D02E119A68D79100EF0
:10F30000B95D04E119A63E7164EC5CF0280E0101C0
:10F31000B95D0AE119A6387575ECD4F001E0098FE2
:10F320009DECC4F0D6EC39F0110E0101B95D02E19B
:10F3300019A6D27B190EB95D02E119A6387F090E14
:10F34000B95D02E119A6967DB95104E119A633749D
:10F350001CEC1FF0320E0101B95D02E119A62A75FD
:10F360002D0EB95D02E119A62A731B0EB95D01E1EC
:10F370002E74300EB95D01E12E72400EB95D02E1CE
:10F3800019A63771130EB95D02E119A62A7F2F0E57
:10F39000B95D0CE119B608D05F9FF10EE66EE20E82
:10F3A000E66E010EF6ECC9F08BEC20F0120043EC97
:10F3B000D5F025ECD0F0EFCFDFFFFB0EDB50D8808F
:10F3C000DF5403E2FB0EDB50DF6EFC0EDB50DF5C34
:10F3D00003E2FC0EDB50DF6E0DAE0CD0FC0EDB50FA
:10F3E000D880DF5402E2DF0605D032B603D0FB0E30
:10F3F000DB50DF6E0D040BE1FB0EDB50DF5C02E245
:10F40000DF2A05D032B603D0FC0EDB50DF6E25ECD0
:10F41000D0F0DFCFEFFFE552C2EFC9F095ECD7F0A7
:10F420002CECD0F0C2EFC9F0C6ECC9F032861AEC71
:10F43000D0F0FDECCDF02CECD0F03296C2EFC9F05C
:10F4400095ECD7F064ECDBF0C2EFC9F0500E036E20
:10F45000E4ECD5F005E01B50080B02E11E0E036E34
:10F46000120043ECD5F0F3DE310E0101B95D2AE163
:10F470003651070B006E0D040EE136BF02D0368FF9
:10F480001AD036BD03D0368D006A15D0070E005C49
:10F4900012E2002A10D0FF0E0D5C0DE1005005E0D5
:10F4A000000600AE08D0006A02D036AD02D0369D0C
:10F4B00002D036BF369F0050070BF36EF80E36159C
:10F4C000F310366F1F0EB95D13E10D0408E156B15C
:10F4D00002D056810DD056B50BD0568509D0FF0EFF
:10F4E0000D5C06E156A502D0569502D056B1569154
:10F4F0000D0EB95D0AE1150E57ECDBF0550EE66E08
:10F50000010E04ECCAF08CEC04F00E0E0101B95DA2
:10F5100008E1050EE66E830EE66E010EFFECC9F003
:10F52000339C0C0E0101B95D15E1020EE66E840EEE
:10F53000E66E010EFFECC9F0300E010184250401D6
:10F54000F76F020E0101845D03E10401340EF76FD1
:10F55000A5ECA7F0230E0101B95D13E1030ED01550
:10F56000066F065102E1010E066F030EFFECDAF0A2
:10F57000FC0E0101D0170651D0138BEC20F00501D1
:10F5800047892C0E0101B95D07E119A6D2711E9AB7
:10F5900052ECCCF081EC2EF0120E0101B95D2EE19F
:10F5A0000D0411E1080E505D02E10D0E26D0050E8E
:10F5B000505D1EE0030E505D16E050050FE00D0E8D
:10F5C000505D1CE006D0FF0E0D5C18E1030E505D8F
:10F5D00002E1010E12D0050E505D02E1030E0DD0C6
:10F5E000080E505D02E1050E08D00D0E505D02E1DF
:10F5F000080E03D0500502E0010E506F240EB95DD5
:10F600002DE1E7AB03D0E3EC0BF028D0640E006EE5
:10F610000701BEAB02D00A0E006E0D0409E1000125
:10F62000005001016927000E6A236B236C2310D060
:10F63000FF0E0D5C0DE14FECDAF04B6A4C6A49505D
:10F640000101695F4A506A5B4B506B5B4C506C5BCD
:10F6500074ECC7F024843388D6EC39F0140E010121
:10F66000B95D0BE1030E4F15066F020E9CECDAF04C
:10F67000FC0E01014F1706514F13150EB95D11E134
:10F68000300E4F15066F06390F0B066F020E9CECFD
:10F69000DAF001010639F00B066FCF0E4F17065155
:10F6A0004F130F0EB95D09E1820EE66E520EE66E43
:10F6B000510EE66E010E04ECCAF03D0E0101B95D7B
:10F6C00019E10701BE51E840E8403F0B0101066F18
:10F6D000030E06179CECDAF00101040E0603F3CFCB
:10F6E00006F1F30E0701BE17010106510701BE1313
:10F6F00088EC09F0430E0101B95D13E1E6A508D0DD
:10F70000B40EE66E640EE66E4A0EE66E010E07D08B
:10F71000730EE66E460EE66E520EE66E010E04ECB9
:10F72000CAF0FFECD2F036E12050040B03E11B508D
:10F73000080B30E00D0414E12B50040B02E0140E12
:10F7400001D0010E496E4A6A49BE4A682250040B34
:10F7500001E0010E7EECCDF04950EE264A50ED223C
:10F76000FF0E0D5C14E12B50040B02E0140E01D0CF
:10F77000010E496E4A6A49BE4A682250040B01E0F4
:10F78000010E7EECCDF04950EE5E4A50ED5AB7ECDA
:10F7900015F01E88350E0101B95D07E1D30EE66E46
:10F7A000D30EE66E010ED1ECCDF03A0E0101B95D3B
:10F7B00029E133A60BD0AB0EE66ED30EE66E010E3A
:10F7C000E66EE3EC26F0E552E55218D02B510A081C
:10F7D00017E3E6ECC2F0E66E3CEC13F0E55264ECA5
:10F7E000CBF00EE100C006F1DC0EFFECDAF006C152
:10F7F00000F0F9EC3AF0E66A88EC1CF0E55202D031
:10F80000E3EC0BF0180E0101B95D20E1E3AD12D07D
:10F810000C0EE66E030EE66EEBECD4F004E1950EF2
:10F82000496E010E03D0930E496E010E4A6E32EC02
:10F83000CBF008D0780EE66E280EE66E870EE66EE8
:10F84000010EE66E64ECDBF01DEC09F0250E010103
:10F85000B95D07E1FA0EE66E880EE66E020EFFEC69
:10F86000C9F01A0E0101B95D07E1020EE66E700ED5
:10F87000E66E020EFFECC9F0210E0101B95D1CE13C
:10F88000020EE66E390EE66E010EFFECC9F00101C4
:10F89000395104E10DECDAF056EC25F061ECCFF0D3
:10F8A000006A0101395102E0010E006E00C0D4F27D
:10F8B00000C0D3F200C0EBF9B90507E1050EE66E12
:10F8C000940EE66E010EFFECC9F00B0E0101B95D5E
:10F8D00001E085D039512CE030A227D00901E85150
:10F8E00004E10D0401E079D016D0E80511E10D0422
:10F8F00008E1010EE86FE50EE66EE20EE66E010E1F
:10F9000011D0E86BDF0EE66EE20EE66E010E0AD055
:10F91000FF0E0D5C62E1010EE86FEB0EE66EE20E8B
:10F92000E66E010E27ECCAF058D0E3EC0BF057D08E
:10F930001E862950020B0AE03A5108E03A510108AC
:10F9400002E2010E01D0020E3A6F07D0130EE66EEE
:10F950003A0EE66E010EFFECC9F06EEC09F0010103
:10F960003A5102E08D8303D03A5101E18D93030EA9
:10F970003A5D33E33A51130830E3000E036E026E32
:10F98000016E030E3A5D006E080E005C0BE2010E84
:10F9900000C0E7FFE75204E0E846FE0BE706FCE1A3
:10F9A000016E12D0100E005C0CE2080E005C496E75
:10F9B000010E495204E0E846FE0B4906FCE1026EE6
:10F9C00003D0100E005C036E010EE66E0350E66E6F
:10F9D000F9ECD9F0E4ECCDF002D07EECBDF0030EF2
:10F9E0000101B95D0AE11E0E57ECDBF0700EE66E08
:10F9F000010E04ECCAF01AEC1FF0070E0101B95D0C
:10FA000051E1E95109E1080EE66E040EE66E470E7B
:10FA1000E66E010E04ECCAF00101E90508E1E668B2
:10FA2000C80EE66E7D0EE66E010E04ECCAF0020E04
:10FA30000101E95D08E1C80EE66EE66A4B0EE66E6E
:10FA4000010E04ECCAF0030E0101E95D14E10701A7
:10FA5000BEA308D0960EE66E780EE66E4D0EE66EEC
:10FA6000010E07D0320EE66E0A0EE66E4C0EE66E02
:10FA7000010E04ECCAF0040E0101E95D09E10F0E6C
:10FA8000E66E0A0EE66E410EE66E010E04ECCAF05A
:10FA9000050E0101E95D04E119A662732AEC1EF06E
:10FAA0001AEC1FF02A0E0101B95D39E1016AD45147
:10FAB00002E0010E016E020E0901E55D1BE155EC4D
:10FAC000D6F00AE1E2ECD6F004E6E20E495C000E64
:10FAD0004A5802E2190E0026FF0E0D5C05E10050A7
:10FAE000180802E2190E005E015066ECCAF000C070
:10FAF000EFFF13D0020EE55D10E2FA0E57ECDBF0DB
:10FB00000150030D0CECCDF0B80E4B26020E4C222A
:10FB1000E5519DECD7F064ECDBF03CEC4EF0340E9C
:10FB20000101B95D07E1640EE66E850EE66E010E19
:10FB3000FFECC9F0040E0101B95D09E1020EE66EA9
:10FB4000310EE66E010EFFECC9F0B0EC1EF0370E80
:10FB50000101B95D10E12B510A0806E20F0EE66EB5
:10FB60007B0EE66E010E05D00F0EE66E860EE66E7B
:10FB7000010EFFECC9F03B0E0101B95D0CE1FFEC99
:10FB800018F0190EE66EE66A7A0EE66E010E04ECC7
:10FB9000CAF082EC15F0390E0101B95D0BE1280EB7
:10FBA000E66E1E0EE66E890EE66E010E04ECCAF0DD
:10FBB00012ECD3F0410E0101B95D09E13C0EE66E95
:10FBC0006E0EE66E010EFFECC9F0EAEC18F0420E84
:10FBD0000101B95D09E13C0EE66E6F0EE66E010EA5
:10FBE000FFECC9F0EAEC18F0330E0101B95D28E131
:10FBF00081C306F13B0E016E03017F5104E180C316
:10FC000006F1170E016E020E7F5D02E182C306F15E
:10FC10000150C9ECD5F0F8ECCCF003017F5102E1C2
:10FC200006C180F37F0502E106C181F3020E7F5D0C
:10FC300002E106C182F30101835102E080ECE3F0AE
:10FC4000080E0101B95D16E103017F5107E1170EAE
:10FC5000E66E830EE66E030EF8ECCCF003017F0532
:10FC600007E13B0EE66E840EE66E030EF8ECCCF078
:10FC700089ECE3F0020E0101B95D0EE11B50080BA7
:10FC800002E0060E01D0050EE66E800EE66E010E55
:10FC9000FFECC9F0D9EC04F017ECD5F02CE1016AC7
:10FCA000D5CA03F0D251010B12E03751080B0FE017
:10FCB000040E036E1BA00BD0030E036E010E016E2B
:10FCC0000A011C5104E1280E216F21CA1CFAFE0E04
:10FCD0004EECCEF005011751050D0CECCDF0140ED5
:10FCE0004B260A0E4C2203509DECD7F02CECD0F0A2
:10FCF00024847CEC0DF03C0E0101B95D0FE1FA0E9D
:10FD0000E66E2250040B01E0010E4A6A910F496E23
:10FD1000020E86ECD7F0B7EC15F01E88270E010115
:10FD2000B95D03E0380EB95D1BE1030ED45D03E15C
:10FD3000E3EC0BF015D00BECD5F0F9EC77F004C048
:10FD400006F1200E9CECDAF001505BECCFF006C11E
:10FD5000EFFF308E06C104F002EC78F022EC1EF0CA
:10FD60001E0E0101B95D06E119B602D002017879D3
:10FD7000ACEC15F0260E0101B95D09E1030EE66E4B
:10FD8000430EE66E010EFFECC9F05DEC21F01C0E97
:10FD90000101B95D0FE13EC1DFFF188C3E6B070E1C
:10FDA000E66E3F0EE66E010EFFECC9F0ACECD4F04F
:10FDB000DFCF3EF1200E0101B95D02E10D50332786
:10FDC000160EB95D09E10C0EE66E070EE66E3D0EED
:10FDD000E66E010E04ECCAF05CC3E6FF31EC0CF0F9
:10FDE000E552440E0101B95D14E119B611D03FECA2
:10FDF000DBF0040A01E0010E496EFAECC9F049504B
:10FE0000010BF36EF346F346FB0EEF14F310EF6EA7
:10FE10002E86450EB95D32E11DECD8F0016E15EC71
:10FE2000D7F0026E0D50022602AE0ED0630E026EA7
:10FE30000106015037ECCBF007E24950F908000EFB
:10FE40004A5402E2F90E016E0250630802E2026AAD
:10FE5000012A015037ECCBF006E24950F908000EB8
:10FE60004A5401E2016AFAECC9F0030E01C0EBFF4B
:10FE7000FAECC9F0020E02C0EBFF2E86460EB95D09
:10FE80001BE118ECD8F0016E0D50E824012601505A
:10FE90000A0802E20A0E016E080E015C02E1090E78
:10FEA000016E030E015C02E2030E016EFAECC9F072
:10FEB000010E01C0EBFF2E86480EB95D50E1A8ECA3
:10FEC000D9F0496E4A6AA3ECD9F00A0DF3504924DF
:10FED000DA6FF4504A20DB6FADECD9F002E106ECAA
:10FEE000D2F00D040CE1D890DB5104E6E70EDA5DA8
:10FEF000030EDB5911E2DA2B000EDB230DD0FF0ECF
:10FF00000D5C0AE1DB3504E3DA511908FC0EDB5520
:10FF100003E2DA07000EDB5B2888800EDB1503E0C6
:10FF2000289806ECD2F0DAC149F0DBC14AF00A0E9B
:10FF3000E0ECC9F0FAECC9F0040E49C0EBFFFAECB2
:10FF4000C9F0050E39C0EBFFFAECC9F02850100BD0
:10FF500002E0EF8001D0EF902E8681EC2EF0470E6C
:10FF60000101B95D3FE1FAECC9F0060EEB50006EFD
:10FF7000FAECC9F00490EF50020B01E004800D5040
:10FF80000026005006E10470048026EC7AF003504D
:10FF9000006E26EC7AF00350D880005404E204701E
:10FFA0000480010E006E91ECD6F001E00490048014
:10FFB000FAECC9F00450010B02E0EF8201D0EF929D
:10FFC000FAECC9F0060E00C0EBFF100E01012B5D2C
:10FFD00003015C5D06E100C048F14DECCCF05CC370
:10FFE00000F02E86490E0101B95D39E1049091ECD3
:10FFF000D6F001E00480FAECC9F0EF50016E0F0E6C
:020000040001F9
:100000000114006E01380F0B016E0D50012604A083
:100010000CD00150800803E2090E016E04900150DB
:1000200009080CE2090E016E09D0015002E1010E2F
:10003000016E0150090802E2016A04800138F00BE8
:10004000016E0150001249ECD9F0090E60ECD6F0B7
:100050000450010B02E0EF8E01D0EF9E2E86E55298
:10006000C2EFC9F05C0E0024C4ECD9F00101100EFF
:10007000136F145102E1100E146F120015ECD7F03B
:1000800056ECCEF01DECD8F0006E0101030E006FAF
:1000900061ECE1F0060EE66E030E67EFCFF069EC5F
:1000A000D5F00A0809E2FE0EDB50F00F006E00509A
:1000B0000DECCFF0E3DF23D0FE0EDB50006ED2DF7D
:1000C000020E4CECCAF00DE20101010E146F080E95
:1000D000156FFE0EDB040DE1030E146F050E156F98
:1000E00008D013C112F114C113F115C114F10101AB
:1000F000156B07ECD5F002E1090E156F158FC2EFF5
:10010000C9F0E6EC25F02E801200140E006E04A05B
:1001100002D0110E006E81EF80F00E0E006E04A072
:1001200002D0080E006E81EF80F0A4EC11F0D0C771
:10013000F3FFD1C7F4FF120095ECD6F00101B551E1
:10014000800B04E02F50100B01E1E3D07CECDBF0DE
:1001500025EC8DF0010139510DE00B0EB95D0AE17E
:10016000016BD70EE66EE20EE66E010E72ECD7F072
:100170000101198F0A0EB95D01E1198F070EB95DF2
:1001800049E1040E016F2A0E196FE95108E1D30EFF
:10019000E66EE20EE66E010EE66E5DECCAF001015F
:1001A000E90508E1CF0EE66EE20EE66E010EE66EA0
:1001B0005DECCAF0020E0101E95D08E1CB0EE66ECE
:1001C000E20EE66E010EE66E5DECCAF0030E010172
:1001D000E95D08E1C70EE66EE20EE66E010EE66E20
:1001E0005DECCAF0040E0101E95D08E1C30EE66EA4
:1001F000E20EE66E010EE66E5DECCAF0050E010140
:10020000E95D08E1BF0EE66EE20EE66E010EE66EF7
:100210005DECCAF02A0E0101B95D0FE1420E1C6FC0
:100220000901E50503E10101440E1C6F020E0901FD
:10023000E55D03E101014D0E1C6F350E0101B95D55
:1002400011E10201B0510EE07CECDBF0B80EE66E7D
:10025000E20EE66E010E72ECD7F02CA203D0010183
:10026000370E1B6F17ECD5F007E13751080B04E090
:100270004C0E1B6F2A0E1C6F240EB95D0CE196A369
:1002800002D0230E07D057A906D02A0E196F57BBEC
:1002900002D03F0E196F1FA805D07CECDBF0006A7E
:1002A000FBEC25F0C0EC63F0000905E0310E030122
:1002B0005C250101186F1D0E0101B95D05E1310ECC
:1002C00003015D2501011C6F270EB95D03E0380EA7
:1002D000B95D05E1310E03015E2501011C6F430E7E
:1002E000B95D0CE1E651040B09E0016BB00EE66E5E
:1002F000E20EE66E010EE66E5DECCAF0180E01012C
:10030000B95D07E1E351400B04E0500E166F4C0E4F
:10031000176F6CECDBF059ECD8F00E0E136F146F06
:100320003FEC78F0000907E00101006B280EE66E53
:1003300005ECE2F0E552016A410E0101B95D08E108
:100340006EC100F0016802016E0EA46F010EA56F70
:10035000420E0101B95D08E16FC100F001680201C0
:100360006F0EA46F010EA56F200E0101B95D08E1AB
:100370000201330EA46F010EA56F33C100F00168B6
:10038000160E0101B95D0BE1050E3D03F350410F5F
:10039000006E016802013D0EA46F010EA56F1C0ED8
:1003A0000101B95D08E13F29006E016802013F0EBD
:1003B000A46F010EA56F180E0101B95D26E18751EA
:1003C000FE0BE842006E0201870EA46F010EA56FBE
:1003D0000101E3AD18D093C100F00201930EA46FA8
:1003E000010EA56F330E875D0AE101019551FE0BE9
:1003F000E842006E0201950EA46F010EA56F050E76
:100400000002F3CF00F001682E88070E0101B95DEC
:1004100065E1E95106E10201470EA46F010E1FECF0
:10042000CBF00101E90506E102017D0EA46F010E8A
:100430001FECCBF0020E0101E95D06E102014B0E5B
:10044000A46F010E1FECCBF0030E0101E95D1DE16D
:10045000006B0701BEA30CD0AC0EE66EE20EE66E9A
:10046000010EE7ECC9F002014D0EA46F010E0BD096
:10047000A80EE66EE20EE66E010EE7ECC9F0020190
:100480004C0EA46F010E1FECCBF0040E0101E95DD0
:1004900006E10201410EA46F010E1FECCBF00168D2
:1004A000050E0101E95D17E1016A62A306D0A40E01
:1004B000E66EE20EE66E010E05D0A00EE66EE20ECE
:1004C000E66E010EE7ECC9F00201620EA46F010EA8
:1004D000A56F020EA66F0101050E006F2A0EB95D11
:1004E0001CE1026AD45102E0010E026E0250030DBB
:1004F00007ECD6F0B80E4926020E4A220901E55152
:100500008FECD8F0020E0901E55D05E1190E11EC42
:10051000D6F0F6ECCDF001682E883D0E0101B95DF4
:100520000AE1D4C1E6FF15EC0DF0E5520168A3EC39
:10053000D1F00C0EA66F015002E061ECE1F0160E56
:100540000101B95D09E0180EB95D08E1E351400B06
:1005500005E0EBECD4F002E00101148F3D0E010147
:10056000B95D09E0180EB95D0CE1E351400B03E001
:10057000EBECD4F006E10101135102E1100E136F10
:10058000158F0D0E0101B95D20E1150E555D0BE1D2
:10059000006B970EE66EE20EE66E010EE66EFFEC65
:1005A000E1F0E5520BD0050E5503F35056ECCEF0BA
:1005B000060EE66E050EE66E33EC09F0E552E552E6
:1005C0000201550EA46F010EA56F3F0E0101B95D2A
:1005D00010E1D1AB02D0080E01D00E0E54ECCDF0DC
:1005E0002E800201D10EA46F010EA56F200EA66F02
:1005F0002E88050E0101B95D0DE10701BEB102D0E3
:100600000E0E01D0080E54ECCDF0A3ECD1F0010E8B
:10061000A66F2E80060E0101B95D17E10701BEB37A
:1006200006D0A80EE66EE20EE66E010E07D00101BE
:100630000007920EE66EE20EE66E010EE7ECC9F0E0
:10064000A3ECD1F0020EA66F2E800101B9052EE1B8
:100650000B0E54ECCDF00101945106E1010E006F38
:10066000440E006EE6EC25F001019451010819E2F8
:10067000006B890EE66EE20EE66E010EE7ECC9F045
:10068000050E0101945D02E1158F0BD0050E006F80
:100690009405190DF35056ECCEF00101100E136FB6
:1006A000148F0201940EA46F010EA56F110E0101AB
:1006B000B95D1EE12BC1E6FFF2DCE55212C10EF17D
:1006C00013C10FF114C110F115C111F10101100E88
:1006D000126F050E006FD2AB02D0290E01D02A0E88
:1006E000E66E05ECE2F0E552A9ECD1F0200EA66F23
:1006F0002C0E0101B95D1AE16EECCCF059ECD8F08A
:100700000B0E54ECCDF00101D2A10BD0050E006F01
:10071000850EE66EE20EE66E010EE7ECC9F0010111
:10072000158FA9ECD1F0010EA66F2E88230E0101C2
:10073000B95D20E16EECCCF00101030E006F7F0E7D
:10074000E66EE20EE66E010EE7ECC9F00101D05153
:10075000010B05E0D051020B02E0030E03D0D0A341
:1007600002D0020E126F0201D00EA46F010EA56F0F
:10077000030EA66FFFECD2F041E12250040B01E022
:10078000010E010F0E6F030E006F04902250040B38
:1007900001E0010E7EECCDF0EECF0EF0EDCF0FF0CC
:1007A0000CECD6F04B6A4B34000E4B1807E6D880A1
:1007B000F00E4954D80E4A54000E4B5403E235EC67
:1007C000D4F0048072EC26F00101100E116F04A029
:1007D00002D00E0E116F2BA402D0100E156F2250F6
:1007E000040B01E0010E020DF3CFF3F6F4CFF4F6A3
:1007F0008D0E0601F327020EF4232E88350E01011B
:10080000B95D01E019D124B80CD0006B84EC64F020
:1008100056ECCEF059ECD8F08DEC64F056ECCEF0FE
:100820000AD11BEC10F0F2ECCEF01BEC10F00E50E5
:100830000101D8270F50D923D8C10EF0D9C10FF02C
:10084000010E0F0B04E034ECD2F0E806FCE10701E6
:100850000E500C5D0F500D5905E20C510E5E0D51FE
:100860000F5A02D00E6A0F6A0EC00EF70FC00FF7B4
:100870000201B0511CE0190E11ECD6F0B0C23EF0EE
:10088000EFECD4F004E17EEC04F00201B16FB1C2F0
:1008900000F00101126B35ECD8F03CECFEF03EC0EC
:1008A00013F13AC014F10101110E156F138F84EC8E
:1008B00064F0026E006E2CA204D08DEC64F0026E27
:1008C000006E0201B05157E0960E0101D86FD96B4E
:1008D0001FA003D0F00ED86FD96BEBECD2F004E080
:1008E000320E0101D86FD96B0101D8510E5CD9517C
:1008F0000F5810E2E2ECD6F004E6F00E495C000E70
:100900004A5808E2002A640E0201B05D1DE2190E89
:10091000B0271AD00C0E4A6AD825496ED9514A22FE
:100920000BECD7F005E20050640802E200060CD0A0
:100930000201B05137ECCBF007E24950C808000E75
:100940004A5402E2C80EB06F0250005C73E02CB251
:1009500008D0E66A0050E66E96EC64F0E552E66E6A
:1009600007D00050E66EA6EC64F0E552E66EE66A4B
:100970003AECCEF05FD02CB244D084EC64F0496EF7
:10098000640E495C09E384EC64F04A6E4B6A4B34B4
:100990000DE215ECD2F00AE284EC64F00701266F58
:1009A000510EFFECCAF032EC8EF044D0E66AE66AF3
:1009B0003AECCEF00201FA0EB06F6FECD6F005E023
:1009C000D8900D330C33E806FBE18DEC64F0496EF2
:1009D000640E495C09E38DEC64F04A6E4B6A4B345B
:1009E00008E215ECD2F005E2A00EE66EA6EC64F08B
:1009F000E5528DEC64F0E66EE66A3AECCEF02C82BD
:100A000019D032EC8EF08DEC64F0496E640E495CC6
:100A100009E38DEC64F04A6E4B6A4B340AE215EC44
:100A2000D2F007E28DEC64F00701266F540EFFEC64
:100A3000CAF02C9225822E88390E0101B95D18E189
:100A4000020E006F080E006E8AB102D00E0E006E0C
:100A5000E6EC25F089C100F002ECCEF0100E136F29
:100A6000158F02018A0EA46F010EA56F010EA66FED
:100A7000120E0101B95D25E1156B15C114F1100EBF
:100A8000136F0D0E505D03E1010E146F17D0080EA9
:100A9000505D02E1050E09D0050E505D02E1030E26
:100AA00004D0030E505D03E1020E156F07D0500510
:100AB00005E1010E156F006FC8ECD9F00101158F2B
:100AC0002E883B0EB95D17E1020E006F080E006E16
:100AD0008AB302D00E0E006EE6EC25F07AC100F06B
:100AE00002ECCEF0100E136F02018A0EA46F010EFD
:100AF000A56F020EA66F370E0101B95D1BE1C1ECB7
:100B00006BF0050F56ECCEF0C1EC6BF0000904E180
:100B100003ECD3F0C8ECD9F00201860EA46F010EED
:100B2000A56F52ECCEF005E202017B0EA46F010E20
:100B3000A56F2E88030E0101B95D11E170C100F0AF
:100B400061ECE1F01E0E0101705D04E1010E006F29
:100B5000C8ECD9F00201700EA46F010EA56F340E1F
:100B60000101B95D11E1855104E10B0E54ECCDF0AA
:100B700006D085C100F061ECE1F00101158F0201A2
:100B8000850EA46F010EA56F040E0101B95D1FE172
:100B90000201310EA46F010EA56F0101040ECCEC11
:100BA000D9F00101310506E1020E006F9E0E006EC4
:100BB000E6EC25F0020E0101315D09E1020E006F45
:100BC000790EE66EE20EE66E010EE7ECC9F0250E38
:100BD0000101B95D11E102018851140D97ECCAF0D1
:100BE0006DECCFF00101100E116F006B328A020123
:100BF000880EA46F020EA56F270E0101B95D03E0F8
:100C0000380EB95D34E1CDEC77F0026A080E025C73
:100C10002EE20150022449ECD4F0006E100E005C6C
:100C200003E019ECCCF002E1020E13D000501208E0
:100C300002E2040E0ED00050100802E2030E09D0AA
:100C40000E0E005C02E2006A05D0100E005C02E2AB
:100C5000010E006E410E00247BECCBF0D00FE66E4F
:100C60000250E3ECCAF05CECCCF0022ACFD7130EB2
:100C70000101B95D0EE1100E146F14C113F1110ED4
:100C8000156F2ABF152B0201B0ECD4F0800EA66FB1
:100C90002E80430E0101B95D18E1050E006F52C1AF
:100CA00000F00201520EA46F010EA56F0101E6A52E
:100CB00007D04AC100F002014A0EA46F010EA56FD1
:100CC00061ECE1F00101148F2E883A0EB95D4AE122
:100CD000006B740EE66EE20EE66E010EE7ECC9F0F4
:100CE00033B603D001010E0E0E6F52ECCEF039E395
:100CF000050E006F64ECCBF003E13FECD4F01FD0A5
:100D00000101E49DB00E0D25CBECCBF00F0E005C85
:100D100003E3005030080DE2230E006E0901EB5191
:100D20000E0807E2310EEB5D04E2EBC900F00101B1
:100D3000E48D0101E4BD03D00050B4ECD5F061ECCA
:100D4000E1F00101135102E1100E136F64ECCBF0DE
:100D500008E00101158F240E136FE4AD02D0110ECF
:100D6000136F2E882E0E0101B95D09E15EEC09F0CA
:100D70009C0E0E5C630E0F5802E26DECCFF0D7ECC8
:100D8000D2F001E022D1006BE7ABF4D03BECD9F01C
:100D900048ECCAF03D5056ECCEF00101240E0E6F27
:100DA0009D0EFDECD7F00EC0DEFF0FC0DDFFC80EBC
:100DB000A0ECD0F004E3840E5FECD0F004E2070175
:100DC000080E02ECD7F06DECCFF00101100E116FA0
:100DD000160E126F95EC80F0F3CF57F0F4CF58F069
:100DE00057C0E6FF58C0E6FF47ECD2F0E7CF58F017
:100DF000E552E7CF57F05750F324556E5850F42082
:100E0000566E55C0E6FF56C0E6FF47ECD2F0E7CF7E
:100E100056F0E552E7CF55F05550F324536E565037
:100E2000F420546E53C0E6FF54C0E6FF47ECD2F006
:100E3000E7CF54F0E552E7CF53F05350F324516E0F
:100E40005450F420526E51C0E6FF52C0E6FF47EC0A
:100E5000D2F0E7CF52F0E552E7CF51F05150F324F2
:100E60004F6E5250F420506E4FC0E6FF50C0E6FF68
:100E700047ECD2F0E7CF50F0E552E7CF4FF093ECDC
:100E8000CFF047ECD2F0E7CF4EF0E552E7CF4DF090
:100E90009BECD3F058ECD4F047ECD2F0E7CF4CF019
:100EA000E552E7CF4BF04AECCBF0030E0F0B03E01B
:100EB00073ECD0F0FDE131ECD0F00101E7AD58D09A
:100EC0006C0EE66EE20EE66E010EF6ECC9F0020E56
:100ED000DBCFD8F1030EDBCFD9F101017F0ED88033
:100EE000D855050ED95505E20701090E02ECD7F0D9
:100EF0003FD021ECD4F0070E5BECD0F0FDE16A0EA0
:100F00004924096ED8C149F05DECD8F0FF0E005CB1
:100F10002EE1010EDB50ACECD0F0012ADF50ACEC3E
:100F2000D0F001012A0E1C6F670EE66EE20EE66E2F
:100F3000010E27ECCAF0020EDBCFE6FF030EDBCF7B
:100F4000E6FFB5ECD4F0630EE66EE20EE66E010E3F
:100F500027ECCAF0DECFE6FFDDCFE6FFB5ECD4F03C
:100F60005C0EE66EE20EE66E010E27ECCAF0096A30
:100F700025822AD069C11DF16AC11EF16BC11FF122
:100F80006CC120F10A0E22ECD8F01DC13BF01EC14D
:100F90003CF01FC13DF020C13EF011ECFDF03BC024
:100FA0001DF13CC01EF13DC01FF13EC020F19EEC82
:100FB000E1F0C8ECE1F00101118F148F0701BEBB15
:100FC00003D00101100E156F2E880490190E010137
:100FD000B95D06E138BF048061ECD9F0800EA66FE0
:100FE000100E0101B95D09E13E5101E00480FAEC07
:100FF000D0F03E0EA46F010EA56F090E0101B95D80
:101000000AE196BD0480FAECD0F0960EA46F010EB2
:10101000A56F400EA66F310E0101B95D22E136AD1C
:1010200015D06CECDBF0550EE66EE20EE66E010EAE
:10103000E7ECC9F001013651070B050DF3500A0F1B
:10104000006E35ECD8F0A2ECD3F004D036BF0480AB
:101050008DEC80F00201360EA46F010EA56FC70E55
:10106000A66F280E0101B95D06E138B5048061EC78
:10107000D9F0040EA66F400E0101B95D0AE137B147
:101080000480FAECD0F0370EA46F010EA56F010EAC
:10109000A66F0C0E0101B95D23E1845106E1050E36
:1010A000006F0B0E54ECCDF015D06CECDBF00101B1
:1010B000840506E14C0EE66EE20EE66E010E08D0E7
:1010C000020E845D07E1430EE66EE20EE66E010E4F
:1010D000E7ECC9F00201840EA46F010EA56F2E8803
:1010E000170E0101B95D13E1050E006F0E0E006EC3
:1010F0003BA904D04B0E006E040E006F02013B0EA4
:10110000A46F010EA56F100EA66F81EC80F01F0E6C
:101110000101B95D23E156A50BD0006B3A0EE66ED6
:10112000E20EE66E010EE7ECC9F00101148F0ED05D
:1011300056A108D0360EE66EE20EE66E010EE7EC22
:10114000C9F004D00E0E006EE6EC25F00201560E3A
:10115000A46F010EA56F050EA66F2E800101B95177
:1011600006E133B404808DEC80F02E88328A020EC2
:101170000101B95D4FE1006B2D0EE66EE20EE66EE9
:10118000010EE7ECC9F00101006B800507E1240EB8
:10119000E66EE20EE66E010EE7ECC9F0020E01010A
:1011A000805D07E11B0EE66EE20EE66E010EE7ECD7
:1011B000C9F0030E0101805D07E1120EE66EE20E3A
:1011C000E66E010EE7ECC9F0040E0101805D07E157
:1011D000090EE66EE20EE66E010EE7ECC9F0050EB2
:1011E0000101805D07E1000EE66EE20EE66E010E83
:1011F000E7ECC9F0060E0101805D07E1F70EE66E2F
:10120000E10EE66E010EE7ECC9F00201800EA46F5C
:10121000010EA56F0E0E0101B95D3FE1835106E19C
:10122000010E006F440E54ECCDF032D083050DE179
:10123000010E006FEF0EE66EE10EE66E010EE66E39
:10124000FFECE1F0E552E55206D033AC06D0010EDA
:10125000E66EB3ECE4F0E5521BD0030E006FE90E2E
:10126000E66EE10EE66E010EE7ECC9F001018305C2
:10127000040DF350006E35ECD8F03CECFEF03EC0AF
:1012800011F13AC012F10101115102E1100E116F7A
:101290000201830EA46F010EA56F2D0E0101B95D31
:1012A00012E10B0E006E04902AB3048004B004D047
:1012B000010E006F440E006E81EC80F00201B0EC74
:1012C000D4F0020EA66F2F0E0101B95D0DE10B0ED9
:1012D000006E5FAF02D0CF0E006E81EC80F0AFECFD
:1012E000D1F0800EA66F2E88320E0101B95D08E1A3
:1012F0002AB50480FAECD0F0B0ECD4F0040EA66F5E
:101300000101040E006F1E0EB95D0DE1050E006FA8
:10131000020178B90480FAECD0F0780EA46F020EC6
:10132000A56F100EA66F220E0101B95D17E18DA900
:1013300008D0050E006FA00EE66EE20EE66E010EFE
:1013400006D0006BE00EE66EE10EE66E010EE7ECF5
:10135000C9F0A9ECD1F0800EA66F2E801A0E010103
:10136000B95D3CE16CECDBF0110E0201702557EC2D
:10137000CCF001010E6F140E0201702557ECCCF079
:1013800001010F6F0E6A0F6A0201705103E1A8ECB0
:10139000CEF014D0700506E14CEC20F00101200ED7
:1013A000106F0CD0020E705D09E1BAECD4F00101AF
:1013B000395104E0EFC90EF0F0C90FF00E0ED880DD
:1013C0000E54270E0F5402E20E6A0F6A6DECCFF036
:1013D0000101115102E1100E116F148F0A0EB95D57
:1013E00019E1395103E0E3EC0BF014D0030E006F68
:1013F000DA0EE66EE10EE66E010EE7ECC9F00101D1
:101400005FA702D0020E156F328A2E80AFECD1F0AA
:10141000080EA66F0B0E0101B95D60E1395120E0A5
:1014200030A213D0040E006F0901E85102E12A0E28
:101430000FD0E80508E1D50EE66EE10EE66E010E6E
:10144000E7ECC9F008D04B0E03D0010E006F440E3C
:10145000006EE6EC25F00201E80EA46F090E3DD007
:1014600039ECBCF003ECD3F03A5102E1440E0CD05D
:101470003A0504E1040E006F2A0E06D0020E3A5D12
:1014800006E1040E006F4B0E54ECCDF020D0030E9D
:101490003A5D1DE33A5113081AE3550E54ECCDF0B2
:1014A000030E01013A5D006E080E005C04E21C0EA2
:1014B000146F00280BD0100E005C05E2130E146FA1
:1014C000070E005C03D0130E146F240E156F328AC2
:1014D0002E8002013A0EA46F010EA56F210E0101AC
:1014E000B95D17E1395102E10E0E03D0390504E16F
:1014F000080E54ECCDF008D0006BCC0EE66EE10E79
:10150000E66E010EE7ECC9F00201390EA46F010E80
:10151000A56F1B0E0101B95D3BE12EA435D0016A18
:101520001E0E015C0AE2A9ECD3F0EF50E66EB0ECBF
:10153000D3F05CECCCF0012AF3D77CECE2F0D0ECF9
:10154000E0F00101279D269D1750800B0CE1010161
:101550002651400B08E12751400B05E18BEC53F07D
:10156000CCEC41F0F1D7016A1E0E015C0AE2B0EC4E
:10157000D3F0EF50E66EA9ECD3F05CECCCF0012A8E
:10158000F3D7D0ECE0F00101050ECCECD9F0328AB3
:10159000300E0101B95D42E1050ECCECD9F02EA26E
:1015A0003BD003ECD3F02F0E54ECCDF08250010B66
:1015B00003E08250020B0DE16CECDBF00101010E47
:1015C000106F82B202D0040E106F050E006F006A19
:1015D0001DD0066A060E065C1EE20650040DF3508E
:1015E0008309006E050E065C02E1BB0E006E005022
:1015F000F5ECD9F01A080DE2F00E005C0AE26CEC92
:10160000DBF006C010F10101050E006F61ECE1F0A6
:1016100002D0062ADFD725822E88328A17ECD5F031
:1016200061E1D5CA03F0D251010B10E03751080B2C
:101630000DE0040E036E1BA009D0030E036E0A0119
:101640001C5104E1280E216F21CA1CFA0201D65157
:1016500019E00101170E0E6F010E006F035043ECED
:10166000CFF0EF5056ECCEF00101200E126F050EB8
:10167000006F035049ECCFF0EF5056ECCEF0010173
:10168000128F2FD06CECDBF00501170506E1C70EB9
:10169000E66EE10EE66E010E05D0C10EE66EE10EBD
:1016A000E66E010EE7ECC9F01BA009D003ECD3F005
:1016B000BC0EE66EE10EE66E010EE7ECC9F0050128
:1016C0001751050D07ECD6F0140E49260A0E4A22D2
:1016D00003508FECD8F002ECCEF0135102E1100E63
:1016E000136F2E883C0EB95D27E16CECDBF022B461
:1016F00006D0C70EE66EE10EE66E010E05D0C10EF5
:10170000E66EE10EE66E010EE7ECC9F02250040B26
:1017100001E0010E0201A46FA56B910EA427020E39
:10172000A52327ECD7F0EF50006E02ECCEF013515A
:1017300002E1100E136F2E880F0EB95D1DE1050E2C
:10174000006F51C100F061ECE1F00101158F135100
:1017500002E1100E136F0601426B010151510201AB
:101760000B5D05E20601700E426F5A0E436F0201D7
:10177000510EA46F010EA56F290E0101B95D0AE19A
:10178000775101E00480FAECD0F0770EA46F010EDF
:10179000A56F2E88260E0101B95D1AE1020E006FB9
:1017A0001E0E4325C4ECD9F00101006B1A0E43252F
:1017B000C4ECD9F00101136B100E146F120E156FEB
:1017C0000E5102E1100E0E6F0F5102E1100E0F6F5D
:1017D0003E0EB95D17E1050E006F420506E1B80E39
:1017E000E66EE10EE66E010E05D0B40EE66EE10E79
:1017F000E66E010EE7ECC9F00201420EA46F010E85
:10180000A56F2E80140E0101B95D1BE14FA305D019
:10181000040E006F96ECD8F00DD0006B640E54EC03
:10182000CDF05D0E006E01014FA102D0600E006E82
:10183000E6EC25F002014F0EA46F010EA56F030E1A
:10184000A66F150E0101B95D1EE1040E006F4FBBBE
:1018500011D01C0E0E6F160E0F6F240E106F0D0E92
:10186000116F5D0E006E4FA902D0600E006EE6ECA7
:1018700025F002D096ECD8F002014F0EA46F010EB5
:10188000A56F300EA66F330E0101B95D02E104ECC5
:10189000E4F0080E0101B95D1DE16CECDBF0010123
:1018A0005FB904808DEC80F06BECCAF083C33EF02E
:1018B0003CECFEF03EC012F13AC013F16BECCAF002
:1018C00084C33EF0A2ECD3F00101148FAFECD1F051
:1018D000100EA66F5CC305F005500DECCFF059EC6F
:1018E000D8F0440EB95D0BE1140E006E3FECDBF056
:1018F00002E0110E006E81EC80F0328A2E88450ED7
:101900000101B95D14E115ECD7F0496E4A6A1DEC8E
:10191000D8F0640DF1ECCCF0030E006F72EC26F001
:10192000060EE66E030E67ECCFF0328A2E88460E66
:101930000101B95D07E118ECD8F0006E32EC80F0DF
:10194000328A2E88480E0101B95D12E1A3ECD9F06C
:10195000006E040E08ECD4F0100E126FADECD9F04E
:1019600002E10E0E126FA8ECD9F0156F148F2E88BD
:10197000470EB95D1FE191ECD6F006E1FAECC9F033
:10198000B7ECD3F00A0803E1FAECC9F0EF92FAECF5
:10199000C9F0060EEB50006E005001E1002A61EC28
:1019A000E1F00101135102E1100E136F180E126FD6
:1019B000158F2E88490EB95D1DE1FAECC9F0B7EC20
:1019C000D3F0006E240E126F220E136F1E0E146FD2
:1019D00091ECD6F008E0010E0E6F1E0E0F6F240E74
:1019E000106F118F04D0005002E10528006E00C076
:1019F00015F12E88129E129C2E50100B07E01E50DF
:101A0000040B04E11B50080B01E1128C200EB95DA0
:101A100003E01C0EB95D05E1060EE66E050E67ECEF
:101A2000CFF02A0E0101B95D08E1135106E1100E55
:101A3000136F145102E1100E146F040EE15C02E208
:101A4000E16AE552E16EC2EFC9F047ECD5F0010161
:101A5000B951DE6EDD6A35ECCEF0070EEC02F3CF45
:101A6000EDFFEF02F3CFEEFFF450ED26026ABA0E5F
:101A7000496ED60E4A6E010E4B6E0250E76E000E96
:101A8000DFCF4CF0010EDBCF4DF0E7504C26000EBF
:101A90004D22CEECD5F0F550006E0FECE2F0022AAC
:101AA000070E025CE4E3020EE15C02E2E16AE55249
:101AB000E16EC2EFC9F012000201030E686FA46B61
:101AC000A56BA6691996D7ECD2F004E1E79DE79BD8
:101AD000D0EC0AF00601426B83ECDFF024B8C2D8E8
:101AE000FFECD2F003E03C0EB95D06E12050040BA0
:101AF00003E0209430ECCEF08CEC09F02DA454D00F
:101B00002D940E0E0101B95D1DE1339C83C100F0DF
:101B10000050010813E20004E66E2AECE4F0E552FE
:101B2000338CC80EF1ECC9F0E66AB3ECE4F0E55290
:101B3000000908E00201020E686F04D0E66A2AEC90
:101B4000E4F0E5521EA602D0E2EC35F01E96FAEC67
:101B50000DF00DEC0EF024A405D055ECCFF024943C
:101B6000FFECD3F01EA80BD01E980DC1E6FFCAEC07
:101B70005AF0E5520DC1E6FFE4EC5AF0E5522EA60C
:101B80000ED02E96C3EC5BF052ECCEF008E207ECE0
:101B9000CDF0FFECCEF074EC21F081EC2EF030AE05
:101BA00003D0309EE1EC77F018AC03D0189CACEC7D
:101BB000D4F01E9412007BEC0CF0299202013551F6
:101BC00001E1258A78EC16F02E942E92CEEC0CF0E2
:101BD0000601426B0101B59383ECDFF070EC6FF00E
:101BE0002D9C0201686B0C0E076EEBEC63F001019B
:101BF000129C3B51010B01E0128C129E3B51020BD7
:101C000001E0128E17A004D0E66A4D0E57ECCAF020
:101C10009C0E2CECCAF00101E79DE79B12000D50D1
:101C20000101B927B9AF02D0490EB96FB9514908BE
:101C300001E2B96B1200230EDFECCAF0020E006E57
:101C40001A0E155C05E1005068ECCBF0320EEF6E19
:101C500012000101AE6BD890AC33D890AC3328960B
:101C6000CCEFCDF007010B9F9BECC4F08DECD7F0CF
:101C7000209C33869FECD4F0249809ECCFF073EFCE
:101C800069F0E66AE66A3AECCEF00701086BD5EC3B
:101C9000C4F07FEC16F08A96208C33969FECD4F03B
:101CA00007010B8F9BEFC4F0C6ECC9F0100EE126C4
:101CB0003250200B14E01D50040B02E17DEF96F032
:101CC0001D50080B02E17DEF96F01EECCDF002E115
:101CD0007DEF96F0EEECD0F002E07DEF96F00201A1
:101CE0006851030A02E17BEF96F0010A1DE0030A46
:101CF00002E07DEF96F02D942E9024982E98329A43
:101D0000189C0101B5830201A46BA56BA669199605
:101D10004AECE3F01F960101269D279D0201020E69
:101D2000686F258278EC3DF02950020B16E02E50AA
:101D3000010B13E02E50100B10E131EC7AF02992D8
:101D40002F889CEC80F00101B58DB58F640EAC6FCF
:101D5000DFEC78F0B1DE57C2B9F117AE17EF96F0AD
:101D600072ECCFF0A4EC14F0FF0813E0BFEC14F019
:101D7000006E0101395105E01B0E005C02E19DEC93
:101D8000D8F00101B59BB599179E2582238A7DEF76
:101D900096F02E50100B12E01E50040B0FE11B505A
:101DA000080B0CE1090E155C09E00C0E155C03E153
:101DB0001750100B03E1FFEC08F004D00B0E155C7C
:101DC00004E17ADE179E7DEF96F017A0B9EF94F04C
:101DD00028B6BDEF94F0090E155C02E1C3EF94F054
:101DE00080ECCBF075E01750010B72E0100E155C23
:101DF00009E0110E155C06E0080E155C03E0290EE3
:101E0000155C66E11550DF6E91C2F9F692C2FAF6E2
:101E10008DC2F5F68EC2F6F68FC2F7F690C2F8F6CE
:101E2000080EDF5C03E0290EDF5C01E118844BEC57
:101E300097F0189481EC2EF0080EDF5C03E0290E79
:101E4000DF5C15E1110E0101B95D11E0230EB95DF2
:101E50000EE00068B3EC26F059ECD8F06EECCCF054
